:100000000C94C0090C940F0A0C940F0A0C940F0A5C
:100010000C940F0A0C940F0A0C940F0A0C940F0AFC
:100020000C940F0A0C94EE1D0C940F0A0C940F0AFA
:100030000C94B0390C940F0A0C940F0A0C940F0A0C
:100040000C940F0A0C940F0A0C947F190C940F0A4D
:100050000C94E10F0C940F0A0C94AB0F0C940F0A44
:100060000C94E0200C940F0A0C9422350C940F0A87
:100070000C94AD9E0C940F0A0C94A4940C940F0A4B
:100080000C940F0A0C940F0A0C940F0A07210C21F0
:1000900011211A213121482158216821A32132241C
:1000A0004821BF22D022FF221D233A239423EF238D
:1000B000DB269E274428BB28F3289629A52B062C4F
:1000C000802CB12C092D372D642DC72D112E5B2EC0
:1000D000542F41357535B835283640368136383796
:1000E000FF37FF37FF37FF37FF37FF37FF37FF3760
:1000F000FF37FF37FF37B437B637BB37D337D5377E
:10010000CE74BD7542766D759476C2760B759C750E
:10011000C2856686EB864D87A1870A885B8F8B88B0
:10012000BD88BD88BD88BD88BD88BD88BD88BD88A7
:10013000BD88EB886689F7891C8A5F8AB78A428BFB
:100140002B8C928C928C928C928C928C928C928C26
:10015000928C928CCA8CE88C0D8D698DA58D098E40
:10016000368ED68E5B8F368F368F368F368F368FA4
:10017000368F368F368FEB9CEE9CEE9CEE9CF79C78
:10018000FA9CFD9C0F9D0C9D0A0D3D3D3D3D3D3D66
:100190003D3D3D3D3D3D3D3D3D3D3D3D3D3D3D3D8F
:1001A0003D3D3D3D3D3D3D3D3D3D3D3D3D000A0D1F
:1001B000426174743A002025642043656C6C73209E
:1001C00000204C6F77207761726E696E673A202548
:1001D000642E2564000A0D466F756E6420424C2D16
:1001E0004374726C3A20002564000A0D0A0D212127
:1001F000204D495353494E4720424C2D4354524CB5
:100200003A202564202121000A0D43616C69627245
:100210006174696E6720707265737375726520739F
:10022000656E736F722E2E004F4B0A0D000A0D463D
:100230006C696768742D74696D65202575206D691A
:100240006E20546F74616C3A2575206D696E0041A3
:100250006E676C654E69636B202020202020204152
:100260006E676C65526F6C6C20202020202020412E
:1002700063634E69636B20202020202020202041D2
:100280006363526F6C6C2020202020202020205996
:1002900061774779726F2020202020202020204184
:1002A0006C746974756465205B302E316D5D20411E
:1002B00063635A2020202020202020202020204757
:1002C0006173202020202020202020202020204377
:1002D0006F6D706173732056616C756520202056B8
:1002E0006F6C74616765205B302E31565D20205243
:1002F00065636569766572204C6576656C2020477C
:1003000079726F20436F6D70617373202020204DD0
:100310006F746F7220312020202020202020204D5B
:100320006F746F7220322020202020202020204D4A
:100330006F746F7220332020202020202020204D39
:100340006F746F7220342020202020202020205025
:10035000414E2D436F73202020202020202020504C
:10036000414E2D53696E2020202020202020205037
:10037000414E2D536572766F20202020202020537F
:100380006572766F2D526F6C6C20202020202053D8
:100390006572766F2D4E69636B20202020202048E7
:1003A0006F76657267617320202020202020204313
:1003B000757272656E74205B302E31415D20204372
:1003C00061706163697479205B6D41685D202048CC
:1003D000656967687420536574706F696E74203244
:1003E00035202020202020202020202020202032E6
:1003F00036202020202020202020202020202043C4
:100400006F6D7061737320536574706F696E74499A
:1004100032432D4572726F7220202020202020420E
:100420004C204C696D69742020202020202020471A
:1004300050535F4E69636B202020202020202047EE
:1004400050535F526F6C6C202020202020202021F0
:10045000212120494E434F4D50415449424C4520A3
:10046000212121002A002E000A0D20444143206F43
:100470007220493243204552524F52212043686531
:10048000636B204932432C2033567265662C20441E
:10049000414320616E6420424C2D4374726C005BBA
:1004A00025695D005B25695D002B204D696B726FCE
:1004B0004B6F70746572202B0048573A5625642E96
:1004C00025642053573A25642E256425632056342D
:1004D0000053657474696E673A2564202573004D76
:1004E00069786572204572726F72210045525225FB
:1004F00032643A00486172647761726520457272B5
:100500006F7220313A2564202121004D697373698F
:100510006E6720424C2D4374726C3A256421210091
:10052000493243204552524F5221212100486569EA
:100530006768743A202025356900536574706F69C7
:100540006E743A2535690050726573737572653A39
:10055000253569004F66667365743A202025356934
:10056000002841290048656967687420636F6E74CC
:10057000726F6C0044495341424C454400616374BE
:100580002E2062656172696E67004E69636B3A2066
:10059000202020202025356900526F6C6C3A2020E5
:1005A0002020202025356900436F6D706173733AF8
:1005B000202020253569004B25693A253469202003
:1005C0004B25693A25346920004E693A2534692063
:1005D00020526F3A253469200047733A2534692048
:1005E0002047693A253469200050313A2534692082
:1005F0002050323A253469200050333A253469209E
:100600002050343A25346920004779726F202D201C
:1006100053656E736F72004E69636B2534692028D1
:100620002533692E25692900526F6C6C25346920A9
:10063000282533692E2569290047696572253469A3
:10064000202825336929004E69636B2025346920F1
:10065000282533692E25782900526F6C6C202534AB
:100660006920282533692E257829005961772020B3
:10067000253469202825336929004E69636B2025BC
:100680003469202825336929282533692900526FC8
:100690006C6C202534692028253369292825336985
:1006A00029005961772020253469202825336929BC
:1006B000282533692900414343202D2053656E735B
:1006C0006F72004E69636B202534692028253369D9
:1006D0002900526F6C6C2025346920282533692944
:1006E000005A20202020253469202825336929003C
:1006F000566F6C746167653A2020202533692E257A
:100700003169560043757272656E743A2020202557
:1007100033692E2531694100506F7765723A202088
:10072000202020253469570044697363686172672B
:10073000653A202535696D416800526563656976C3
:1007400065720052432D5175616C6974793A2025A8
:1007500034690052432D4368616E6E656C733A25AF
:10076000346900436F6D70617373004D61676E652E
:10077000743A202020253569004779726F3A20208D
:1007800020202025356900536574706F696E743AB6
:100790002025356900506F746925693A202025337A
:1007A0006900506F746925693A2020253369005328
:1007B0006572766F202000536574706F696E7420C7
:1007C0002025336900506F736974696F6E3A202574
:1007D00033690052616E67653A2533692D253369A7
:1007E00000424C2D4374726C204572726F727320FC
:1007F00000253364202533642025336420253364A9
:100800002000424C2054656D70657261747572658C
:100810000025336420253364202533642025336488
:100820002000424C2D4374726C20666F756E6420FC
:100830000020256320202025632020202563202000
:1008400020256320002025632020202563202020F0
:100850002563202020256320002025632020202DD3
:100860002020202D2020202D20003130003131008B
:10087000313200466C696768742D54696D652020BB
:1008800000546F74616C3A2535756D696E00416373
:10089000743A20202535756D696E00287265736580
:1008A0007429000A0D2D2D3E204861726477617213
:1008B000652056657273696F6E20427974652043B6
:1008C00068616E676564203C2D2D000A0D47656EDA
:1008D00065726174696E672064656661756C742009
:1008E000506172616D657465722053657420256472
:1008F000000A0D5573696E6720506172616D6574F1
:10090000657220536574202564000A0D47656E6585
:10091000726174696E672064656661756C74204DE0
:1009200069786572205461626C65000A0D4D6978C2
:1009300065722D436F6E6669673A202725732720FD
:10094000282575204D6F746F727329000A0D41437D
:1009500043206E6F742063616C69627261746564B8
:10096000210D0A0000008F001E01AD013B02CA02EA
:100970005803E603740402058F051B06A706330718
:10098000BE074808D2085B09E3096B0AF20A780B34
:10099000FD0B810C040D860D070E870E060F840FCC
:1009A00000107B10F5106E11E5115B12CF1242138F
:1009B000B31323149214FE146A15D3153B16A11613
:1009C00005176717C81727188318DE1837198E19E7
:1009D000E319361A871AD61A231B6E1BB61BFD1B8A
:1009E000411C831CC31C001D3C1D751DAB1DE01D5F
:1009F000121E421E6F1E9A1EC31EE91E0D1F2E1FC1
:100A00004D1F691F841F9B1FB01FC31FD31FE11FF2
:100A1000EC1FF51FFB1FFF1F002006010000147CC8
:100A2000000201015A7D01030202EE7D020403036C
:100A3000967E030504044B7E04060505357F0500FC
:100A400006067F7F2532692E2531695600253364DD
:100A5000256320253033646D2563005374617475FC
:100A600073004552524F523A20253264200053659C
:100A70007425643A257320200025346920253269C5
:100A80003A25303269002534696D256300253369C4
:100A900020253369202533692025336900253369F2
:100AA0002025336920253369202533690054656D7D
:100AB0007065726174757265732020202000256353
:100AC000432020202020002532692E253169562020
:100AD0002533692E25316941002534695720253693
:100AE000696D4168004D61676E65743A253369250B
:100AF0002520253369256300496E636C692E3A25EC
:100B000033692563202825692920002532756D2F3A
:100B100073205361743A2564200020203344004E32
:100B20006F4678004447505300486F6D653A25334F
:100B3000646D202533642563202563004E6F204EAD
:100B40006176694374726C21003E2533693D5365BB
:100B50007269616C706F7431003E2533693D536575
:100B60007269616C706F743200000005000500044A
:100B70000106010800060102000400040007000746
:100B80000007000700070007000700030103010535
:100B90000017010F01060009010A011901050105ED
:100BA0000119011A010F0100004E6F204572726F8A
:100BB000722020202020202020004E6F7420636FA0
:100BC0006D70617469626C652020004D4B334D611E
:100BD00067206E6F7420636F6D7061004E6F2046EA
:100BE0004320636F6D6D756E6963617400436F6D53
:100BF0007061737320636F6D6D756E69630047502C
:100C00005320636F6D6D756E69636174696F006306
:100C10006F6D706173732076616C756520202000A4
:100C20005243205369676E616C206C6F737420208F
:100C300000464320737069207278206572726F726B
:100C400020004E6F204E4320636F6D6D756E69639B
:100C50006174004643204E69636B204779726F20B0
:100C600020202000464320526F6C6C204779726F21
:100C70002020202000464320596177204779726F59
:100C80002020202020004643204E69636B204143F2
:100C900043202020202000464320526F6C6C2041CE
:100CA00043432020202020004643205A2D41434327
:100CB0002020202020202020005072657373757240
:100CC000652073656E736F7220004932432046437E
:100CD0002D3E424C2D4374726C2000426C204D69B5
:100CE0007373696E67202020202020004D6978658D
:100CF00072204572726F72202020202000436172A2
:100D00006566726565204572726F722020004750DB
:100D10005320466978206C6F737420202020004D8A
:100D200061676E6574204572726F7220202020000A
:100D30004D6F746F7220726573746172742020201D
:100D400000424C204C696D69746174696F6E20209B
:100D500020004750532052616E67652020202020DC
:100D60002020004E6F2053442D43617264202020C8
:100D70002020200053442D4C6F6767696E67206503
:100D800072726F7200466C79696E672072616E676D
:100D90006521202020004D617820416C74697475B4
:100DA000646521202020004E6F2047505320666943
:100DB0007820202020202000636F6D7061737320E5
:100DC0006E6F742063616C2E0053657420203A00AE
:100DD000202121204C69506F20766F6C746167650B
:100DE00020212120200020202020204D696B726FBF
:100DF0004B6F70746572202020202000202020205E
:100E000020202020202020202020202020202020E2
:100E1000200020202532692E25316956202000200F
:100E2000202532692E25316956202000414C543A44
:100E30002534696D20256300414C543A2534696D91
:100E4000202000414C543A2D2D2D2D20002020250E
:100E500032693A2530326920200020202532693A53
:100E6000253032692020004449523A202533642538
:100E70006300430020002020253569202000202029
:100E8000253569202000493A2532692E25316941EE
:100E900020003A003A003A002D2D2D2D2D2D2D2D1C
:100EA0002D2B2D2D2D2D2D2D2D2D2D2D2D002D2DA1
:100EB0002D2D2D2D2D2D2D2D2D2D2D2D2D2D2D2D62
:100EC0002D2D2D003A005341543A25326420004420
:100ED0004953543A2533646D0044200033440021C3
:100EE00021004D41473A25337525252000484D3ACC
:100EF000253364256320256300696E636C3A2532CF
:100F00006425632825326929002020202025327598
:100F10006D2F733A2020484D3A25336425632025F0
:100F200063004552523A2025326420210045525236
:100F30003A20002121204C69506F20766F6C74613B
:100F4000676520212100207777772E4D696B726FBE
:100F50004B6F707465722E64652020002025326905
:100F60003A2530326920202532692E2531695620F4
:100F70002534696D416800202532693A253032698F
:100F800020202532692E25316956202534696D418E
:100F900068004449523A253364256300414C543A71
:100FA0002534696D00414C543A2534696D00414C3B
:100FB000543A2D2D2D2D2000256300484D3A253320
:100FC0006425632020444953543A2533646D202519
:100FD00063005057523A2532692E25316941202845
:100FE0002569572920004346002020004750533AE6
:100FF0002532756D2F73205341543A25642000200B
:1010000020334420004E4F46495800444750532057
:10101000002020204E6F204E6176694374726C2050
:10102000202020202020002532692E25692025320D
:10103000692E2569202532692E2569202532692EE1
:10104000256941002533692025336920253369202E
:10105000253369256343002532692E256920253211
:10106000692E256941002532692E256920253269BE
:101070002E2569202532692E2569202532692E25E5
:1010800069410025336920253369256343202020E9
:101090002020202020002533692025336920253396
:1010A0006920253369256343004552523A20253291
:1010B000642021004552523A20002121204C6950E1
:1010C0006F20766F6C74616765202121002077772F
:1010D000772E4D696B726F4B6F707465722E6465FD
:1010E00020200053657474696E673A257520257356
:1010F00020004D696E3A2532692E2531695620252A
:10110000732000414C543A00504F54493A253375EE
:101110002000284F4E29202000284F464629200035
:101120004C494D495400564152494F00444953419E
:10113000424C45440043463A0044495341424C45E1
:10114000440020284F4E29200020284F46462900E1
:10115000205445414348004750533A0044495341C5
:10116000424C4544002846524545290028484F4DE9
:101170004529002841494429200028484F4C44294A
:10118000002046533A257573656B2000484F4D4546
:1011900020414C543A0025756D00484F4C442000C6
:1011A0004E693A25346920526F3A25346920433A12
:1011B0002533690047733A2534692059613A25344B
:1011C00069200050313A2534692050323A2534697B
:1011D00020333A2533690050343A2534692050359C
:1011E0003A25346920363A25336900434F55504C2F
:1011F000494E47204F46462120004C4F4F50494E04
:10120000472120004848212000434F4D504153536F
:10121000204F4646212000004F5051525354535600
:101220005748005859005A554546474841004942D9
:101230004A4A0000000000000000000000444C4D3D
:1012400000000000004E0000004B00430A0D7777BD
:10125000772E4D696B726F4B6F707465722E64657B
:101260002028632920486953797374656D7320477A
:101270006D6248000A0D74686520757365206F669D
:10128000207468697320736F667477617265206972
:1012900073206F6E6C79207065726D69747465640B
:1012A000200A0D6F6E206F726967696E616C204D48
:1012B000696B726F4B6F707465722D4861726477E1
:1012C000617265005573657200486F54542056343E
:1012D000004143542044534C004A657469005370E4
:1012E000656B7472756D0050504D000A0D52656348
:1012F00065697665723A2000532E42757300756EEB
:101300006B6E6F776E2E205573696E672050504D4F
:101310002E2E2E006E6F7420737570706F72746550
:101320006420627920686172647761726521000AC5
:101330000D466C69676874436F6E74726F6C0A0D4A
:1013400048617264776172653A25642E25640A0DDE
:10135000536F6674776172653A5625642E2564254D
:101360006320000A0D202D204C4942204E4F54206E
:10137000434F4D50415449424C45202121212100E9
:1013800011241FBECFEFD0E4DEBFCDBF13E0A0E03D
:10139000B1E0EAE2F3E401E00BBF02C007900D9276
:1013A000A030B107D9F71CE0A0E0B3E001C01D9266
:1013B000A43DB107E1F77AEAE2E0F0E081E2809350
:1013C0005700D4907E010894E11CF11C20EF37EF08
:1013D00041E050E087016FE0DA01C9012F5F3F4F24
:1013E0004F4F5F4FABBFFC018791F80181938F0195
:1013F000615067FFF1CFF7016EE08191782770951A
:10140000615067FFFACF8889781729F0F7E9DF166E
:1014100011F40000FECF0E94DB0A0C9494A10C94FE
:10142000000088E891E09F938F938AE596E19F936F
:101430008F93E091B805F091B90509950F900F9041
:101440000F900F90089580915D08E82FFF27EE0F11
:10145000FF1FEE56F64F808191818D5E9F4F14F0F5
:1014600010920301808191818A5B9F4FCCF480911F
:1014700003018823A9F481E0809303018091EC05A6
:101480008F5F8093EC05853038F088EE93E0909381
:10149000380380933703089566E970E00E94403D69
:1014A00008951F93CF93DF93182F882389F08EEA36
:1014B00091E09F938F938AE596E19F938F93E091BC
:1014C000B805F091B90509950F900F900F900F9006
:1014D00080918008823308F044C084EF91E00E943C
:1014E000611AEC01112329F0CE010E946A1A8823A7
:1014F000D9F3C2E0D0E026E530E08091220190915E
:1015000023018217930730F02196255D3F4FC730A6
:10151000D10598F3809180089927C89F9001C99FB1
:10152000300DD89F300D1124209301011123D9F0E3
:1015300068EC70E08C2F0E94403DDF93CF9386EBE8
:1015400091E09F938F938AE596E19F938F93E0912B
:10155000B805F091B90509958DB79EB706968DBF70
:1015600002C080930101112311F1809101016AE011
:101570000E94E7A0892F99279F938F938091010163
:101580000E94E7A099279F938F9381EC91E09F930E
:101590008F938AE596E19F938F93E091B805F09140
:1015A000B90509952DB73EB7285F3F4F2DBFDF9195
:1015B000CF911F910895CFEFD0E4DEBFCDBF882437
:1015C0009924C1E07C2E14B815B88AE08AB98FE559
:1015D0008BB9B7EEEB2EB3E0FB2E2EEC3FEFE20E15
:1015E000F31EF7FEFACF6624199B08C04C9B04C07B
:1015F00085E18093020108C086E101C087E1809304
:10160000020181E080931D0481E887B93E9A8FEF43
:1016100088B98BE184B981E085B9469A84B7877F20
:1016200084BF8091600088618093600010926000A8
:1016300084EC99E0909338038093370310926F0401
:1016400010926E04109297091092960910927104EC
:10165000109270041092730410927204209102018F
:10166000243128F084EC94E0A0E0B0E004C08BE0EA
:1016700095E0A0E0B0E080933E0190933F01A093FD
:101680004001B09341012A3011F0243110F0289824
:1016900001C0289A2C3010F0273111F4299A01C08A
:1016A00029980E94CA1A0E949B1A0E9462160E94E0
:1016B00073390E94711F81E00E94D6340E947473B6
:1016C0000E94228083E00E94639D809102018C3001
:1016D00010F0873111F4299A01C0299878940E945A
:1016E000BD338091800382608093800310928303D6
:1016F0000E94484984EF91E00E94611A7C01809128
:10170000800380FD05C0C7010E946A1A8823B9F3CF
:1017100085ED91E09F938F93AAE5AA2EA6E1BA2EBC
:10172000BF92AF92E091B805F091B905099580EAB2
:101730009FE00E94611A7C01C0E0D0E00F900F9002
:101740000F900F9004E319E0F8EECF2EF8E0DF2EB3
:101750000E9448498091800380FD05C0C7010E9416
:101760006A1A8823B9F3F60180811816ACF40BC00D
:101770000E9448498091800380FD05C0C7010E94F6
:101780006A1A8823B9F3C7010E946A1A882321F4D0
:10179000F8018081882364F7F801808187FF19C0F0
:1017A0002196DF93CF93219787EE91E09F938F93BC
:1017B000BF92AF92E091B805F091B905099580917B
:1017C00001038F5F809301032DB73EB72A5F3F4F20
:1017D0002DBF219684E090E0C80ED91E085F1F4FF0
:1017E000CC30D10508F4B4CFC0E0D0E001E319E07B
:1017F000E8EEEE2EE8E0FE2EF801838187FD1DC0A5
:10180000F70180811816CCF42196DF93CF932197AE
:101810008AEE91E09F938F938AE596E19F938F9351
:10182000E091B805F091B905099582E08093350300
:101830002DB73EB72A5F3F4F2DBFF80183818078D7
:101840008383219624E030E0E20EF31E085F1F4FF1
:10185000CC30D10588F20E94110A90915B088091EA
:101860000103981728F48091D20580618093D205F6
:1018700088E092E09F938F93CAE5D6E1DF93CF9300
:10188000E091B805F091B905099588EE93E00E94C2
:10189000611A7C010E94771F0F900F900F900F909C
:1018A000C7010E946A1A8823D9F388E292E09F93C5
:1018B0008F93DF93CF93E091B805F091B905099527
:1018C00080E00E94243E809102010F900F900F90C3
:1018D0000F908A3011F0843110F0289801C0289AB6
:1018E00080ED97E0909338038093370385E58093EC
:1018F000EE058EE090E00E94DD319927182F002739
:101900008FE090E00E94DD31080F111D1093070356
:10191000009306038AE090E00E94DD319927182F9A
:1019200000278BE090E00E94DD31080F111D10931D
:101930000503009304030F5F1F4F39F080910603E6
:10194000909107038F5F9F4F41F41092070310920D
:1019500006031092050310920403809104039091F2
:1019600005039F938F9380910603909107039F93A4
:101970008F938DE292E09F938F93DF93CF93E091CB
:10198000B805F091B90509950E944D2688E893E1C4
:101990009093390180933801C1E0C093ED058C2FFD
:1019A0000E94510A809183080E94AF9C0E94110AF4
:1019B00080ED97E00E94611A7C018AEF90E00E941E
:1019C000611A83E08093B507109200038091CC08E0
:1019D0002DB73EB7285F3F4F2DBF84FF02C0C09395
:1019E000080312BC11BC80910A03882311F04798A8
:1019F000FECF80913B03882309F49EC2809114019D
:101A0000882309F499C210923B038091EC05882346
:101A100019F00E94230A02C00E94F34C0E94484918
:101A2000209102012A3011F0243110F0289801C0D1
:101A3000289A80916204882331F080916204815059
:101A4000809362040EC080916F00806280936F006B
:101A500010929309109292098091D2058860809328
:101A6000D205809138019091390101979093390105
:101A7000809338018091380190913901892B21F0B0
:101A8000809181038823C9F18091380190913901B7
:101A9000892BD9F40E94003585E090E090933901BC
:101AA000809338018091EF079091F0070196909311
:101AB000F0078093EF078091D20581608093D20573
:101AC0008091B60782608093B60780910A01909159
:101AD0000B018F5F9F4FC1F4809161048823A1F0B7
:101AE00088EA91E6909338038093370380E890E08A
:101AF00090930B0180930A0107C02A3011F0243122
:101B000010F0289801C0289A0E94309E80913B03D3
:101B1000882309F00FC280918505882319F00E945F
:101B2000DB8F08C280911201882311F00E94231BD1
:101B30000E94AB160E943112C7010E946A1A8823C4
:101B400009F4F4C184E190E0E80EF91E0E94E11A64
:101B500080918308863019F40E94868504C0843001
:101B600011F40E94AB9080911D04882331F1809183
:101B7000FC079091FD078C52914074F08091C5074D
:101B80009091C60780509240C4F48091FC079091D8
:101B9000FD07835593408CF0639432E3361570F45F
:101BA00080916104882331F08091D1058062809317
:101BB000D10504C080934D0401C066248091810347
:101BC000882349F08091D20582608093D20580916C
:101BD000B60782600FC08091370390913803892B3C
:101BE00059F48091380190913901079728F080913C
:101BF000B6078D7F8093B60780910803882361F034
:101C000080916204873940F01092080388E893E1DC
:101C1000909338038093370380910501882321F046
:101C20008150809305012EC08093F80510923504F1
:101C30001092340410923304109232041092310442
:101C400010923004809162048823E1F480910A01AB
:101C500090910B018F5F9F4FA9F4209108032230D0
:101C600089F088E99AE3909338038093370380E002
:101C70009CE090930B0180930A01222319F082E0EB
:101C8000809308038091C101893C70F0815080935A
:101C9000C1018091D2058B7F8093D2058091D505BB
:101CA00081608093D50551C080919B0A8823F9F00B
:101CB0008091D20584608093D20589E080934805A5
:101CC00080910A0190910B018F5F9F4F81F4809169
:101CD0006104882361F088E99AE390933803809344
:101CE000370380E098EA90930B0180930A011092E9
:101CF0003A05109239051092380510923705109266
:101D0000360510928E0A8FEF8093030B1092CD0A46
:101D10001092CC0A1092CF0A1092CE0A8FEF9FEF4A
:101D20009093CB0A8093CA0A1092510410925204E5
:101D30001092530410925404109255048091D505CA
:101D40008E7F8093D5051092C10180910101282FCB
:101D50003327809122019091230182179307CCF4BD
:101D60008091250480628093250480910A019091DE
:101D70000B018F5F9F4FC1F480E797E19093380389
:101D80008093370380E093E090930B0180930A01E6
:101D90000BC08091370390913803892B29F48091EF
:101DA00025048F7D8093250483E08093360312BC45
:101DB00011BC809109038F5F80930903813309F07F
:101DC0006CC01092090380917205882319F081502C
:101DD000809372058091250481FF0AC080910203DF
:101DE000909103030196909303038093020304C030
:101DF0005AEA852E55E0952E80912604909127046D
:101E00008050944008F049C02091FE073091FF07B0
:101E1000409100085091010880911A0190911B0196
:101E2000A0911C01B0911D01281739074A075B07D3
:101E300064F48091FE079091FF07A0910008B09193
:101E400001080596A11DB11D20C02091FE0730910B
:101E5000FF07409100085091010880911A0190916C
:101E60001B01A0911C01B0911D0182179307A407CB
:101E7000B5079CF48091FE079091FF07A0910008A0
:101E8000B09101080597A109B1098093FE079093CD
:101E9000FF07A0930008B09301080894811C911CCF
:101EA00082E788168BE0980609F040C088249924C0
:101EB00020910603309107032F5F3F4F30930703B4
:101EC000209306038091040390910503019690935B
:101ED000050380930403832F9927682F8EE090E0F9
:101EE0000E94E53180910603909107039070682F5E
:101EF0008FE090E00E94E53180910403909105030A
:101F0000892F9927682F8AE090E00E94E53180911F
:101F10000403909105039070682F8BE090E00E947D
:101F2000E53184E190E00E94611A7C010E94B8785A
:101F30000E94398071107A94772029F40E94817868
:101F40008CE0782E50CD80913603882309F04BCD5C
:101F50000E94957348CD1F920F920FB60F921124D5
:101F60008F939F93EF93FF93809107018823E1F470
:101F700080912403909125030196909325038093EB
:101F80002403FC01E752F94FE081ED3019F08C3D5C
:101F9000910539F4109225031092240381E0809377
:101FA0000701E093C60004C0109225031092240399
:101FB000FF91EF919F918F910F900FBE0F901F9007
:101FC00018951F920F920FB60F9211242F933F93E3
:101FD0004F935F936F937F938F939F93AF93BF9331
:101FE000CF93EF93FF9390E080910A03813029F41F
:101FF0008091C6008093CE00CCC080910A038230CD
:1020000029F48091C6008093FB05C3C08091C6006F
:1020100080931C0350912A035C3D10F090932B0396
:1020200080911C038D3009F065C080912B038230B4
:1020300009F060C090932B03852F992785509A4F04
:10204000FC01329740812091260330912703241B05
:102050003109DC0111978C91281B3109C9019F704E
:10206000909327038093260346E0969587954A959B
:10207000E1F7982F935C909328032F733070235CC3
:10208000209329038081981729F48C91281711F443
:1020900091E006C090E0809119038F5F809319034F
:1020A000C0911B03CC2309F074C0992309F471C0BB
:1020B00081E080931B03580F509318035150E52F74
:1020C000FF27E550FA4F8DE080838091FD05823532
:1020D00009F05FC00E944D2688E190E02CE00FB629
:1020E000F894A895809360000FBE20936000C09381
:1020F00035034FC020912B03822F99278130910502
:10210000F9F0823091051CF4892B21F040C0029730
:1021100011F13DC080911C03833239F480911B037F
:10212000882319F481E080932B0380911C03809312
:10213000FB0581E080932A0380911C03992722C02C
:102140002F5F20932B03E52FFF27E550FA4F809157
:102150001C03808309C0E52FFF27E550FA4F8091CB
:102160001C0380835C3D20F45F5F50932A0302C010
:1021700010922B0320911C0380912603909127033A
:10218000820F911D909327038093260302C0109223
:102190002B03FF91EF91CF91BF91AF919F918F91C1
:1021A0007F916F915F914F913F912F910F900FBE53
:1021B0000F901F901895AC01A0E0B0E09D01A8170A
:1021C000B90748F4E9EDF6E08191280F311D119629
:1021D000A417B507C8F33F70FD01E752F94FC901D5
:1021E00056E0969587955A95E1F7835C8083119622
:1021F000FD01E752F94F2F733070822F835C80838B
:10220000A652B94F8DE08C93109207018091D906A8
:102210008093C6000895A0E0B0E0E1E1F1E10C9404
:1022200060A12C859D850E85BB2483E28093D90611
:102230009F599093DA062093DB0633E0E32EF12CCE
:10224000002309F49EC0CF84D888BE016D5E7F4F05
:10225000A989BA890150109709F493C01097B9F071
:10226000F601EB0DF11DB3949081119791F40023C9
:1022700049F1FB016E5F7F4FDB01C080D1806E5F53
:102280007F4F0D90BC91A02DBB24015002C090E067
:1022900019C01097B9F0F601EB0DF11DB394408110
:1022A000119791F4002341F1FB016E5F7F4FDB0139
:1022B000C080D1806E5F7F4F0D90BC91A02DBB245C
:1022C000015002C040E018C01097B1F0F601EB0DCC
:1022D000F11DB3941081119781F4002371F0FB017B
:1022E0003296DB01CD90DC90BF016E5F7F4FA08105
:1022F000B181BB24015001C010E0F701E752F94F52
:10230000892F86958695835C80830894E11CF11C57
:10231000F701E752F94F892F99278370907024E0D5
:10232000880F991F2A95E1F755279A0194E0369571
:1023300027959A95E1F7822B835C80830894E11CB2
:10234000F11CF701E752F94F4F705070440F551FC1
:10235000440F551F812F992726E0969587952A953A
:10236000E1F7842B835C80830894E11CF11CF70166
:10237000E752F94F1F73135C10830894E11CF11CA2
:102380006ACFC7010E94DB10E9E00C947CA1A3E0B6
:102390007A2F409118034650442309F458C0E72F80
:1023A000FF27E550FA4F80818D537F5FE72FFF278E
:1023B000E550FA4F20812D537F5FE72FFF27E5502F
:1023C000FA4F30813D537F5FE72FFF27E550FA4FEB
:1023D00060816D537F5F9927880F991F880F991F20
:1023E000522F52955F70582B822F99278F709070C3
:1023F000F4E0880F991FFA95E1F7232F269526958B
:10240000282B832F992783709070E6E0880F991FFF
:10241000EA95E1F7682B41504F3FC9F0EA2FFF27BB
:10242000E550FA4F5083AF5F41504F3F81F0EA2FA4
:10243000FF27E550FA4F2083AF5F41504F3F39F0FF
:10244000EA2FFF27E550FA4F6083AF5FA5CF8EEFED
:1024500095E09093170380931603A350A093150360
:102460000895A2E0B0E0E7E3F2E10C9466A1809168
:102470001B03882309F41AC40E94C7118091FC052C
:10248000823609F0E6C28091FD05992780379105D3
:1024900009F4ABC081379105C4F48A36910509F47B
:1024A00043C28B36910544F48B34910571F1863625
:1024B000910509F470C1CDC28D36910509F469C04A
:1024C0008E36910509F44DC0C4C28437910541F19F
:1024D000853791054CF48137910509F48DC0833718
:1024E000910509F4E0C0B5C28737910509F4DEC152
:1024F000883791052CF48537910509F49AC1A9C252
:102500008937910509F47FC1A4C2E0911603F091C7
:102510001703808191819093AE018093AD0199C2A0
:1025200080911803A0911603B0911703853140F0F4
:1025300080E1E6EDF5E00D9001928A95E1F70DC09E
:102540008D919D910D90BC91A02D8093D605909377
:10255000D705A093D805B093D90580EF80931303D6
:1025600047C0809107018823E1F38DE490E09F93B9
:102570008F938BED98E09F938F9381E08F938F9350
:102580008EE48F930E940B118DB79EB707968DBF77
:1025900060C2A0911603B09117031C91113081F411
:1025A0008DE4EBEDF8E00D9001928A95E1F70E9441
:1025B000F83219838091D2058F7E8093D20501C0B5
:1025C0001982809107018823E1F381E090E09F93D5
:1025D0008F93CE0101969F938F9381E08F938F937A
:1025E0008DE48F930E940B1109C181E080931E033B
:1025F0008FEF809305012DC280916104882309F03B
:1026000028C2E0911603F0911703E0818E2F8A50C3
:102610008A3058F48983882311F481E003C086301E
:1026200010F085E0898361E00EC08E2F84518A30DE
:1026300070F48983882311F481E003C0863010F0A0
:1026400085E0898360E089810E947A3312C0E98342
:10265000EF3F19F40E945B3389838981882311F449
:1026600081E003C0863010F085E0898389810E9473
:10267000FB31809107018823E1F38EE790E09F937F
:102680008F938CE598E09F938F9381E090E09F93E8
:102690008F93CE0101969F938F9382E08F9381E079
:1026A0008F9381E539C12091160330911703D90129
:1026B0008C918150853008F045C0F90181818F35BA
:1026C00009F040C0809161048823E1F52F5F3F4FFE
:1026D0008EE7ECE5F8E0D9010D9001928A95E1F7DB
:1026E000F90182910E94683280919D089927AA275A
:1026F000BB27BC01CD0124EC39E040E050E00E9452
:10270000C8A0DC01CB018093A5019093A601A09302
:10271000A701B093A80180919E089927AA27BB27FB
:10272000BC01CD010E94C8A0DC01CB018093A101B6
:102730009093A201A093A301B093A4010E945B33E4
:10274000898301C01982809107018823E1F381E028
:1027500090E09F938F93CE0101969F938F9381E09A
:102760008F938F9383E58F930E940B118DB79EB744
:1027700007968DBF80916104882329F46EE670E08E
:1027800089810E94403D80E00E94510A8091830827
:102790000E94AF9C5EC180916104882309F059C1F9
:1027A000E0911603F0911703E0818E2F8150853060
:1027B00018F48E2F0E94FB310E945B338983809135
:1027C00007018823E1F381E090E09F938F93CE018E
:1027D00001969F938F9381E08F938F9386E48F93DD
:1027E0000E940B116EE670E089810E94403D80E0FE
:1027F0000E94510A809183080E94AF9CADB7BEB77A
:102800001796ADBF26C119822981A0911603B091F8
:102810001703E2E9F9E08D91992787FD909593A33D
:1028200082A3822F8F5F8983282F32968C3098F372
:1028300010C1E0911603F091170380810E94CC38FB
:102840008A83882319F481E0898301C019828091E9
:1028500007018823E1F388E090E09F938F9389E25A
:1028600099E09F938F9321E030E03F932F938091E5
:102870001603909117039F938F933F932F93CE014D
:1028800002969F938F933F932F93CE01820F931FB6
:102890009F938F9384E08F9381E08F9385E58F934F
:1028A0000E940B11EDB7FEB773963CC080911503E3
:1028B000893008F4CEC020911603309117032F5FA2
:1028C0003F4F88E0A9E2B9E0F90101900D928A95A5
:1028D000E1F7D9018E910E9422388A83882319F466
:1028E00081E0898301C01982809107018823E1F387
:1028F00021E030E03F932F93CE0102969F938F9378
:102900003F932F93CE01820F931F9F938F9382E06B
:102910008F9381E08F9387E58F930E940B11EDB722
:10292000FEB73B96EDBF95C080916104882309F006
:1029300090C00E94669C8983823019F0843009F02F
:1029400088C020E430E0F8948091C1008F738093B8
:10295000C1008091C9008F738093C9008091C1002C
:10296000877E8093C1008091C900877E8093C900D3
:102970008091C80087FF03C08091CE00F9CF80917D
:10298000C00087FF03C08091C600F9CFE091160315
:10299000F0911703E081E13021F482E080930A0393
:1029A0002EC0E43611F421E830E081E080930A0380
:1029B000832F99278093CD002093CC008091CD0068
:1029C0008093C5008091CC008093C4008091CA00A0
:1029D0008F7D8093CA008091CA008F7E8093CA0049
:1029E0008091C9008B7F8093C9008091CA00846068
:1029F0008093CA008091CA0082608093CA0080914F
:102A0000CA00877F8093CA008091C200877F80932D
:102A1000C2008091C9008E7F8093C9008091C1005F
:102A200088618093C1008091C90088618093C9004A
:102A30008091C10080688093C1008091C900806846
:102A40008093C90010926E0010926F001092700077
:102A500078948091FD0599278436910509F4BBC0CF
:102A600085369105ACF48136910509F46FC0823644
:102A700091052CF48B34910509F45DC00FC18236A9
:102A8000910509F470C08336910509F47FC006C131
:102A90008C36910509F4EDC08D3691054CF48736DE
:102AA000910509F4F8C08836910509F4B2C0F6C062
:102AB0008437910529F08637910509F4E8C0EEC006
:102AC00080911803A0911603B0911703803140F054
:102AD00080E1E6EDF5E00D9001928A95E1F70DC0F9
:102AE0008D919D910D90BC91A02D8093D6059093D2
:102AF000D705A093D805B093D90580910701882305
:102B0000E1F31F92809104018F9384E58F930E94DB
:102B10000B118AEF809313038FEF8093050180EAF6
:102B20009FE00E94611A90930C0380930B030F9017
:102B30000F900F90B3C0E0911603F09117038081BE
:102B400091819093AE018093AD01A8C0E0911603EE
:102B5000F0911703808180930601803298F08FE115
:102B6000809306010FC0A0911603B09117038BE06C
:102B7000EEEEF5E00D9001928A95E1F78091F70570
:102B80008093F7078FEF8093050188C080910F0332
:102B900090911003892B89F4E0911603F0911703AB
:102BA000E081EE2351F08AE0E89FC00111240E94E9
:102BB000611A9093C9058093C805E0911603F091BE
:102BC000170390818AE0989FC0011124909310030D
:102BD00080930F0315C08FEF80930501E0911603DA
:102BE000F091170390818AE0989FC001112490937F
:102BF000120380931103892B19F081E08093200345
:102C000080EA9FE00E94611A90930C0380930B036B
:102C100045C08FEF80930501E0911603F0911703F3
:102C2000908197FD08C082E080931D0310920E03EF
:102C300010920D031AC0909580917903892B80938F
:102C4000790391818AE0989FC001112490930E032B
:102C500080930D0384E080931D0380EA9FE00E942F
:102C6000611A90930C0380930B0381E080932103FE
:102C700015C08FEF80930501E0911603F0911703C3
:102C8000808180937A0381E08093220307C081E0F2
:102C900080931F0303C081E08093230310921B03E2
:102CA000109217031092160310921503E3E0CE5F03
:102CB0000C9482A1982F8091C00085FFFCCF909347
:102CC000C60008950F931F9388E18093C1008091FF
:102CD000C00082608093C0008091C10080688093B2
:102CE000C1008091C10080648093C10000E010E0C9
:102CF0000093C5008AE290E08093C40080911103A4
:102D0000909112030E94611A9093CB058093CA059B
:102D10008CED90E00E94611A9093FA058093F9057A
:102D20001092CC058BE58093CD058BE08093D00588
:102D30008093CE051092CF051092D40580910201A8
:102D40008093D30510931703009316031092150375
:102D50001F910F910895A0E1B0E0E1EBF6E10C9432
:102D600063A180910701882309F4C5C280910B03F8
:102D700090910C030E946A1A882361F010920E034E
:102D800010920D031092120310921103109210036F
:102D900010920F0380910D0390910E03892B41F047
:102DA0008091D7069091D8060E946A1A882329F448
:102DB00080912103882309F460C080910701882352
:102DC00009F45BC080911D030BE018E08430A8F08B
:102DD0000E94632680E590E09F938F931F930F934B
:102DE00081E08F938F9388E48F930E940B112DB70E
:102DF0003EB7295F3F4F2DBF34C010927B038FE455
:102E000094E09F938F9386E596E29F938F93E09152
:102E1000B805F091B905099584E190E09F938F93EF
:102E20001F930F9381E090E09F938F938DE193E048
:102E30009F938F9382E08F9381E08F9388E48F93A9
:102E40000E940B1180911D03982F8F5F80931D03AB
:102E50002DB73EB7215F3F4F2DBF943010F0109239
:102E60001D0380910D0390910E030E94611A9093AF
:102E7000D8068093D70610922103809122038823DD
:102E800051F180910701882331F10E94632680E58A
:102E900090E09F938F938BE098E09F938F9321E036
:102EA00030E03F932F9384E291E09F938F933F9381
:102EB0002F938AE793E09F938F9383E08F9381E032
:102EC0008F938CE48F930E940B11109222038DB785
:102ED0009EB70F968DBF80911F038823D1F08091FC
:102EE00007018823B1F08AE090E09F938F938CECE8
:102EF00095E09F938F9381E08F938F9386E58F93D7
:102F00000E940B1110921F032DB73EB7295F3F4F50
:102F10002DBF809123038823D9F080910701882356
:102F2000B9F08BE090E09F938F938EEE95E09F93A6
:102F30008F9381E08F93809104018F9387E48F9327
:102F40000E940B11109223038DB79EB707968DBF79
:102F50008091110390911203892B41F08091CA0551
:102F60009091CB050E946A1A882321F48091200356
:102F7000882341F180910701882321F10E94003CC0
:102F800082E490E09F938F9385EB97E09F938F93DC
:102F900081E08F938F9384E48F930E940B111092A2
:102FA00020032DB73EB7295F3F4F2DBF80911103FE
:102FB00090911203009731F00E94611A9093CB0513
:102FC0008093CA0580910F0390911003892B09F417
:102FD000B7C08091C8059091C9050E946A1A8823DC
:102FE00009F4AEC080910701882309F4A9C080913B
:102FF00078089927880F991F880F991F7C0100274F
:10300000F7FC0095102F8091BC049091BD04A09115
:10301000BE04B091BF04BC01CD01A80197010E947C
:103020003CA13093BB052093BA058091B4049091E4
:10303000B504A091B604B091B704BC01CD01A801BC
:1030400097010E943CA13093BD052093BC052091BF
:10305000830A3091840A4091850A5091860ADA01E8
:10306000C90163E0880F991FAA1FBB1F6A95D1F79A
:10307000820F931FA41FB51F820F931FA41FB51F9C
:1030800020913E0130913F0140914001509141011A
:10309000BC01CD010E943CA13093BF052093BE0529
:1030A0008091840490918504A0918604B091870456
:1030B00059E0B595A795979587955A95D1F780933F
:1030C000C0058091800490918104A0918204B09108
:1030D000830449E0B595A795979587954A95D1F7CB
:1030E0008093C10580918C0490918D04A0918E04F1
:1030F000B0918F0439E0B595A795979587953A9546
:10310000D1F78093C2058EE090E09F938F938AEB76
:1031100095E09F938F9381E08F938F9383E48F93B8
:103120000E940B1180910F03909110030E94611A6D
:103130009093C9058093C8058DB79EB707968DBF3C
:10314000809106018F3F79F1992724E0880F991F1C
:103150002A95E1F7815B9D4F40E150E0BC01CE0133
:1031600001960E94129F80E190E09F938F93CE0181
:1031700001969F938F9381E090E09F938F9386E0D9
:1031800091E09F938F9382E08F9381E08F9381E40E
:103190008F930E940B118FEF809306012DB73EB7DE
:1031A000255F3F4F2DBF8091F7078823C9F080919D
:1031B00007018823A9F081E090E09F938F9387EF28
:1031C00097E09F938F9381E08F938F9382E48F9307
:1031D0000E940B111092F7078DB79EB707968DBF0F
:1031E00080911E038823D1F0809107018823B1F0DC
:1031F00086E490E09F938F9382E999E09F938F9369
:1032000081E08F938F9380E58F930E940B11109232
:103210001E032DB73EB7295F3F4F2DBF8091F905A3
:103220009091FA050E946A1A882309F464C080917B
:103230000701882309F45FC0809178089927880FD7
:10324000991F880F991F7C010027F7FC0095102F0C
:103250008091BC049091BD04A091BE04B091BF04C4
:10326000BC01CD01A80197010E943CA13093E70564
:103270002093E6058091B4049091B504A091B60422
:10328000B091B704BC01CD01A80197010E943CA1F7
:103290003093E9052093E8051092EA051092EB05BA
:1032A00088E090E09F938F9386EE95E09F938F93B5
:1032B00081E08F9383E08F938BE68F930E940B11B5
:1032C0008091EC052DB73EB7295F3F4F2DBF85306C
:1032D00018F086E08093EC058091C101882319F4F1
:1032E00083E690E002C087EE93E00E94611A90931B
:1032F000FA058093F905E6E0C05F0C947FA11F9268
:103300000F920FB60F9211242F933F935F936F93F9
:103310007F938F939F93AF93BF93EF93FF9380918E
:103320003603882329F08091360381508093360339
:1033300080915A05882319F0815080935A05809115
:103340003E03815080933E038F3F09F04BC089E0DC
:1033500080933E0380913C0390913D0301969093AE
:103360003D0380933C03809113018F5F81708093B4
:103370001301882319F481E080933B03349903C03F
:1033800081E0809334038091370390913803892B37
:1033900011F180913703909138030B9750F0809191
:1033A0003703909138030A9790933803809337033B
:1033B00004C0109238031092370380913703909124
:1033C000380320910A0130910B0182239323892B2A
:1033D00041F0479A07C08FEF9FEF90930B018093C6
:1033E0000A01479880913403882309F45AC0209138
:1033F000C101222309F055C08091730A83FF51C097
:1034000086B19927FC01E071F07084FF13C08091B0
:10341000390390913A03019690933A0380933903CC
:103420008091390390913A03895E9340D0F12093C3
:10343000340337C08091390390913A03892B69F1A5
:103440008091390390913A038A56914030F58091EA
:10345000390390913A0369E270E00E94F3A08091F1
:10346000390390913A03860F971F90933A03809304
:1034700039038091390390913A030B9750F0809172
:10348000390390913A030A979093AE018093AD016E
:1034900004C0F093AE01E093AD0110923A03109294
:1034A0003903FF91EF91BF91AF919F918F917F91E0
:1034B0006F915F913F912F910F900FBE0F901F90D2
:1034C000189520913C0330913D03280F391FC90105
:1034D0000196089520913C0330913D03821B930B8C
:1034E000892F99278695807490700895CF93DF93E4
:1034F0000E94611AEC01CE010E946A1A8823D9F356
:10350000DF91CF910895CF93DF930E94611AEC0170
:1035100009C080911401882329F0909314018FEC45
:1035200080937A00CE010E946A1A982F882389F32B
:10353000DF91CF9108959FB7F8945F983E9A469A8D
:103540008091B0008F708093B0008091B000836054
:103550008093B0008091B1008B738093B100809113
:10356000B1008B608093B1001092B2008FEF809316
:10357000B3008091B00080688093B00080917000AB
:103580008A7F8093700080917000826080937000C9
:103590009FBF08958AE090E00E94611A9093F90716
:1035A0008093F80782E085BD83EA84BD17BC84EB75
:1035B00088BD86E086BD80916E00816080936E003C
:1035C00008958091CB0820918A0182FF30C09091AC
:1035D0008C088CE3989FB001112490918B0880E5B2
:1035E000989FA0011124922F905897FD9D5F95956B
:1035F000959586E09802C001112420910801309130
:103600000901281B390B3093090120930801421747
:1036100053072CF050930901409308010895261791
:10362000370784F070930901609308010895822F91
:10363000992736E0880F991F3A95E1F79093090191
:10364000809308010895A0E0B0E0E9E2FBE10C946A
:103650005DA1EE24FF248701570168014091930882
:103660008090240A282D33272D573040809137042D
:1036700099278D579040289FB001299F700D389F42
:10368000700D1124CB0168EC70E00E9407A1640F5B
:10369000711D77FF0DC020E330E088279927861B36
:1036A000970BB9010E9407A1B901681B790B06C0ED
:1036B000CB0160E370E00E9407A1BC01DB01AC5BC1
:1036C000BE4FFD018485282F332727FD3095220F1B
:1036D000331F4091700A842F992787FD9095281BEE
:1036E000390B2F5F3F4F37FF02C02F5F3F4F35959C
:1036F0002795420F4093700A8C91282F332727FD7E
:103700003095220F331F6091570A862F992787FD26
:103710009095281B390B2F5F3F4F37FF02C02F5F5B
:103720003F4F35952795962E920E9092570A80918D
:10373000120190913804813009F021C1923308F0D0
:103740005BC0842F992787FD9095A92FB92F2091D1
:10375000BC043091BD044091BE045091BF04BC0133
:10376000CD010E94C8A097FF04C061507E4F8F4FCB
:103770009F4F7B018C01F9E015950795F794E7942D
:10378000FA95D1F7892D992787FD9095A92FB92F03
:103790002091B4043091B5044091B6045091B7041F
:1037A000BC01CD010E94C8A097FF04C061507E4FAC
:1037B0008F4F9F4FE9E09595879577956795EA95A7
:1037C000D1F757016801A61AB70AC80AD90A809129
:1037D0004105909142059C0153E0220F331F5A95F9
:1037E000E1F7281B390BC901AA2797FDA095BA2F2D
:1037F000A81AB90ACA0ADB0A809188019927AA2760
:10380000BB27BC01CD01A60195010E94C8A097FF6E
:1038100004C061507E4F8F4F9F4F5B016C0149E0A8
:10382000D594C794B794A7944A95D1F71091CB0833
:10383000609108017091090112FF05C07093110198
:103840006093100118C040911001509111018091B6
:103850009208282F3327CB01841B950BB9010E94B6
:1038600007A18091100190911101860F971F9093ED
:1038700011018093100110FF14C0809110019091EC
:10388000110197FD0F9634E0959587953A95E1F7EC
:10389000AA2797FDA095BA2FA80EB91ECA1EDB1E37
:1038A00015C0809110019091110197FD0F9624E0B1
:1038B000959587952A95E1F7AA2797FDA095BA2FA8
:1038C0008A199B09AC09BD095C016D012091C608EC
:1038D000222321F133278091300390913103829F7D
:1038E000A001839F500D929F500D1124CA01AA2759
:1038F00097FDA095BA2F8A0D9B1DAC1DBD1D2F5F96
:103900003F4F442737FD4095542FBC01CD010E9405
:103910003CA1309331032093300304C0B0923103B3
:10392000A092300380918B08282F3327220F331F5A
:10393000220F331F80913003909131038217930738
:103940007CF080918C08282F3327220F331F220F01
:10395000331F80913003909131032817390724F4E5
:10396000309331032093300380910201843108F4B5
:103970002EC1809112018F5F809312012AC194366B
:1039800008F046C0842F992787FD9095A92FB92F5D
:103990002091B4043091B5044091B6045091B7041D
:1039A000BC01CD010E94C8A097FF04C061507E4FAA
:1039B0008F4F9F4F5B016C0119E0D594C794B7946A
:1039C000A7941A95D1F7892D992787FD9095A92F4E
:1039D000B92F2091BC043091BD044091BE04509198
:1039E000BF04BC01CD010E94C8A097FF04C0615074
:1039F0007E4F8F4F9F4F7B018C01C9E01595079536
:103A0000F794E794CA95D1F7EA0CFB1C0C1D1D1D19
:103A1000809187019927AA27BB27BC01CD01A80166
:103A200097010E94C8A097FF04C061507E4F8F4F3E
:103A30009F4F7B018C01B9E015950795F794E794AA
:103A4000BA95D1F7809189019927A6E0880F991F2F
:103A5000AA95E1F740910E0150910F01C091920893
:103A60002C2F3327841B950BB9010E9407A180914D
:103A70000E0190910F01860F971F90930F01809375
:103A80000E018091CB0881FF14C080910E019091AE
:103A90000F0197FD0F96F4E095958795FA95E1F75C
:103AA000AA2797FDA095BA2FE80EF91E0A1F1B1F23
:103AB00015C080910E0190910F0197FD0F96E4E0E3
:103AC00095958795EA95E1F7AA2797FDA095BA2FD6
:103AD0008E199F09A00BB10B7C018D012091C708A5
:103AE000222321F1332780912E0390912F03829F6F
:103AF000B001839F700D929F700D1124CB01AA27F6
:103B000097FDA095BA2F8E0D9F1DA01FB11F2F5F8F
:103B10003F4F442737FD4095542FBC01CD010E94F3
:103B20003CA130932F0320932E0304C0F0922F0367
:103B3000E0922E0380918F08282F3327220F331F06
:103B4000220F331F80912E0390912F03821793072A
:103B50007CF080919008282F3327220F331F220FEB
:103B6000331F80912E0390912F032817390724F4D7
:103B700030932F0320932E03882D992756E0880F2A
:103B8000991F5A95E1F720910C0130910D014C2FAE
:103B90005527821B930BBA010E9407A180910C014B
:103BA00090910D01860F971F90930D0180930C014A
:103BB00080910C0190910D0197FD0F9644E0959531
:103BC00087954A95E1F790932D0380932C031092EB
:103BD0001201ECE0CDB7DEB70C9479A11F920F92E1
:103BE0000FB60F9211242F933F934F935F938F93B0
:103BF0009F93EF93FF938091020190913F03843153
:103C000008F04CC0992309F02BC18091B00086FFC9
:103C100024C08091B0008F7B8093B00080913003EE
:103C20009091310387559E4F9093330380933203D5
:103C300025E08D3D920718F08CED95E005C0875783
:103C4000914030F487E791E09093330380933203FF
:103C50008091320390913303C4C08091B00080649E
:103C60008093B00080919108282F33278DED96E046
:103C7000289FA001299F500D389F500D1124CA0183
:103C80002091400330914103821B930B90933303A7
:103C90008093320381E080931201DFC0992309F001
:103CA000DFC08091B00086FFA1C08091B0008F7B03
:103CB0008093B000E091420320919108EE23D9F463
:103CC00033278DED96E0289FA001299F500D389F46
:103CD000500D1124CA012091400330914103821BF1
:103CE000930B90933303809332031092410310920D
:103CF0004003469AB2C02E1738F48AE090E09093C1
:103D0000330380933203A9C089EA93E0909333038D
:103D1000809332038E2F992783309105D9F0843018
:103D2000910534F48130910549F0029761F022C089
:103D30008430910591F00597A9F01CC08091300363
:103D40009091310304C080912E0390912F038755E9
:103D50009E4F1FC080914C0A07C080912C03909108
:103D60002D03F5CF8091550A9927880F991F880F49
:103D7000991FEDCFFF27EE0FFF1FEE56F64F208164
:103D80003181220F331F8091320390913303820FD0
:103D9000931F909333038093320380913203909169
:103DA000330355E08D3D950718F08CED95E005C087
:103DB0008757914030F487E791E0909333038093E5
:103DC000320320913203309133032C5B3040309327
:103DD0003303209332038091400390914103820F7B
:103DE000931F909341038093400337C08091B000AC
:103DF00080648093B0008CEB90E0909333038093C9
:103E00003203809140039091410384549F4F9093DB
:103E100041038093400380913503882321F08091F2
:103E20006204882321F480913503823011F446988E
:103E300001C0469A809142038F5F80934203282FEE
:103E400033278091910899270196821793072CF4C4
:103E500081E0809312011092420381E080933F033E
:103E6000209132033091330341E02F37340730F093
:103E70008FEF8093B3002F5F30400FC02F3F31058D
:103E8000C9F0C0F0A9014F5F50404F37510550F4C1
:103E900080E88093B3002058304030933303209360
:103EA000320312C08FEF8093B300509333034093DB
:103EB00032030AC0809132038093B300109233031F
:103EC0001092320310923F03FF91EF919F918F91D7
:103ED0005F914F913F912F910F900FBE0F901F90C8
:103EE000189510927C008FEC80937A000895CF9300
:103EF000DF9310924B0386E987BD83E090E00E9438
:103F0000DD31C82F863E08F4C65FC8BD84E690E068
:103F10000E94831A80911801909119018152934057
:103F200010F0C0EF02C0C530F8F0C8BD82E390E0E9
:103F30000E94831A84E694E09F938F938AE596E12A
:103F40009F938F93E091B805F091B9050995809101
:103F50001801909119010F900F900F900F908152BE
:103F6000934010F4C550DFCF6C2F83E090E00E94A7
:103F7000E531CF3018F0CCE8D0E002C0C0E0D0E0AE
:103F8000CA3FD105F8F4C7BD82E390E00E94831ACE
:103F900086E694E09F938F938AE596E19F938F93B3
:103FA000E091B805F091B9050995809118019091BB
:103FB00019010F900F900F900F908052934010F0C6
:103FC0002196DECFC09308088091690880FF09C060
:103FD0008C2F8A508B3E28F08091D105806480938D
:103FE000D105C7BD8CE291E00E94831ADF91CF9189
:103FF0000895EF92FF921F93CF9310E080ED97E02A
:104000000E94611A7C01CCE8133019F4CB3008F01F
:10401000C9E010E080915A0390915B038C5F93405C
:1040200024F48091170181500AC080915A03909125
:104030005B038750944034F0809117018F5F809329
:10404000170101C011E080915803909159038C5FD2
:10405000934024F48091160181500AC08091580346
:10406000909159038750944034F0809116018F5FEE
:104070008093160101C01F5F8091560390915703F2
:104080008C5F934024F48091150181500AC0809187
:1040900056039091570387509440C4F080911501C6
:1040A0008F5F8093150113C088E694E09F938F93F0
:1040B0008AE596E19F938F93E091B805F091B90559
:1040C00009950F900F900F900F905FC01F5F82E1D6
:1040D00080938603809180038E7F8093800385EA9E
:1040E0008093BC00809117018A3040F48091D10503
:1040F00081608093D1058AE0809317018091170138
:10410000863F40F08091D10581608093D10585EF95
:1041100080931701809116018A3040F48091D10577
:1041200082608093D1058AE0809316018091160108
:10413000863F40F08091D10582608093D10585EF64
:1041400080931601809115018A3040F48091D10549
:1041500084608093D1058AE08093150180911501D8
:10416000863F40F08091D10584608093D10585EF32
:104170008093150180918603882339F0C7010E943E
:104180006A1A882309F090CFF5CF109214018FECB2
:1041900080937A00809114018823E1F3CA3020F4DF
:1041A0008AE090E00E94831AC15009F02DCF86E486
:1041B00090E00E94831ACF911F91FF90EF90089595
:1041C0001F920F920FB60F921124EF92FF920F934E
:1041D0001F932F933F934F935F936F937F938F938F
:1041E0009F93AF93BF93EF93FF9380916303282F27
:1041F0003327442755278F5F80936303F9012231CA
:10420000310508F025C5EA5BFF4F0C948EA1809123
:1042100078009091790046C0809178009091790063
:10422000B8C1809178009091790090936703809352
:104230006603E3C18091C6049091C7042091780081
:1042400030917900821B930B9093FB078093FA07C0
:104250008091FA079091FB0790937103809370030C
:10426000EAC180917800909179002091C804309142
:10427000C904821B930B90930708809306088091D2
:104280000608909107089093730380937203E2C429
:1042900080916A0390916B032091780030917900AE
:1042A000820F931F90936B0380936A0381E0D3C4C2
:1042B0008091680390916903209178003091790092
:1042C000820F931F909369038093680384E0C3C4B3
:1042D0008091CC0883FF1AC0809122019091230124
:1042E0009C01220F331F280F391F409178005091F5
:1042F00079008BE090E0489FB001499F700D589F76
:10430000700D1124CB016EE170E00FC0809122018D
:10431000909123019C01220F331F280F391F809198
:1043200078009091790063E070E00E94F3A0260F7E
:10433000371F36952795369527953093230120937F
:10434000220185E088C48091780090917900909353
:10435000FD078093FC078091FC079091FD07409139
:10436000C2045091C304841B950B6091C104262F95
:10437000332727FD3095821B930B90935103809335
:10438000500380911D04882309F071C0809150036F
:104390009091510302977CF172E04E3E57070CF06A
:1043A000A7C020916403309165032B5F3F4F30938A
:1043B000650320936403255030408091260490913A
:1043C0002704845F914030F4215F3F4F30936503B1
:1043D0002093640380916403909165038536910571
:1043E0000CF486C04F5F5F4F5093C3044093C204E8
:1043F0008456904037C080915003909151038F5F55
:104400009F4F0CF075C082E0473258070CF470C023
:10441000209164033091650325503040309365034B
:10442000209364032B5F3F4F8091260490912704D3
:10443000845F914030F42F503040309365032093D7
:10444000640380916403909165037FEF8C39970733
:104450000CF04EC0415050405093C3044093C204EE
:104460008C599F4F909365038093640341C0809162
:10447000410A9091420A8F5C9F41D4F18091500390
:10448000909151030297ACF0209164033091650341
:10449000C901019690936503809364038958934101
:1044A0003CF166301CF46F5F6093C10427583341C0
:1044B0001BC080915003909151038F5F9F4FC4F4B4
:1044C0002091640330916503C901019790936503BE
:1044D0008093640388579C4E5CF46B3F1CF06150E2
:1044E0006093C10429573C4E3093650320936403C5
:1044F00080915003909151039C01442737FD4095D2
:10450000542F80917C0490917D04A0917E04B09101
:104510007F04820F931FA41FB51F80937C04909388
:104520007D04A0937E04B0937F0420917C0430919D
:104530007D0440917E0450917F0457FF04C02150B8
:104540003C4F4F4F5F4F7AE05595479537952795EC
:104550007A95D1F780917C0490917D04A0917E049E
:10456000B0917F04821B930BA40BB50B80937C044A
:1045700090937D04A0937E04B0937F042EC180911C
:104580006803909169032091780030917900820F3F
:10459000931F9093690380936803109262035DC335
:1045A000809102018A3071F48091780090917900B5
:1045B0002091660330916703820F931F01969695B1
:1045C000879517C04091660350916703843158F076
:1045D0002091780030917900240F351F8FEF97E0FC
:1045E000821B930B06C08091780090917900840F14
:1045F000951F909357038093560386E02CC38091B8
:10460000C6049091C7042091780030917900821BF4
:10461000930B9093FB078093FA078091FA07909190
:10462000FB072091700330917103820F931F9093C9
:1046300055038093540387E00EC3809178009091D6
:1046400079002091C8043091C904821B930B909388
:10465000070880930608809106089091070820912A
:10466000720330917303820F931F909353038093CF
:104670005203F0C220916A0330916B03809178005D
:1046800090917900280F391F30936B0320936A03B0
:10469000809102018A3019F4220F331F04C0220FC7
:1046A000331F220F331F30936B0320936A03209133
:1046B0006A0330916B03C90137FD079643E0959576
:1046C00087954A95E1F790935B0380935A03809115
:1046D0006C0390916D03820F931F97FD0196959542
:1046E000879590936D0380936C032091D204309151
:1046F000D304821B930B909321018093200120917E
:104700006003309161038091200190912101280F75
:10471000391F37FF02C02F5F3F4F359527953093E4
:10472000610320936003C2CD209168033091690337
:104730008091780090917900280F391F3093690398
:1047400020936803809102018A3019F4220F331FED
:1047500004C0220F331F220F331F309369032093AD
:1047600068032091680330916903C90137FD0796FA
:1047700013E0959587951A95E1F7909359038093E7
:10478000580380916E0390916F03820F931F97FDE2
:1047900001969595879590936F0380936E03209172
:1047A000D0043091D104821B930B90931F0180930E
:1047B0001E0120915E0330915F0380911E01909154
:1047C0001F01280F391F37FF02C02F5F3F4F35955C
:1047D000279530935F0320935E0383E03CC2809172
:1047E0001D04882309F180E00E943B9B9B01AC01E2
:1047F00020503F4F4F4F5F4F57FF06C09B01AC010A
:1048000021503D4F4F4F5F4FF9E0559547953795F4
:104810002795FA95D1F720934303309344034093AF
:1048200045035093460310C080915C0490915D0451
:10483000A0915E04B0915F0480934303909344037E
:10484000A0934503B09346031092630381E08093E5
:104850001401809147039091480301969093480377
:104860008093470380913B04282F33278091500386
:1048700090915103289FA001299F500D389F500D02
:1048800011249A0157FF02C021503F4F832F9927CF
:1048900087FD9A952091780030917900280F391F73
:1048A000309319012093180180911D04882309F485
:1048B0007EC080911801909119017C010027112779
:1048C00080914B03992787FD9095A92FB92FBC01A3
:1048D000CD012BE032E040E050E00E94C8A0DC01B6
:1048E000CB01E81AF90A0A0B1B0BE0927403F09251
:1048F0007503009376031093770320911A0130918A
:104900001B0140911C0150911D0157FF04C0215F04
:104910003F4F4F4F5F4F74E055954795379527951B
:104920007A95D1F780911A0190911B01A0911C01F9
:10493000B0911D01821B930BA40BB50B80931A0140
:1049400090931B01A0931C01B0931D0180911A014B
:1049500090911B01A0911C01B0911D018E0D9F1D16
:10496000A01FB11F80931A0190931B01A0931C01FB
:10497000B0931D018091FE079091FF07A091000860
:10498000B091010820911A0130911B0140911C0146
:1049900050911D01821B930BA40BB50B80935C04FB
:1049A00090935D04A0935E04B0935F0453C1809123
:1049B000180190911901AA27BB2720917403309107
:1049C00075034091760350917703280F391F4A1FD2
:1049D0005B1F2093740330937503409376035093C9
:1049E0007703809178038F5F80937803803108F498
:1049F00031C180911A0190911B01A0911C01B091CD
:104A00001D017C018D0163E0EE0CFF1C001F111FD6
:104A10006A95D1F7E81AF90A0A0B1B0BE20EF31E8E
:104A2000041F151F80914B03992787FD9095A92F8F
:104A3000B92FBC01CD0120EB30E240E050E00E94F4
:104A4000C8A0DC01CB01E81AF90A0A0B1B0BD8013C
:104A5000C7010496A11DB11DB7FF05C0D801C7014C
:104A60000B96A11DB11D23E0B595A7959795879548
:104A70002A95D1F780931A0190931B01A0931C01F2
:104A8000B0931D01E090FE07F090FF070091000831
:104A90001091010880911A0190911B01A0911C01B5
:104AA000B0911D01E81AF90A0A0B1B0BE0925C0495
:104AB000F0925D0400935E0410935F0420914C0318
:104AC00030914D0340914E0350914F0357FF04C066
:104AD000215F3F4F4F4F5F4F84E055954795379586
:104AE00027958A95D1F780914C0390914D03A09121
:104AF0004E03B0914F03821B930BA40BB50B809315
:104B00004C0390934D03A0934E03B0934F038091B9
:104B10004C0390914D03A0914E03B0914F038E0D25
:104B20009F1DA01FB11F80934C0390934D03A09332
:104B30004E03B0934F0380914C0390914D03A0918D
:104B40004E03B0914F03B7FF03C00F96A11DB11DD7
:104B500014E0B595A795979587951A95D1F720916B
:104B60005C0430915D04281B390B54E0213035077B
:104B70001CF020E034E006C06CEF2030360714F45F
:104B800020E03CEF8091490390914A0380914903D2
:104B900090914A0397FF03C0909581959F4FA9017B
:104BA000F3E0440F551FFA95E1F78D5B9240C4F096
:104BB0008091490390914A039C01E4E0220F331F46
:104BC000EA95E1F7281B390B240F351F37FF02C088
:104BD000215F3F4F74E0359527957A95E1F717C02F
:104BE0008091490390914A039C0165E0220F331F95
:104BF0006A95E1F7281B390B240F351F37FF02C0D8
:104C0000215E3F4F45E0359527954A95E1F7309372
:104C10004A03209349038091740390917503A091F6
:104C20007603B0917703B7FF03C00196A11DB11DB4
:104C3000B595A79597958795809374039093750381
:104C4000A0937603B093770388E08093780302C043
:104C50001092630382E080936203809162038093E9
:104C60007C0080916303882319F08FEC80937A0095
:104C7000FF91EF91BF91AF919F918F917F916F9134
:104C80005F914F913F912F911F910F91FF90EF9066
:104C90000F900FBE0F901F90189590E2EBE0F8E098
:104CA0008FE49193815087FFFCCF089590917B030F
:104CB000903540F4E92FFF27E55FF74F80839F5F32
:104CC00090937B030895AF92BF92CF92DF92FF92B1
:104CD0000F931F93CF93DF932091790320FF0AC096
:104CE00080917A03882311F0815002C080912401C1
:104CF00080937A0321FF0CC090917A038091240164
:104D0000981719F410927A0303C09F5F90937A0367
:104D1000822F992780FF04C081FF02C010927A037E
:104D20000E944D2680917A03282F332796E5C92EBD
:104D300096E2D92EC091B805D091B9058A3098F481
:104D400081E180937B033F932F938FE994E09F93BE
:104D50008F93DF92CF92FE0109952DB73EB72A5F60
:104D60003F4F2DBF11C080E180937B033F932F9372
:104D700084EA94E09F938F93DF92CF92FE0109958E
:104D80008DB79EB706968DBF20917A03822F992703
:104D9000AA27BB27FC01419710F00C94B42FE85AC6
:104DA000FF4F06E5C02E06E2D02EC091B805D09187
:104DB000B9050C948EA110927B0389EA94E09F932D
:104DC0008F9306E516E2DF92CF92FE01099584E10A
:104DD00080937B030F900F900F900F908CE690E0E4
:104DE0009F938F938BE590E09F938F931F921F92D9
:104DF000809102016AE00E94E7A0892F99279F9382
:104E00008F93809102010E94E7A099279F938F932F
:104E100089EB94E09F938F93DF92CF92E091B80556
:104E2000F091B905099588E280937B03EDB7FEB751
:104E30003E96EDBF8CED98E09F938F93809100019B
:104E400099279F938F9381ED94E09F938F93DF92A7
:104E5000CF92E091B805F091B90509958091D205FE
:104E600099272DB73EB7285F3F4F2DBFEC01C0718A
:104E7000D07084FF06C08CE380937B038FED94E0B9
:104E8000FEC090914805992359F18CE380937B03F0
:104E9000892F99279F938F938CEE94E09F938F9304
:104EA0001F930F93E091B805F091B9050995DF9331
:104EB000CF939091480581E1989FC00111248755B7
:104EC000944F9F938F931F930F93E091B805F091A8
:104ED000B90509958DB79EB70C968DBF0C94BD2F63
:104EE0009091D105992351F08CE380937B03892F16
:104EF00099279F938F9384EF94E038C19091810319
:104F0000992371F08CE380937B03892F99279F93DA
:104F10008F938BE095E09F938F931F930F93E6C43D
:104F20008091380190913901069710F00C94BD2FB3
:104F30008CE380937B0380E295E0A8C78091730A9D
:104F400016E5C12E16E2D12EC091B805D091B90553
:104F500080FF82C010927B0380915C0490915D047D
:104F6000A0915E04B0915F04BC01CD0125E030E06A
:104F700040E050E00E943CA13F932F938DE295E0EA
:104F80009F938F93DF92CF92FE01099584E18093E6
:104F90007B038DB79EB706968DBF80915804909184
:104FA0005904A0915A04B0915B04BC01CD0125E0E5
:104FB00030E040E050E00E943CA13F932F938AE311
:104FC00095E09F938F93DF92CF92E091B805F09197
:104FD000B905099588E280937B03EDB7FEB7369655
:104FE000EDBF80911801909119019F938F9387E4F1
:104FF00095E09F938F93DF92CF92E091B805F09167
:10500000B90509958CE380937B032DB73EB72A5FE2
:105010003F4F2DBF87B599279F938F9384E595E0E8
:105020009F938F93DF92CF92E091B805F091B905ED
:1050300009958DB79EB706968DBF80911D04882374
:1050400009F49BC78DE480937B0387B599279F93D1
:105050008F9381E695E0CFC410927B0385E695E0BF
:105060009F938F93DF92CF92FE01099584E1809305
:105070007B030F900F900F900F9084E795E09F9324
:105080008F93DF92CF9206C710927B038DE795E056
:105090009F938F9306E516E2DF92CF92FE0109956A
:1050A00084E180937B030F900F900F900F9080917D
:1050B000BC049091BD04A091BE04B091BF04B7FFA1
:1050C00004C081509C4FAF4FBF4FCAE0B595A79524
:1050D00097958795CA95D1F7BF93AF939F938F9379
:1050E0008AE895E09F938F931F930F93E091B80503
:1050F000F091B905099588E280937B032DB73EB7FF
:10510000285F3F4F2DBF8091B4049091B504A091CA
:10511000B604B091B704B7FF04C081509C4FAF4FA5
:10512000BF4FFAE0B595A79597958795FA95D1F772
:10513000BF93AF939F938F9389E995E09F938F934C
:105140001F930F93E091B805F091B90509958CE391
:1051500080937B038DB79EB708968DBF80912C0AF4
:1051600090912D0A9F938F9388EA95E09F938F9358
:105170001F930F9344C4E1E0FE2EC1E0D0E004E9A8
:1051800019E09F2D969584E1989FC001112480938A
:105190007B03F801828193819F938F932196DF9304
:1051A000CF932197808191819F938F93DF93CF93AA
:1051B00087EB95E09F938F9386E596E29F938F937D
:1051C000E091B805F091B90509952DB73EB7245F78
:1051D0003F4F2DBF32E0F30E22960C5F1F4F88E049
:1051E0008F1578F6CAC610927B0380915E08E82F6F
:1051F000FF27EE0FFF1FEE56F64F808191819F93A0
:105200008F9380915D08E82FFF27EE0FFF1FEE566A
:10521000F64F808191819F938F9389EC95E09F93C6
:105220008F93DF92CF92FE01099584E180937B03F7
:10523000EDB7FEB73896EDBF80916008E82FFF27E5
:10524000EE0FFF1FEE56F64F808191819F938F9353
:1052500080915F08E82FFF27EE0FFF1FEE56F64FF5
:105260008081918181589F4F9F938F9389ED95E025
:105270009F938F93DF92CF92E091B805F091B9059B
:10528000099588E280937B032DB73EB7285F3F4F97
:105290002DBF80916208E82FFF27EE0FFF1FEE560B
:1052A000F64F8081918181589F4F9F938F9380917A
:1052B0006108E82FFF27EE0FFF1FEE56F64F8081A3
:1052C000918181589F4F9F938F9389EE95E09F9393
:1052D0008F93DF92CF92E091B805F091B9050995CF
:1052E0008CE380937B038DB79EB708968DBF80912A
:1052F0006408E82FFF27EE0FFF1FEE56F64F808160
:10530000918181589F4F9F938F9380916308E82FDD
:10531000FF27EE0FFF1FEE56F64F808191818158D7
:105320009F4F9F938F9389EF95E06BC210927B0301
:1053300089E096E09F938F9306E516E2DF92CF9285
:10534000FE010995809102010F900F900F900F9030
:105350008A3009F0A9C084E180937B038091D20454
:105360009091D3049C0197FF02C0295F3F4F287F93
:10537000821B930B9F938F938091D2049091D304BF
:1053800097FD079673E0959587957A95E1F79F933A
:105390008F932091D2043091D30437FF02C0295F4C
:1053A0003F4F63E0359527956A95E1F780915A0361
:1053B00090915B03821B930B9F938F9387E196E001
:1053C0009F938F931F930F93E091B805F091B905C8
:1053D000099588E280937B032DB73EB7265F3F4F48
:1053E0002DBF8091D0049091D1049C0197FF02C001
:1053F000295F3F4F287F821B930B9F938F93809150
:10540000D0049091D10497FD079653E09595879528
:105410005A95E1F79F938F932091D0043091D10456
:1054200037FF02C0295F3F4F43E0359527954A95E6
:10543000E1F78091580390915903821B930B9F933E
:105440008F9388E296E09F938F931F930F93E09141
:10545000B805F091B90509958CE380937B038DB76E
:105460009EB70A968DBF8091CE049091CF049F93F2
:105470008F938091CE049091CF0420915603309168
:105480005703821B930B9F938F9389E396E09F931F
:105490008F931F930F93E091B805F091B90509958B
:1054A000EDB7FEB73896B3C28B3019F0843108F4EB
:1054B000A9C084E180937B038091D2049091D304AE
:1054C0009C0197FF02C0215F3F4F207F821B930BFF
:1054D00097FD0196959587959F938F938091D20420
:1054E0009091D30497FD0F9624E0959587952A9582
:1054F000E1F79F938F932091D2043091D30437FF2B
:1055000002C0295F3F4FC3E035952795CA95E1F763
:1055100080915A0390915B03821B930B9F938F930F
:1055200087E496E09F938F931F930F93E091B805C4
:10553000F091B905099588E280937B032DB73EB7BA
:10554000265F3F4F2DBF8091D0049091D1049C01E4
:1055500097FF02C0215F3F4F207F821B930B97FD77
:105560000196959587959F938F938091D004909104
:10557000D10497FD0F96A4E095958795AA95E1F73C
:105580009F938F932091D0043091D10437FF02C0B4
:10559000295F3F4FF3E035952795FA95E1F7809124
:1055A000580390915903821B930B9F938F9389E526
:1055B00096E09F938F931F930F93E091B805F0911E
:1055C000B90509958CE380937B038DB79EB70A9646
:1055D0008DBF8091CE049091CF0497FD0196959553
:1055E00087959F938F938091CE049091CF042091C3
:1055F000560330915703821B930B9F938F938BE637
:1056000096E045CF8D3009F0B8C484E180937B03E8
:105610008091170199279F938F938091D204909145
:10562000D30497FD0F9674E0959587957A95E1F7E9
:105630009F938F932091D2043091D30437FF02C0FF
:10564000295F3F4F63E0359527956A95E1F7809193
:105650005A0390915B03821B930B9F938F938AE76E
:1056600096E09F938F931F930F93E091B805F0916D
:10567000B905099588E280937B032DB73EB7265F75
:105680003F4F2DBF8091160199279F938F93809153
:10569000D0049091D10497FD0F9654E0959587958D
:1056A0005A95E1F79F938F932091D0043091D104C4
:1056B00037FF02C0295F3F4F43E0359527954A9554
:1056C000E1F78091580390915903821B930B9F93AC
:1056D0008F938EE896E09F938F931F930F93E091A3
:1056E000B805F091B90509958CE380937B038DB7DC
:1056F0009EB70A968DBF8091150199279F938F932E
:105700008091CE049091CF0497FD01969595879551
:105710009F938F938091CE049091CF042091560354
:1057200030915703821B930B9F938F9382EA96E0ED
:105730009F938F931F930F93E091B805F091B90554
:105740000995EDB7FEB73A9662C110927B0386EBDE
:1057500096E09F938F93DF92CF92FE01099584E1AB
:1057600080937B030F900F900F900F908091C8044F
:105770009091C9049F938F9380915203909153030A
:105780009F938F9383EC96E09F938F93DF92CF92BA
:10579000E091B805F091B905099588E280937B0303
:1057A0002DB73EB7285F3F4F2DBF8091C604909123
:1057B000C7049F938F9380915403909155039F93B7
:1057C0008F9382ED96E09F938F93DF92CF92E0913B
:1057D000B805F091B90509958CE380937B038DB7EB
:1057E0009EB708968DBF8091C2049091C3049F9389
:1057F0008F9380915003909151039F938F9381EEEB
:1058000096E09F938F93DF92CF9245CE10927B03C9
:1058100080912201909123016AE070E00E9407A12B
:105820009F938F9380912201909123016AE070E011
:105830000E9407A17F936F9380EF96E09F938F93D1
:10584000DF92CF92FE01099584E180937B032DB70F
:105850003EB7285F3F4F2DBF8091080B9091090BF9
:105860006AE070E00E94F3A09F938F938091080BF1
:105870009091090B6AE070E00E94F3A07F936F9310
:1058800084E097E09F938F93DF92CF92E091B805E9
:10589000F091B905099588E280937B038DB79EB797
:1058A00008968DBF80910A0B90910B0B9F938F935D
:1058B00088E197E09F938F93DF92CF92E091B805B4
:1058C000F091B90509958CE380937B03EDB7FEB7A2
:1058D0003696EDBF80910C0B90910D0B9F938F939B
:1058E00088E297E09F938F93DF92CF92E091B80583
:1058F000F091B90509952DB73EB72A5F3F4F45C1D5
:1059000010927B038AE397E09F938F93DF92CF926D
:10591000FE01099588E280937B030F900F900F9012
:105920000F908091620499279F938F9383E497E06F
:105930009F938F93DF92CF92E091B805F091B905D4
:1059400009958CE380937B038DB79EB706968DBF38
:1059500080919109992701979F938F9383E597E011
:105960004AC010927B0383E697E09F938F93DF9268
:10597000CF92FE01099584E180937B030F900F90F5
:105980000F900F908091AD019091AE019F938F93F6
:105990008BE697E09F938F93DF92CF92E091B805CB
:1059A000F091B905099588E280937B032DB73EB746
:1059B0002A5F3F4F2DBF80912C0A90912D0A9F9313
:1059C0008F9389E797E09F938F93DF92CF92E09137
:1059D000B805F091B90509958CE380937B038DB7E9
:1059E0009EB706968DBF80917A0490917B049F9319
:1059F0008F9387E897E09F938F93DF92CF92E09108
:105A0000B805F091B9050995EDB7FEB73696EDBF2B
:105A1000B4C2C3E6CC2EC4E0DC2E20E030E0E901C5
:105A2000B3E0FB2EC0937B03F60181916F019927B0
:105A30009F938F9389010F5F1F4F1F930F9385E9EA
:105A400097E09F938F9386E596E29F938F93E091E3
:105A5000B805F091B90509952DB73EB7285F3F4FBE
:105A60002DBFFA9464969801F7FEDCCF86C2A7E6B4
:105A7000CA2EA4E0DA2EC0E0D0E08E01F3E0FF2EC3
:105A800000937B03F60181916F0199279F938F9378
:105A90002596DF93CF9382EA97E09F938F9386E5D5
:105AA00096E29F938F93E091B805F091B90509951F
:105AB0002DB73EB7285F3F4F2DBFFA940C5E1F4FA6
:105AC0002497F7FEDDCF59C210927B038FEA97E04F
:105AD0009F938F9306E516E2DF92CF92FE01099520
:105AE00084E180937B030F900F900F900F90809133
:105AF0008A0199279F938F9387EB97E09F938F93CA
:105B0000DF92CF92E091B805F091B905099588E24E
:105B100080937B038DB79EB706968DBF809130032F
:105B20009091310397FD0396959587959595879567
:105B30009F938F9385EC97E09F938F931F930F9381
:105B4000E091B805F091B90509958CE380937B034A
:105B5000EDB7FEB73696EDBF80918C0899279F93DD
:105B60008F9380918B0899279F938F9383ED97E074
:105B70009F938F931F930F93E091B805F091B90510
:105B800009952DB73EB7285F3F4F2DBFF6C1109244
:105B90007B0381EE97E09F938F9376E5A72E76E2C5
:105BA000B72EDF92CF92FE0109950F900F900F90C4
:105BB0000F90C1E3D9E000E010E062E0F62E802F04
:105BC0008C5E80937B038B8D99278F7790709F934A
:105BD0008F938B8999278F7790709F938F938B8565
:105BE00099278F7790709F938F938B8199278F77C9
:105BF00090709F938F9381EF97E09F938F93BF92C5
:105C0000AF92E091B805F091B90509958DB79EB7AF
:105C10000C968DBFFA940C5E1F4FA096F7FECFCF67
:105C2000ACC110927B0382E098E09F938F9356E57E
:105C3000A52E56E2B52EDF92CF92FE0109950F9068
:105C40000F900F900F90C1E3D9E000E010E042E028
:105C5000F42E802F8C5E80937B038F8D992787FD98
:105C600090959F938F938F89992787FD90959F9308
:105C70008F938F85992787FD90959F938F938F8121
:105C8000992787FD90959F938F9381E198E09F934B
:105C90008F93BF92AF92E091B805F091B905099545
:105CA000EDB7FEB73C96EDBFFA940C5E1F4FA09681
:105CB000F7FECFCF62C110927B0382E298E09F9300
:105CC0008F9306E516E2DF92CF92FE01099584E1FB
:105CD00080937B030F900F900F900F9080914C0951
:105CE000881F8827881F97E0899FC00111248D96FF
:105CF0009F938F9380914409881F8827881F96E07F
:105D0000899FC00111248D969F938F9380913C09A8
:105D1000881F8827881F95E0899FC00111248D96D0
:105D20009F938F9380913409881F8827881F992714
:105D3000880F991F880F991F8D969F938F9381E3EA
:105D400098E09F938F93DF92CF92E091B805F09106
:105D5000B905099588E280937B032DB73EB7245F90
:105D60003F4F2DBF80916C09881F8827881F9BE0BB
:105D7000899FC00111248D969F938F938091640910
:105D8000881F8827881F9AE0899FC00111248D965B
:105D90009F938F9380915C09881F8827881F99E0C3
:105DA000899FC00111248D969F938F9380915409F0
:105DB000881F8827881F992723E0880F991F2A9515
:105DC000E1F78D969F938F9385E498E09F938F934F
:105DD000DF92CF92E091B805F091B90509958CE377
:105DE00080937B038DB79EB70C968DBF809174090D
:105DF000881F8827881F9CE0899FC00111248D96E9
:105E00009F938F9389E598E09F938F93DF92CF9232
:105E1000E091B805F091B905099580917C09EDB73D
:105E2000FEB73696EDBF87FF12C080E480937B03F8
:105E30008AE698E09F938F93DF92CF92E091B80526
:105E4000F091B90509950F900F900F900F908091E8
:105E5000840987FF12C084E480937B038DE698E079
:105E60009F938F931F930F93E091B805F091B9051D
:105E700009950F900F900F900F9080918C0987FFDC
:105E80007CC088E480937B0380E798E09F938F93A6
:105E90001F930F93E091B805F091B90509950F9004
:105EA0000F900F900F9069C010927B0383E798E0EA
:105EB0009F938F93DF92CF92FE01099584E18093A7
:105EC0007B030F900F900F900F908091040390919F
:105ED00005039F938F9381E898E09F938F93DF92C0
:105EE000CF92E091B805F091B905099588E28093C9
:105EF0007B032DB73EB72A5F3F4F2DBF809106032E
:105F0000909107039F938F938EE898E09F938F93D0
:105F1000DF92CF92E091B805F091B905099589E437
:105F200080937B038DB79EB706968DBF8BE998E073
:105F30009F938F93DF92CF92E091B805F091B905CE
:105F40000995809179030F900F900F900F9083FF28
:105F500014C0109207031092060360E070E08EE018
:105F600090E00E94F63109C080912401281719F4AD
:105F700021502093240110927A0310927903DF912B
:105F8000CF911F910F91FF90DF90CF90BF90AF9076
:105F90000895F999FECF92BD81BDF89A80B59927F1
:105FA0000895F999FECF1FBA92BD81BD60BD0FB6AD
:105FB000F894FA9AF99A0FBE08954AEA20E030E080
:105FC0002617370740F4FC018191480F2F5F3F4FA0
:105FD00026173707C8F3842F99270895EAEA40E087
:105FE00050E04617570778F49C01F999FECF32BD6F
:105FF00021BDF89A80B5E80F4F5F5F4F2F5F3F4F8D
:106000004617570790F38E2F9927089581E08093C4
:106010005F0882E080935E0883E080935D0884E0FF
:106020008093600885E08093610886E08093620831
:1060300087E08093630888E08093640889E0809318
:1060400065088AE0809366088BE0809367088CE09F
:106050008093680808958FE580935C088CE0EEECEF
:10606000F8E011928A95E9F780910201843150F0AD
:106070008AE080937C081092A0088BE180937808D6
:106080008EE40AC083E080937C0880E28093A008BD
:106090008EE18093780885E580939D0880939E0823
:1060A00080E280939F081092CA088AE6809369086C
:1060B00082E68093CC0886E0809383081092C00823
:1060C0001092BD0848E04093760886EE80937708EA
:1060D00030E4309379082EE120936A0885E08093BC
:1060E0006C0890911D049923A9F084E180936D08B8
:1060F00088E280936B0820936F0881E0809370089A
:10610000109271088FE7809372083093CD08209326
:10611000C30812C08FE080936D0820936B089093A2
:106120006F084093700884E180937108909372081F
:106130003093CD089093C3088FE080936E0810923F
:10614000C8088CE08093C9081092850848E2409303
:10615000860887E080938708E8E0E093880810923B
:10616000A2081092A3081092A4085DE75093A50816
:1061700090E89093890832E330938A0872E0709334
:10618000CB0888E180938B0886EE80938C0884E0AE
:1061900080939108509394085093950850939608D3
:1061A00090938D0865E560938E0886E480938F0850
:1061B0008CED809390088CE3809392081092930862
:1061C0008FE58093A60883EF8093A8088AEA8093DE
:1061D000AA088093AB084093A7084093A90810929F
:1061E000AC08309397089AE59093980830939908F3
:1061F00026E02093AD0884E68093AE088093AF0834
:106200009093B00888E78093B1084093B5088BE479
:106210008093B2086093B3088093B4082093B608C3
:10622000E093B7083093B8088AE28093B90885EF05
:106230008093BA088CE88093BB087093BC081092D6
:10624000BE081092BF0881E28093800881E48093A9
:106250008108909382081092C1081092C20886E9C2
:106260008093C40850939A0884E380939B0810920B
:10627000C5081092C6081092C70808950E942B30D6
:106280008AE08093730880E18093740826E020936D
:1062900075089AE590937A0888E780937B08909335
:1062A0007D0880937E0820937F0880E28093840895
:1062B0008CE380939C088BE48093A10886E491E6AC
:1062C000A3E7B4E78093CE089093CF08A093D008BB
:1062D000B093D1086EE770E08CE598E00E94DD2F66
:1062E0008093DA080895CF93DF930E942B3088E0E3
:1062F0008093730830E13093740826E0209375088A
:1063000094E690937A0888E780937B0890937D08C1
:1063100080937E0820937F083093840886E48093DE
:106320009C088093A108AEECB8E085E0E5E2F1E0DE
:10633000ED01019009928A95E1F76EE770E0CD01D9
:10634000825790400E94DD2F8093DA08DF91CF9131
:1063500008950E942B3026E0209373088AE08093F2
:10636000740884E08093750894E690937A0888E72F
:1063700080937B0890937D0880937E0820937F080C
:1063800080E18093840886E480939C088093A10830
:1063900085E491E6A3E7B9E78093CE089093CF0810
:1063A000A093D008B093D1086EE770E08CE598E038
:1063B0000E94DD2F8093DA080895F999FECF92BDEF
:1063C00081BDF89A80B599270895F999FECF1FBA33
:1063D00092BD81BD60BD0FB6F894FA9AF99A0FBECE
:1063E000089569EC7FE20E94569F089541ED5FE2B7
:1063F0000E94909F0895EF92FF920F931F93CF9367
:10640000C82F8150853008F0C3E08FE7C89F800116
:10641000112485EEE82E8FEFF82EE00EF11E6EE7C8
:1064200070E0C7010E94EE2F682F98012D593F4F51
:106430008FB39927AC014270507081FDF9CF32BD06
:1064400021BDF89A80B5861711F0CA0123C08FB319
:1064500099279C012270307081FDF9CFF2BCE1BC1C
:10646000F89A80B58F3511F0C90114C08FE7C89F25
:10647000C00111244B9729EC3FE24FE750E0BC01EB
:106480008CE598E00E94319F0E94A9780E94D699DD
:1064900081E090E0CF911F910F91FF90EF900895D0
:1064A000282F863010F025E003C0882309F421E06E
:1064B00020930001F999FECF1FBA82E090E092BDCF
:1064C00081BD20BD0FB6F894FA9AF99A0FBE0895CF
:1064D000CF93C82F80915C088F3509F051C0C6302A
:1064E00010F0C5E003C0CC2309F44AC00E941A9EF4
:1064F0008091CD0882FF07C080918108843618F012
:1065000080E5809381086EE770E08CE598E00E945A
:10651000DD2F8093DA088FE7C89FC001112421ED99
:106520003FE24FE750E06CE578E04B970E946E9FAA
:1065300021ED3FE24CE050E06DE578E080E590E051
:106540000E946E9F6CE070E08DE598E00E94DD2F68
:10655000282FF999FECF1FBA8CE590E092BD81BD3E
:1065600020BD0FB6F894FA9AF99A0FBE8C2F0E94AC
:1065700050320E94A9780E94D69981E090E002C032
:1065800080E090E0CF9108956DE470E088EE93E0B4
:106590000E94EE2F482F8FB399279C0122703070F4
:1065A00081FDF9CF85E394E092BD81BDF89A80B575
:1065B000841779F48FB399279C012270307081FD84
:1065C000F9CF88EE93E092BD81BDF89A80B5813015
:1065D00011F0C901089529EC3FE24EE450E068EE65
:1065E00073E08BED98E00E94319F81E090E0089588
:1065F0008091DB088130A9F46DE470E08BED98E0C8
:106600000E94DD2F8093280921ED3FE24EE450E007
:106610006BED78E088EE93E00E946E9F81E090E061
:10662000089580E090E00895CF93DF9381E0809318
:10663000DB08EBEDF8E08FE0158616861786108AEA
:106640008150349687FFF8CF80E48093E8088093E8
:10665000E9081092EA088093EB088093EC0890EC2C
:106660009093ED081092EE088093EF088093F00865
:106670001092F1089093F2089093F3088093F40835
:106680001092F5088093F6089093F708ACEDB8E007
:106690008CE0EBE2F1E0ED01019009928A95E1F7DF
:1066A0006DE470E0CD0101970E94DD2F80932809F1
:1066B000DF91CF910895F999FECF82E090E092BDED
:1066C00081BDF89A80B5282F863078F023E0322FEC
:1066D000F999FECF1FBA82E090E092BD81BD30BD36
:1066E0000FB6F894FA9AF99A0FBE20930001822F00
:1066F000992708951F93CF93C82F162F863010F037
:10670000C5E003C0882309F4C1E08C2F99278230AB
:10671000910541F08330910544F4019731F40E94D2
:106720003E3105C00E94733102C00E94A93111237D
:10673000E1F06CE070E080E590E00E94EE2F282F01
:10674000F999FECF8CE590E092BD81BDF89A80B5B5
:10675000821759F429EC3FE24CE050E060E570E02C
:106760008DE598E00E94319F02C00E9406308C2F78
:106770000E946832CF911F910895DF92EF92FF92AD
:106780000F931F93CF93FF24DF2CEF2C81E190E038
:106790000E94DD3190910201981791F1963169F4D0
:1067A00081E190E00E94DD31853139F44C9905C0DA
:1067B0006F2D81E090E00E94E5316091020181E15E
:1067C00090E00E94E53188E190E028E00FB6F8946F
:1067D000A895809360000FBE2093600083EA98E044
:1067E0009F938F938AE596E19F938F93E091B805ED
:1067F000F091B90509950F900F900F900F90FFCF72
:1068000081E090E00E94DD318F3511F031E0E32E20
:106810006CE070E080E590E00E94EE2FC82FF999BF
:10682000FECF8CE590E092BD81BDF89A80B58C17C3
:1068300011F421E0D22EC1E001E010E0EE2029F4B5
:106840008C2F0E94FB318823B9F591E0F92E1F931C
:106850000F938BEC98E09F938F938AE596E19F933B
:106860008F93E091B805F091B90509952DB73EB722
:106870002A5F3F4F2DBF0130110521F00230110575
:1068800021F006C00E943E3105C00E94733102C053
:106890000E94A931DD2059F029EC3FE24CE050E0A4
:1068A00060E570E08DE598E00E94319F02C00E9493
:1068B00006308C2F0E946832CF5F0F5F1F4FC630AB
:1068C00008F4BCCFFF2019F083E00E9450320E94F0
:1068D0005B33C82F0E94FB318C2F99279F938F9396
:1068E00081EF98E09F938F930AE516E11F930F9332
:1068F000E091B805F091B905099581E090E00E941A
:10690000DD312DB73EB72A5F3F4F2DBF8F3F21F0BE
:106910000E94C432882399F48AE099E09F938F9370
:106920001F930F93E091B805F091B90509950E9466
:1069300014330E94F8320F900F900F900F90EE20BA
:1069400029F06FE581E090E00E94E53110925B084C
:1069500090E0E8EEF8E0CFE08081349618160CF471
:106960009F5FC150C7FFF8CF90935B08892F99278D
:106970009F938F938CED98E09F938F938BE299E098
:106980009F938F931F930F93E091B805F091B905F2
:1069900009950E94110A8DB79EB708968DBFCF91B9
:1069A0001F910F91FF90EF90DF900895982F2FB7D0
:1069B000F8943998389A88B1836088B98091B90081
:1069C0008C7F8093B9008AE28093B800109286038E
:1069D0001092840310928303992379F0E1E3F9E0A4
:1069E0008BE0108211821282138214821582168229
:1069F00017828150389687FFF4CF78942FBF08957F
:106A00001092860384E98093BC0080E88093BC00E8
:106A10001092BD001092BA001092BB001092B90003
:106A20001092B8001092820380E00E94D634109237
:106A3000BB0085E88093BC008091800382608093D6
:106A4000800308951F920F920FB60F9211242F9377
:106A50003F934F935F938F939F93EF93FF93809117
:106A60008603282F3327442755278F5F809386037B
:106A7000F9012731310508F0C2C2E759FF4F0C94E4
:106A80008EA181E08093820309C0809184038C30C1
:106A900090F4809184038F5F8093840380918403BA
:106AA000E82FFF27EE0FFF1FEE0FFF1FE552F74FF6
:106AB0008585181654F7809184038C3070F01092FD
:106AC0007F0310927E031092840385E080938603F7
:106AD00080918303880F8D5A04C080918403880FAE
:106AE0008E5A8093BB0085E87FC280918403E82F93
:106AF000FF2783E0EE0FFF1F8A95E1F7EF5CF64F6B
:106B000081818093BB0085E88093BC0080918403E1
:106B1000E82FFF27EE0FFF1FEE0FFF1FEE0FFF1FE7
:106B2000EF5CF64F808180FF91C080918403E82F55
:106B3000FF27EE0FFF1FEE0FFF1FEE0FFF1FEF5C93
:106B4000F64F8281882329F080915B08873008F412
:106B50006CC280917E0390917F03892B09F065C2FE
:106B600080917C0390917D03892B09F05EC26EC0F9
:106B70008091840321E030E002C0220F331F8A9508
:106B8000E2F780917C0390917D0328233923232B06
:106B900079F080918403E82FFF27EE0FFF1FEE0F9F
:106BA000FF1FEE0FFF1FEF5CF64F80E184830DC0E7
:106BB00080918403E82FFF27EE0FFF1FEE0FFF1FCA
:106BC000EE0FFF1FEF5CF64F148280918403E82FD5
:106BD000FF2753E0EE0FFF1F5A95E1F7EF5CF64FEA
:106BE0008481282F332743E0220F331F4A95E1F792
:106BF00080918403E82FFF2793E0EE0FFF1F9A9503
:106C0000E1F7EF5CF64F82818770822B8093BB00A7
:106C100085E88093BC002091840381E090E002C06D
:106C2000880F991F2A95E2F720917E0330917F0308
:106C300082239323892B51F089E299E090938A0370
:106C40008093890388E080938B03EFC184E089C13E
:106C5000E0918903F0918A0381918093BB0085E8DC
:106C60008093BC00F0938A03E093890380918B03A7
:106C7000815080938B03882309F4D7C183E071C1CD
:106C80008091B900803351F580918703882329F4DE
:106C9000809184038F5F8093870380918403E82F22
:106CA000FF2783E0EE0FFF1F8A95E1F7EF5CF64FB9
:106CB000838199278F7790708F3791057CF480912D
:106CC0008403E82FFF27EE0FFF1FEE0FFF1FEE0FCD
:106CD000FF1FEF5CF64F83818F5F838310928603E3
:106CE00084E98093BC008AE090E09093390180931E
:106CF0003801809184038F5F809384031092860310
:106D00006DC18091B9008034C9F180918303E82F6F
:106D1000FF27EE0FFF1FEE0FFF1FEE0FFF1FEF5CB1
:106D2000F64F83818F778383809183038F5F809376
:106D30008303809183038C30A0F010928303109220
:106D40007D0310927C03809188038F5F809388037A
:106D50008C3038F010928803809180038D7F80936F
:106D6000800380918003816080938003109286036A
:106D700084E98093BC001092820373C080918303E6
:106D8000E82FFF27EE0FFF1FEE0FFF1FEE0FFF1F75
:106D9000EF5CF64F83818068838380918303E82FC3
:106DA000FF27EE0FFF1FEE0FFF1FEE0FFF1FEF5C21
:106DB000F64F808180FF2FC080918303E82FFF274B
:106DC00053E0EE0FFF1F5A95E1F7EF5CF64F848119
:106DD0009927009751F04097D9F589E299E090936F
:106DE0008A038093890388E031C0809183039927C7
:106DF00043E0880F991F4A95E1F78A5C964F90937C
:106E00008A03809389039091830380918803981764
:106E1000E1F483E01BC080918303992733E0880F5E
:106E2000991F3A95E1F78A5C964F90938A03809375
:106E300089038091800381FD06C090918303809136
:106E40008803981711F482E001C081E080938B03DE
:106E500080918B03813011F485E801C085EC80932B
:106E6000BC00809187038093810310928703DDC06B
:106E7000E0918903F0918A038091BB008083809127
:106E8000890390918A03019690938A0380938903E2
:106E900080918B03815080938B03823010F085ECBE
:106EA0005DC0813011F485E859C08091800381FF75
:106EB0002DC08091250480FD1DC080918303E82FA3
:106EC000FF2723E0EE0FFF1F2A95E1F7EF5CF64F57
:106ED00086818A3F79F480918303E82FFF2793E02E
:106EE000EE0FFF1F9A95E1F7EF5CF64F808181600E
:106EF00080830CC080918303E82FFF2783E0EE0F8F
:106F0000FF1F8A95E1F7EF5CF64F108280918303B3
:106F10008F5F80938303809183038C30A0F0109265
:106F2000830310927D0310927C03809188038F5F0E
:106F3000809388038C3038F010928803809180030E
:106F40008D7F809380031092860384E98093BC0038
:106F50008091800381608093800365C08093BC0032
:106F600086E08093860361C088E9BBCD809185036C
:106F7000880F805FB6CD8091850399278130910578
:106F800061F0823091051CF4892B21F04EC00297EC
:106F900039F04BC080911701A4CD80911601A1CD8D
:106FA000809115019ECD80E89CCD1092860384E9E6
:106FB0008093BC00109282038AE090E090933901A4
:106FC0008093380180918503823088F48091850315
:106FD0008F5F8093850382E1809386038091800395
:106FE0008E7F8093800385EA8093BC001EC0109240
:106FF00085038091800381608093800316C0109286
:10700000860384E98093BC00809180038160809333
:1070100080038AE090E090933901809338011092C8
:1070200084031092830310928203FF91EF919F914A
:107030008F915F914F913F912F910F900FBE0F90C5
:107040001F9018951F93CF93DF93182F80916104A1
:10705000882321F480911303882319F081E090E0C4
:1070600097C01D3008F092C01123B1F0E12FFF2727
:1070700023E0EE0FFF1F2A95E1F7EF5CF64F3597FF
:107080008081359688230CF081C03897808180FDFF
:1070900003C083E090E07CC080912909823019F020
:1070A00084E090E075C067E070E089E299E00E94BA
:1070B000DD2F90913009891719F085E090E068C0C4
:1070C00080ED97E00E94611AEC018091800380FDC1
:1070D00005C0CE010E946A1A8823B9F3112319F45E
:1070E0008FEF90E00BC0212F33272150304081E0FB
:1070F00090E002C0880F991F2A95E2F790937F03D2
:1071000080937E03A1E0B0E0E1E3F9E040E050E0ED
:107110006BE0CD01042E02C0880F991F0A94E2F79C
:1071200020917E0330917F0382239323892B11F0DA
:107130001182128261504F5F5F4F389667FFE9CF2F
:107140001092840310928603809180038E7F809337
:10715000800385EA8093BC008091800380FD05C098
:10716000CE010E946A1A8823B9F380917E03909120
:107170007F03892B29F0CE010E946A1A882311F31C
:1071800080917E0390917F03009711F082E090E060
:10719000DF91CF911F9108950F931F93CF93DF93AA
:1071A000982F80916104882321F480911303882310
:1071B00019F081E090E092C09D30A0F4992319F479
:1071C00086E090E08BC0C92FDD27FE0133E0EE0F93
:1071D000FF1F3A95E1F7EF5CF64F359780813596C2
:1071E00087FD03C082E090E079C03897808180FD00
:1071F00003C083E090E072C080ED97E00E94611AC6
:107200008C018091800380FD05C0C8010E946A1A2C
:107210008823B9F3219721E030E0C90102C0880F2B
:10722000991FCA95E2F790937D0380937C03D9015F
:10723000E1E3F9E040E050E06BE0CD01042E02C054
:10724000880F991F0A94E2F720917C0330917D0307
:1072500082239323892B11F01182128261504F5F98
:107260005F4F389667FFE9CF109283031092290988
:107270001092300910928603809180038E7F809354
:10728000800385EA8093BC008091800380FD05C067
:10729000C8010E946A1A8823B9F380917C039091F7
:1072A0007D03892B29F0C8010E946A1A882311F3F3
:1072B00080912909823019F084E090E00FC067E0E6
:1072C00070E089E299E00E94DD2F909130098917E2
:1072D00019F085E090E002C080E090E0DF91CF916E
:1072E0001F910F910895CF93DF9390E021E83FEF36
:1072F000C8EDD9E0E2E9F9E0DF01953020F0892F0F
:107300008151883020F411961C921E9202C0318364
:1073100020831982188222969F5F129632969332AA
:1073200060F38FE790E09093D1098093D00981E8D2
:107330009FEF9093CF098093CE091092D3091092BA
:10734000D2091092CF041092CE041092D104109260
:10735000D0041092D3041092D204DF91CF910895FB
:107360001F920F920FB60F9211240F931F932F931A
:107370003F934F935F936F937F938F939F93AF93BD
:10738000BF93CF93DF93EF93FF938091CC0882FD5F
:10739000C2C0409186005091870080918D039091EA
:1073A0008E03481B590B8091860090918700909323
:1073B0008E0380938D03CA018D549440A0918F0356
:1073C000B0919003835F9A4158F480918F0380932A
:1073D0009109149714F010923C0181E090E096C05E
:1073E000A131B1050CF0F7C1CA018B5F9040845BFD
:1073F000914008F086C080913A0190913B01481B72
:10740000590BE091C508EE2351F0FF27EE0FFF1F47
:10741000EE56F64F8081918184369105ECF4FD01A2
:10742000EA0FFB1FEE56F64F80819181FA01E81BAF
:10743000F90BCF01F7FF03C0909581959F4F0697F9
:107440005CF480916204883C20F480916204865F41
:1074500001C088EC80936204FD01EA0FFB1FEE5629
:10746000F64F808191819C01220F331F280F391F15
:10747000240F351F37FF02C02D5F3F4FE901D5951F
:10748000C795D595C795CA0101968C179D0714F429
:10749000219706C041505040C417D5070CF42196DF
:1074A00080916204833CE0F08D010A0F1B1FF801FC
:1074B000EE56F64F808191819E01281B390BC90140
:1074C00063E070E00E9407A1CB01880F991F860F2F
:1074D000971F0852164FD80111969C938E9307C0A0
:1074E000AA0FBB1FA852B64F11961C921E92E09194
:1074F0008F03F0919003EE0FFF1FEE56F64FD183EE
:10750000C08380918F039091900301969093900394
:1075100080938F0360C140918600509187008091D5
:10752000910390919203481B590B80918600909192
:1075300087009093920380939103CA018D549440E5
:1075400060911B04835F9A4108F07AC060938C03BA
:1075500080918C03843008F453C0909191098091FC
:107560008C03981709F04CC050911C045B3008F450
:107570003FC010923C0110921B0440E05F31C0F00C
:10758000E42FFF27EE0FFF1F9F0129523C4FDF0121
:10759000AE56B64F8D919C91D9018D939C93DF018E
:1075A000A852B64F8D919C91E750FC4F91838083F8
:1075B000E42FFF27EE0FFF1F9F012E56364FDF01EE
:1075C000AD56BC4F8D919C91D90111969C938E9391
:1075D000DF01AB54BC4F8D919C91E852F64F9183E3
:1075E0008083842F8F5F482F813140F280931B046A
:1075F00080911C048F3FB9F08F5F80931C0413C0EF
:1076000080911C04853620F08AE080931C0402C01F
:1076100010921C04809102018A3011F0843110F024
:10762000289A01C0289881E080931B04809161040E
:10763000882309F0D0C080918C0380939109CBC03E
:10764000613108F0A0C0CA018B5F9040845B91401B
:1076500008F090C080913A0190913B01481B590B72
:10766000E62FFF27EE0FFF1FED56FC4F8081918123
:10767000FA01E81BF90BCF0105960B9720F5E09175
:10768000C508EE2351F0FF27EE0FFF1FEE56F64F11
:107690008081918184369105B4F480911C048A31F3
:1076A00020F080916204865F05C08B3028F08091C5
:1076B00062048E5F8093620480916204893C18F0BA
:1076C00088EC80936204E62FFF27EE0FFF1FED5634
:1076D000FC4F808191819C01220F331F280F391F9D
:1076E000240F351F37FF02C02D5F3F4FE901D595AD
:1076F000C795D595C795CA0101968C179D0714F4B7
:10770000219706C041505040C417D5070CF421966C
:10771000809162048E3BD8F0E62FFF27EE0FFF1F0B
:10772000DF01AD56BC4F8D919C919E01281B390BFA
:10773000C90163E070E00E9407A1CB01880F991F87
:10774000860F971FEB54FC4F9183808308C0E62F70
:10775000FF27EE0FFF1FEB54FC4F11821082809128
:107760001B04E82FFF27EE0FFF1FED56FC4FD183C0
:10777000C08309C0809102018A3011F0843110F079
:10778000289A01C0289880911B04843120F48F5FCF
:1077900080931B0420C08431F1F4809102018A306F
:1077A00011F0843110F0289A01C028988EE180935E
:1077B0001B0420E1C8EDD9E0A7EDB3E0E2E9F9E070
:1077C0008D919D91918380833296198218822296A1
:1077D000215027FFF5CFFF91EF91DF91CF91BF911E
:1077E000AF919F918F917F916F915F914F913F9159
:1077F0002F911F910F910F900FBE0F901F90189512
:10780000EF92FF920F931F93809178089927880F2A
:10781000991F880F991F7C010027F7FC0095102FF6
:107820008091BC049091BD04A091BE04B091BF04AE
:10783000BC01CD01A80197010E943CA13093B8077B
:107840002093B7078091B4049091B504A091B60439
:10785000B091B704BC01CD01A80197010E943CA1E1
:107860003093BA072093B9078091770A9091780AEC
:1078700097FD039695958795959587959093BC0769
:107880008093BB078091870A9091880A97FD0396A1
:1078900095958795959587959093BE078093BD079D
:1078A0008091CE049091CF042091560330915703DC
:1078B000821B930B9093C0078093BF0780915C0459
:1078C00090915D04A0915E04B0915F04BC01CD0174
:1078D0002AE030E040E050E00E943CA13093C20733
:1078E0002093C1078091FC079091FD079093C407F6
:1078F0008093C3078091AD019091AE019093C8072A
:107900008093C70780912201909123019093CA0729
:107910008093C9078091620499279093CC07809344
:10792000CB0780912C0A90912D0A9093CE078093DB
:10793000CD078091320999279093D0078093CF0784
:1079400080913A0999279093D2078093D10780912B
:10795000420999279093D4078093D30780914A09CD
:1079600099279093D6078093D5078091700A99271D
:1079700087FD90959093D8078093D7078091570AF9
:10798000992787FD90959093DA078093D907809186
:107990002C0390912D039093DC078093DB0780915B
:1079A0002E0390912F039093DE078093DD07809143
:1079B0003003909131039093E0078093DF0780912B
:1079C0004604909147049093E2078093E1078091E9
:1079D000080B9091090B9093E4078093E307809143
:1079E0000C0B90910D0B9093E6078093E507809127
:1079F000580490915904A0915A04B0915B04BC01C1
:107A0000CD012AE030E040E050E00E943CA13093FC
:107A1000E8072093E70780917A0490917B04909384
:107A2000EE078093ED0780910E0B99279093F20754
:107A30008093F1078091390590913A059093F4076E
:107A40008093F30780913705909138059093F6075E
:107A50008093F5078091D105882321F48091D20588
:107A6000882321F08091B607816003C08091B6071A
:107A70008E7F8093B6071F910F91FF90EF9008952E
:107A8000EF92FF921F93CF93DF93182F7B0180918A
:107A90006104882391F5809102018C3010F08731C8
:107AA00011F4299801C0299A11501F3FE9F0F09272
:107AB0003803E0923703E701809137039091380350
:107AC000892B11F4209781F380913B038823A1F344
:107AD00010923B038091370390913803892B09F46E
:107AE00021970E94309EE8CF809102018C3010F0E7
:107AF000873111F4299A01C02998DF91CF911F9104
:107B0000FF90EF900895CF93DF93809102018D3025
:107B100011F40E94F91F10927A0080915A039091FB
:107B20005B039093380A8093370A809158039091B1
:107B300059039093280A8093270A809156039091C5
:107B4000570390937D0A80937C0A209152033091D1
:107B50005303C901880F991F880F991F820F931F24
:107B6000820F931F9093780A8093770A2091540391
:107B700030915503C901880F991F880F991F820FF3
:107B8000931F820F931F9093880A8093870A8FEC2C
:107B900080937A00A3E6B4E0C1E6D8E097E089914B
:107BA000E82FFF27EE0FFF1FEE56F64F0190F081F2
:107BB000E02DE158FF4F1E161F061CF0E0E0F0E03C
:107BC00005C0EF3FF10514F0EFEFF0E08C91282FA6
:107BD0003327E217F30714F4815004C02E173F0730
:107BE00014F48F5F8C939150119697FFD8CF8091AA
:107BF0009D089927AA27BB27BC01CD0124EC39E0B9
:107C000040E050E00E94C8A0DC01CB018093A501B8
:107C10009093A601A093A701B093A80180919E081C
:107C20009927AA27BB27BC01CD010E94C8A0DC016F
:107C3000CB018093A1019093A201A093A301B093E3
:107C4000A401DF91CF910895A0E0B0E0EAE2FEE365
:107C50000C945BA1682EE1E07E2E00E010E068014C
:107C60005801E8011092D1051093C9040093C8048B
:107C70001093C7040093C6041093C3040093C20476
:107C80001092C1041093D3040093D2041093D10432
:107C90000093D0041093CF040093CE04109285017A
:107CA0001092840110924B030E94833D84E690E081
:107CB0000E94831A0E94833D8091690880FF10C052
:107CC0008091180190911901875B934038F480915D
:107CD0001801909119018E5E924010F40E94771F56
:107CE0007FE1E72E8AE090E00E94831A809156039C
:107CF00090915703080F191F80915A0390915B03CD
:107D0000C80ED91E8091580390915903A80EB91E30
:107D10008091FC079091FD07C80FD91FEA94E7FEF8
:107D2000E1CF9601205F3F4F3695279536952795F1
:107D30003093D3042093D204C5014096969587953D
:107D4000969587959093D1048093D004005F1F4F40
:107D500045E0169507954A95E1F71093CF040093F7
:107D6000CE046096B5E0D695C795BA95E1F7D09365
:107D7000C304C093C2049093CD048093CC04309389
:107D8000CB042093CA0482E06816C9F58091770A73
:107D90009091780A97FF03C0909581959F4F6CE072
:107DA00070E00E9407A19B017093C9046093C8040E
:107DB0008091870A9091880A97FF03C090958195DA
:107DC0009F4F6CE070E00E9407A17093C70460931E
:107DD000C604B90184E090E00E94F6316091C604C7
:107DE0007091C70486E090E00E94F6316091C20471
:107DF0007091C30488E090E00E94F6314FC084E0A7
:107E000090E00E94F1319093C9048093C80486E009
:107E100090E00E94F1319C019093C7048093C604C6
:107E20008091C8049091C9048150984018F4215061
:107E30003840A0F18CE499E09F938F938AE596E116
:107E40009F938F93E091B805F091B90509958091C2
:107E5000770A9091780A97FF03C0909581959F4F7C
:107E60006CE070E00E9407A17093C9046093C8049D
:107E70008091870A9091880A97FF03C09095819519
:107E80009F4F6CE070E00E9407A17093C70460935D
:107E9000C60477240F900F900F900F9012BC11BC66
:107EA0001092380A1092370A1092280A1092270A64
:107EB00010927D0A10927C0A84E690E00E94831A58
:107EC00080915203909153039C01220F331F220F84
:107ED000331F280F391F280F391F3093780A20933A
:107EE000770A80915403909155038C01000F111F64
:107EF000000F111F080F191F080F191F1093880A70
:107F00000093870A80917808C82EDD24EE24FF2490
:107F1000442737FD4095542FC701B6010E94C8A0E1
:107F20004B015C016093BC047093BD048093BE045C
:107F30009093BF049801442737FD4095542FC70103
:107F4000B6010E94C8A0DC01CB018093B4049093D9
:107F5000B504A093B604B093B70480929C049092A9
:107F60009D04A0929E04B0929F04809394049093E9
:107F70009504A0939604B093970410928C041092E9
:107F80008D0410928E0410928F0480911A019091AA
:107F90001B01A0911C01B0911D018093FE079093DD
:107FA000FF07A0930008B093010810924A031092B3
:107FB000490310924C0310924D0310924E031092FD
:107FC0004F0310927C0410927D0410927E04109254
:107FD0007F040091AD011091AE0110937B040093DA
:107FE0007A0484E690E09093AA018093A90182E349
:107FF00090E0909338038093370380919D089927F0
:10800000AA27BB27BC01CD0124EC39E040E050E0B9
:108010000E94C8A0DC01CB018856954CAF4FBF4FE2
:108020008093A5019093A601A093A701B093A80106
:1080300080919E089927AA27BB27BC01CD010E94E9
:10804000C8A0DC01CB018856954CAF4FBF4F809341
:10805000A1019093A201A093A301B093A401109257
:10806000430110924201C801AA2797FDA095BA2F9B
:1080700020913E0130913F014091400150914101DA
:10808000BC01CD010E94C8A0DC01CB018093830A12
:108090009093840AA093850AB093860A109277047D
:1080A000109276040E94A9788091250484608093C0
:1080B00025048FEF8093030B1092040B80E28093D2
:1080C000050BC3E6D4E0A1E6B8E0E7E0EE2E8D9123
:1080D000E82FFF27EE0FFF1FEE56F64F80819181AC
:1080E00081588993EA94E7FEF2CF84E68093620494
:1080F00080913503882311F0579A0DC080E091E1FB
:10810000909309018093080181E0809312010E94FD
:10811000231B0E94231B8091BC049091BD04A0915D
:10812000BE04B091BF04E0903E01F0903F01009189
:10813000400110914101BC01CD01A80197010E94AD
:108140003CA159016A018091B4049091B504A091B9
:10815000B604B091B704BC01CD01A80197010E94FB
:108160003CA1B901C5010E944C928C010E940C7C7B
:108170009C019093420A8093410A8091C20490919D
:10818000C304AA2797FDA095BA2F7DE0880F991FF9
:10819000AA1FBB1F7A95D1F78050904FAF43B040D4
:1081A000442737FD4095542FBC01CD010E943CA1CE
:1081B000C90180509E4F9093C3048093C20405313F
:1081C00011050CF07724662079F080911D04882336
:1081D00059F0C90181599040C39730F08091D10581
:1081E00080628093D10577248091D2049091D3044A
:1081F00080569940815C9B4228F08091D105816036
:108200008093D1058091D0049091D10480569940FB
:10821000815C9B4228F08091D10582608093D105DA
:108220008091CE049091CF048C5291408957954013
:1082300028F08091D10584608093D1058091C80495
:108240009091C9048C529140835C914028F08091B8
:10825000D10588608093D1058091C6049091C704B0
:108260008C529140835C914028F08091D1058061CF
:108270008093D1058091C2049091C30480509240B4
:108280008355914028F08091D10580628093D1057B
:108290008091D1058111772486E480939C010E940E
:1082A000D69982E00E943B9B872D9927EEE0CDB7BF
:1082B000DEB70C9477A1A3E1B0E0E1E6F1E40C9421
:1082C00057A18091CE049091CF0420915603309114
:1082D0005703821B930B90937D0A80937C0A8091B5
:1082E00060039091610397FD07969C0113E035951B
:1082F00027951A95E1F73093380A2093370A809131
:108300005E0390915F0397FD0796B3E0959587957F
:10831000BA95E1F79093280A8093270A3093440A8C
:108320002093430A90933B0A80933A0A8091770AFC
:108330009091780AAC01440F551F480F591F2091A6
:10834000520330915303C901880F991F880F991F59
:10835000820F931F820F931F480F591F57FF02C0B0
:108360004D5F5F4F55954795559547955093780AC2
:108370004093770A8091870A9091880AAC01440F54
:10838000551F480F591F2091540330915503C901BF
:10839000880F991F880F991F820F931F820F931FB9
:1083A000480F591F57FF02C04D5F5F4F55954795C6
:1083B000559547955093880A4093870A2091520318
:1083C00030915303C901880F991F880F991F820F9D
:1083D000931F820F931F9C01442737FD4095542F14
:1083E0008091AC049091AD04A091AE04B091AF0423
:1083F000820F931FA41FB51F8093AC049093AD040C
:10840000A093AE04B093AF04209154033091550370
:10841000C901880F991F880F991F820F931F820F20
:10842000931F9C01442737FD4095542F8091A80449
:108430009091A904A091AA04B091AB04820F931F5C
:10844000A41FB51F8093A8049093A904A093AA0425
:10845000B093AB0480914D0A90914E0A2091520343
:1084600030915303820F931F90934E0A80934D0ACD
:1084700080917F0A9091800A209154033091550396
:10848000820F931F9093800A80937F0A8091C40487
:108490009091C50401969093C5048093C404809183
:1084A000FC079091FD072091C2043091C304821B08
:1084B000930B9C01442737FD4095542F8091A404D1
:1084C0009091A504A091A604B091A704820F931FD8
:1084D000A41FB51F8093A4049093A504A093A604A1
:1084E000B093A7048FEC80937A001092140120912E
:1084F00094043091950440919604509197042987F3
:108500003A874B875C8729543B46414050402CF0CA
:1085100028E43BE641E050E00DC089859A85AB85B3
:10852000BC85885B9449AE4FBF4F4CF428EB34E9CF
:108530004EEF5FEF2D833E834F83588708C08985B8
:108540009A85AB85BC858D839E83AF83B887209148
:108550009C0430919D0440919E0450919F042D876E
:108560003E874F87588B29543B46414050402CF062
:1085700028E43BE641E050E00DC08D859E85AF8547
:10858000B889885B9449AE4FBF4F4CF428EB34E96F
:108590004EEF5FEF29833A834B835C8308C08D8560
:1085A0009E85AF85B88989839A83AB83BC83A0916C
:1085B0007C0AB0917D0ABB8BAA8BFD01CF01AA2753
:1085C00097FDA095BA2FA0908C04B0908D04C09018
:1085D0008E04D0908F04A80EB91ECA1EDB1EA09276
:1085E0008C04B0928D04C0928E04D0928F04E090DF
:1085F000830AF090840A0091850A1091860AE80E99
:10860000F91E0A1F1B1FE092830AF092840A00934E
:10861000850A1093860AF0914504F98BFF2309F02F
:108620009CC180914404882309F097C18091730A0A
:1086300086FF93C18091270A9091280AAA2797FD67
:10864000A095BA2FBC01CD0129813A814B815C8173
:108650000E94C8A09B01AC0197FF04C02150384F75
:108660004F4F5F4FBBE05595479537952795BA9586
:10867000D1F780918401682E772488249924CA0137
:10868000B901A40193010E94C8A0DC01CB01809331
:10869000DE049093DF04A093E004B093E104B7FFFD
:1086A00004C08150904FAF4FBF4F1C012D01ACE073
:1086B0005594479437942794AA95D1F72092DE04D5
:1086C0003092DF044092E0045092E1048091370A36
:1086D0009091380AAA2797FDA095BA2FBC01CD0129
:1086E0002D813E814F8158850E94C8A097FF04C00C
:1086F0006150784F8F4F9F4FFBE095958795779509
:108700006795FA95D1F7A40193010E94C8A0DC01F6
:10871000CB018093E2049093E304A093E404B0932C
:10872000E504B7FF04C08150904FAF4FBF4F9C018D
:10873000AD01ECE05595479537952795EA95D1F72A
:108740002093E2043093E3044093E4045093E5045F
:108750008091DE049091DF0490931F0A80931E0A9B
:108760008091E2049091E3049093230A8093220A7B
:1087700022193309440955092093E2043093E30494
:108780004093E4045093E5048091560A882331F124
:10879000E20EF31E041F151FE092830AF092840A72
:1087A0000093850A1093860A809183018823B1F48F
:1087B00057FF04C02F5F3F4F4F4F5F4F5595479571
:1087C00037952795A21AB30AC40AD50AA0928C0439
:1087D000B0928D04C0928E04D0928F042A893B8976
:1087E00079010027F7FC0095102F8091E204909109
:1087F000E304A091E404B091E504E80EF91E0A1F19
:108800001B1FC801B70129813A814B815C810E94FD
:10881000C8A09B01AC0197FF04C02150384F4F4FB7
:108820005F4F6BE055954795379527956A95D1F73A
:1088300080918501A82EBB24CC24DD24CA01B90176
:10884000A60195010E94C8A0DC01CB018093D6044B
:108850009093D704A093D804B093D904B7FF04C071
:108860008150904FAF4FBF4F3C014D013CE095947C
:108870008794779467943A95D1F76092D604709272
:10888000D7048092D8049092D904C801B7012D81F1
:108890003E814F8158850E94C8A097FF04C0615057
:1088A000784F8F4F9F4F2BE09595879577956795DC
:1088B0002A95D1F7A60195010E94C8A0DC01CB0141
:1088C0008093DA049093DB04A093DC04B093DD047E
:1088D000B7FF04C08150904FAF4FBF4FAC01BD01F7
:1088E0000CE075956795579547950A95D1F7409394
:1088F000DA045093DB046093DC047093DD042A896E
:108900003B8937FF03C0309521953F4F2134310516
:10891000E4F1D401C30197FE07C0B095A0959095EE
:1089200081959F4FAF4FBF4F81389105A105B1058C
:1089300084F4DB01CA0177FF07C0B095A09590953C
:1089400081959F4FAF4FBF4F81389105A105B1056C
:10895000E4F081E08093780418C01092230A10920A
:10896000220A10921F0A10921E0A1092DA04109224
:10897000DB041092DC041092DD041092D6041092F5
:10898000D7041092D8041092D9048091DA049091FF
:10899000DB04A091DC04B091DD04BC01CD0124E630
:1089A00030E040E050E00E943CA1E090D604F0901E
:1089B000D704E21AF30AF092360AE092350A80915F
:1089C000D6049091D704A091D804B091D904BC01E9
:1089D000CD0124E630E040E050E00E943CA1DA0105
:1089E000C9012091DA043091DB048C01021B130BC6
:1089F00010932A0A0093290A80913E0190913F0129
:108A0000A0914001B0914101BC01CD0128E631E0C7
:108A100040E050E00E94C8A02091830A3091840A6F
:108A20004091850A5091860A26173707480759074B
:108A300064F0261B370B480B590B2093830A3093A5
:108A4000840A4093850A5093860A2091830A3091C4
:108A5000840A4091850A5091860A57FF0CC0260F60
:108A6000371F481F591F2093830A3093840A40936D
:108A7000850A5093860A6091270A7091280A6E0D24
:108A80007F1D9B01442737FD4095542F8091900412
:108A900090919104A0919204B0919304820F931F3E
:108AA000A41FB51F8093900490939104A093920407
:108AB000B093930480914A0490914B04681B790B06
:108AC000CB01AA2797FDA095BA2F29853A854B851A
:108AD0005C85820F931FA41FB51F8093940490930D
:108AE0009504A0939604B0939704C090A101D090F0
:108AF000A201E090A301F090A401C816D906EA06ED
:108B0000FB06C4F488EA91E6A0E0B0E08C199D0968
:108B1000AE09BF098093940490939504A0939604A2
:108B2000B09397048093900490939104A09392043F
:108B3000B093930422273327A9012C193D094E092C
:108B40005F098091940490919504A0919604B0914E
:108B5000970482179307A407B507B4F4D701C60199
:108B6000885A9146A040B040809394049093950415
:108B7000A0939604B09397048093900490939104EB
:108B8000A0939204B09393046091370A7091380ACD
:108B9000600F711F9B01442737FD4095542F809132
:108BA000980490919904A0919A04B0919B04820F2B
:108BB000931FA41FB51F8093980490939904A093CA
:108BC0009A04B0939B048091480490914904681BD7
:108BD000790BCB01AA2797FDA095BA2F2D853E854D
:108BE0004F855889820F931FA41FB51F80939C0443
:108BF00090939D04A0939E04B0939F04E090A501E0
:108C0000F090A6010091A7011091A801E816F906BD
:108C10000A071B07C4F488EA91E6A0E0B0E08E19C9
:108C20009F09A00BB10B80939C0490939D04A0938B
:108C30009E04B0939F048093980490939904A0930A
:108C40009A04B0939B0422273327A9012E193F09C8
:108C5000400B510B80919C0490919D04A0919E0427
:108C6000B0919F0482179307A407B507B4F4D80105
:108C7000C701885A9146A040B04080939C049093CD
:108C80009D04A0939E04B0939F04809398049093B6
:108C90009904A0939A04B0939B0480918C049091C2
:108CA0008D04A0918E04B0918F048093A0049093C2
:108CB000A104A093A204B093A30480919C0490917A
:108CC0009D04A0919E04B0919F048093BC04909356
:108CD000BD04A093BE04B093BF048091940490910E
:108CE0009504A0919604B09197048093B404909356
:108CF000B504A093B604B093B70480919804909102
:108D00009904A0919A04B0919B048093B804909325
:108D1000B904A093BA04B093BB04809190049091DD
:108D20009104A0919204B09193048093B004909325
:108D3000B104A093B204B093B30480912001909148
:108D4000210197FD079613E0959587951A95E1F710
:108D50009093380A8093370A80911E0190911F01E9
:108D600097FD0796B3E095958795BA95E1F79093AF
:108D7000280A8093270A809102018A3009F062C094
:108D800080915A0390915B03835F934034F088E5B0
:108D900092E09093380A8093370A80915A03909119
:108DA0005B038A5F934034F080E293E09093380A4B
:108DB0008093370A80915A0390915B030F9734F4A4
:108DC00088EA9DEF9093380A8093370A80915A037E
:108DD00090915B03079734F480EE9CEF9093380AF0
:108DE0008093370A8091580390915903835F934091
:108DF00034F088E592E09093280A8093270A8091C6
:108E00005803909159038A5F934034F080E293E0D5
:108E10009093280A8093270A8091580390915903D0
:108E20000F9734F488EA9DEF9093280A8093270ADD
:108E3000809158039091590307970CF067C080EE1A
:108E40009CEF60C080915A0390915B03815D9740D5
:108E500034F080EB94E09093380A8093370A809145
:108E60005A0390915B03805E974034F080E496E073
:108E70009093380A8093370A80915A0390915B034C
:108E80000F9734F480E59BEF9093380A8093370A6C
:108E900080915A0390915B03079734F480EC99EF2B
:108EA0009093380A8093370A809158039091590320
:108EB000815D974034F080EB94E09093280A809392
:108EC000270A8091580390915903805E974034F0AF
:108ED00080E496E09093280A8093270A80915803B3
:108EE000909159030F9734F480E59BEF9093280AF3
:108EF0008093270A8091580390915903079734F47F
:108F000080EC99EF9093280A8093270A6091920150
:108F1000662309F4AFC04091200150912101809156
:108F2000E6049091E704481B590B5093ED044093DD
:108F3000EC042091200130912101280F391F37FFC7
:108F400002C02F5F3F4F359527953093E70420935C
:108F5000E604413851051CF080E890E005C0405817
:108F60005F4F34F480E89FEF9093ED048093EC041E
:108F700040911E0150911F018091E8049091E904F5
:108F8000481B590B5093EB044093EA0420911E01B7
:108F900030911F01280F391F37FF02C02F5F3F4F4D
:108FA000359527953093E9042093E804413851051D
:108FB0001CF080E890E005C040585F4F34F480E832
:108FC0009FEF9093EB048093EA04462F55278091FE
:108FD000EC049091ED04849FB001859F700D949FE7
:108FE000700D11249B0177FF02C0215F3F4FE4E029
:108FF00035952795EA95E1F78091370A9091380ADF
:10900000820F931F9093380A8093370A8091EA0465
:109010009091EB04849FD001859FB00D949FB00D7B
:109020001124AD019D01B7FF02C0215F3F4F94E0C5
:10903000359527959A95E1F78091270A9091280A0E
:10904000820F931F9093280A8093270A8091200112
:1090500090912101860F971F909321018093200109
:1090600080911E0190911F01840F951F90931F0105
:1090700080931E0100913A0A10913B0A80911E0ACA
:1090800090911F0A101611065CF59C0197FF04C011
:1090900022273327281B390BC901AA2797FDA09542
:1090A000BA2F20918301332744275527BC01CD01D6
:1090B0000E94C8A09B01AC0197FF04C0215C3F4FF8
:1090C0004F4F5F4F86E055954795379527958A9581
:1090D000D1F78091350A9091360A820F931F27C0ED
:1090E00097FF03C0909581959F4FAA2797FDA09564
:1090F000BA2F20918301332744275527BC01CD0186
:109100000E94C8A09B01AC0197FF04C0215C3F4FA7
:109110004F4F5F4FB6E05595479537952795BA95D0
:10912000D1F78091350A9091360A821B930B909368
:10913000360A8093350AE090430AF090440A809101
:10914000220A9091230A1E141F045CF59C0197FFCC
:1091500004C022273327281B390BC901AA2797FDF2
:10916000A095BA2F20918301332744275527BC01AE
:10917000CD010E94C8A09B01AC0197FF04C0215CF7
:109180003F4F4F4F5F4FA6E0559547953795279531
:10919000AA95D1F78091290A90912A0A820F931FEC
:1091A00027C097FF03C0909581959F4FAA2797FDF1
:1091B000A095BA2F20918301332744275527BC015E
:1091C000CD010E94C8A09B01AC0197FF04C0215CA7
:1091D0003F4F4F4F5F4FF6E0559547953795279591
:1091E000FA95D1F78091290A90912A0A821B930B54
:1091F00090932A0A8093290A8091730A87FF44C0BA
:10920000B989BB2309F040C0809144048823E1F56B
:10921000E1E0EE16E1E0FE064CF08091370A909115
:10922000380A8E0D9F1D805091400DC0F0E0EF1662
:10923000FFEFFF0664F48091370A9091380A8E0D93
:109240009F1D80509F4F9093380A8093370A21E0EA
:10925000013012074CF08091270A9091280A800F64
:10926000911F805091400CC03FEF0030130764F411
:109270008091270A9091280A800F911F80509F4F5C
:109280009093280A8093270AE2E1CD5E0C9473A1A3
:1092900080916104882329F5809125048C7F809337
:1092A0002504809124048F7D80932404A6EDB5E0ED
:1092B000E1E3F9E09BE080911303882309F48C93A8
:1092C0008D91818312829150389697FFF4CF8091CF
:1092D0001303882359F08091130381508093130363
:1092E00005C08091250481608093250480918203CC
:1092F000882319F010928203089580938403809349
:109300008603809180038E7F8093800385EA80931B
:10931000BC000895882319F480E090E00895E82FB8
:10932000FF27EE0FFF1FEE56F64F80819181815887
:109330009F4F8F3F910521F01CF08FEF90E004C00C
:1093400097FF02C080E090E099270895CF93DF93C4
:10935000A3E6B4E0C1E6D8E057E08991E82FFF2703
:10936000EE0FFF1FEE56F64F0190F081E02DE15811
:10937000FF4FEF3FF10521F01CF0EFEFF0E004C0EC
:10938000F7FF02C0E0E0F0E0893111F4EC931BC07C
:109390004C91242F3327E217F307A9F0CF01821B4A
:1093A000930B97FD03969595879595958795242F13
:1093B000280F2C93822F9927E817F90714F42150CE
:1093C00001C02F5F2C935150119657FFC6CF80914B
:1093D0006B08883F38F0EFEFF0E0E81BF109ED593A
:1093E000FB4F80818093970180919701882329F01A
:1093F000843618F084E68093970180916D08883F49
:1094000038F0EFEFF0E0E81BF109ED59FB4F8081F8
:109410008093960180919601882329F0843618F074
:1094200084E68093960180917A08883F38F0EFEFC8
:10943000F0E0E81BF109ED59FB4F80818093910129
:10944000809191018B3010F48AE002C08F3F11F4BB
:10945000809391018091A708883F38F0EFEFF0E00A
:10946000E81BF109ED59FB4F808180934F0A8091F1
:109470004F0A863010F485E002C08F3F11F48093CC
:109480004F0A8091A908883F38F0EFEFF0E0E81B21
:10949000F109ED59FB4F808180937A0A80917A0A15
:1094A000863010F485E002C08F3F11F480937A0A71
:1094B00080919408873F19F4429905C006C0863F01
:1094C00031F4439B02C08CE815C086E413C0883F8A
:1094D00038F0EFEFF0E0E81BF109ED59FB4F808128
:1094E00080934C0A80914C0A893110F488E102C0C3
:1094F0008F3F11F480934C0A80919508873F19F4AF
:10950000429905C006C0863F31F4439B02C08CE8F7
:1095100015C086E413C0883F38F0EFEFF0E0E81B99
:10952000F109ED59FB4F80818093240A8091240A30
:10953000893110F488E102C08F3F11F48093240A2E
:1095400080919608883F38F0EFEFF0E0E81BF109D2
:10955000ED59FB4F80818093550A8091550A8931DE
:1095600010F488E102C08F3F11F48093550A809176
:109570006C080E948A4980933F0480916F08883F5D
:1095800038F0EFEFF0E0E81BF109ED59FB4F808177
:109590008093950180917108883F38F0EFEFF0E0FB
:1095A000E81BF109ED59FB4F808180939301809175
:1095B0007908883F38F0EFEFF0E0E81BF109ED594A
:1095C000FB4F80818093940180917B08883F38F025
:1095D000EFEFF0E0E81BF109ED59FB4F808180933C
:1095E000900180917C08883F38F0EFEFF0E0E81BB5
:1095F000F109ED59FB4F80818093920180917D08A4
:10960000883F38F0EFEFF0E0E81BF109ED59FB4F30
:10961000808180938F0180917E08883F38F0EFEF42
:10962000F0E0E81BF109ED59FB4F808180938E013A
:1096300080918408883F38F0EFEFF0E0E81BF109F3
:10964000ED59FB4F808180938C0180918508883F84
:1096500038F0EFEFF0E0E81BF109ED59FB4F8081A6
:1096600080933E0480918608883F38F0EFEFF0E069
:10967000E81BF109ED59FB4F808180933D048091F7
:109680008708883F38F0EFEFF0E0E81BF109ED596B
:10969000FB4F808180933C0480918808883F38F09C
:1096A000EFEFF0E0E81BF109ED59FB4F808180936B
:1096B0003B048091A208883F38F0EFEFF0E0E81B10
:1096C000F109ED59FB4F808180933A048091A30802
:1096D000883F38F0EFEFF0E0E81BF109ED59FB4F60
:1096E0008081809339048091A408883F38F0EFEF9F
:1096F000F0E0E81BF109ED59FB4F808180933804BD
:109700008091A508883F38F0EFEFF0E0E81BF10901
:10971000ED59FB4F80818093370480918908883F01
:1097200038F0EFEFF0E0E81BF109ED59FB4F8081D5
:1097300080938A0180918D08883F38F0EFEFF0E048
:10974000E81BF109ED59FB4F8081809389018091DD
:109750008A08883F38F0EFEFF0E0E81BF109ED5997
:10976000FB4F80818093880180918E08883F38F07C
:10977000EFEFF0E0E81BF109ED59FB4F808180939A
:10978000870180919708883F38F0EFEFF0E0E81B01
:10979000F109ED59FB4F80818093860180919A08F1
:1097A000883F38F0EFEFF0E0E81BF109ED59FB4F8F
:1097B00080818093850180919B08883F38F0EFEF8E
:1097C000F0E0E81BF109ED59FB4F808180938401A3
:1097D00080919C08883F38F0EFEFF0E0E81BF1093A
:1097E000ED59FB4F8081809383018091C408883FAD
:1097F00038F0EFEFF0E0E81BF109ED59FB4F808105
:109800008093330A90914305992321F08091330A84
:10981000981720F08091330A882311F49093330A2B
:10982000809169088093730A8091CC088093540AD0
:109830008091A108883F38F0EFEFF0E0E81BF109D4
:10984000ED59FB4F8081809382018091BD08883F54
:1098500038F0EFEFF0E0E81BF109ED59FB4F8081A4
:1098600080938A0A80918C01282F33272F5F3F4FE6
:109870008CE398E2B9010E9407A170939B01609369
:109880009A0180913E04833380F080913D04282F1B
:1098900033272F5F3F4F8CE398E2B9010E9407A165
:1098A000709399016093980104C07093990160933B
:1098B00098018091AD080E948A498093340A809172
:1098C000560A882311F48093340A80917708809394
:1098D0007B0A8091760880933C0AE091BF08EE23D2
:1098E00009F449C081E080933604FF27EE0FFF1F83
:1098F000EE56F64F80819181805C9F4F14F4109258
:10990000360480919C0120913604821721F1833026
:10991000F8F43091C901222351F08CED95E0909339
:10992000380380933703332369F48EE209C088EC4F
:1099300090E09093380380933703332319F487E141
:109940008093C90185E080934C0420939C0103C05F
:10995000815080939C018091CA0A9091CB0A97FF15
:109960000FC080913604882359F08091D10580681A
:109970008093D10505C0E09336048AE080939C0172
:109980008091CA0A9091CB0A97FF1DC08091610413
:109990008823C9F0809136048823A9F080910A01B8
:1099A00090910B018F5F9F4F71F488E99AE3909338
:1099B00038038093370380E094EA90930B018093FF
:1099C0000A011092360480913604882321F0809198
:1099D0002404816003C0809124048E7F809324043A
:1099E000DF91CF910895A7E1B0E0E9EFFCE40C949A
:1099F00057A10E945B418091250499278471907042
:109A0000892B91F58091CD0882FF27C08091460473
:109A1000909147040097F1F022E088359207D4F442
:109A20009C0197FF02C02D5F3F4F359527953595D7
:109A30002795809181089927289FA001299F500D83
:109A4000389F500D1124CA0164E670E00E9407A1FE
:109A5000CB0106C08DE290E003C080918108992778
:109A600090932304809322042091200430912104B8
:109A700055E72033350759F410926D0410926C04A9
:109A800080913C0A9927909323048093220460914B
:109A90006C0470916D047A83698380913C0A9927E4
:109AA0000A966817790714F49A838983809162046F
:109AB000843608F06AC08091240482FD66C08091DB
:109AC0000A0590910B05009731F0019790930B05D3
:109AD00080930A050BC01092610490932704809331
:109AE0002604809125048D7E8093250480910201B7
:109AF0008A3011F0843110F0289A01C028988091A2
:109B0000260490912704895E9340E0F180910E0B2A
:109B10008536C0F180912204909123049A83898331
:109B20008091250480618093250480915D08A82F91
:109B3000BB27AA0FBB1FFD01E852F64F118210820E
:109B400080915E08282F3327220F331FC9018852C6
:109B5000964FFC0111821082AE56B64F11961C92A0
:109B60001E922E56364FD90111961C921E9280914C
:109B70006008E82FFF27EE0FFF1FEE56F64F118209
:109B80001082A3C510926104A0C5809162048D3833
:109B900008F471C59091C808992309F445C08091D3
:109BA000C908882309F440C0E92FFF27EE0FFF1FE3
:109BB000EE56F64F80819181C397BCF08091B10140
:109BC000823361F48091240485FF08C080912404CD
:109BD00080648093240480E38093C90180912404ED
:109BE0008F778093240486E917C0808191818E5CF1
:109BF0009F4FACF48091B101863941F480912404E7
:109C00008068809324048FE28093C90180912404AA
:109C10008F7B8093240482E38093B10105C08091FF
:109C200024048F7380932404809125048F7E809375
:109C300025049091820882E3989FC001112490939B
:109C40000B0580930A05E981FA81B9978CF0809120
:109C50006104882369F08091260490912704FFEF26
:109C60008F3F9F0729F00196909327048093260445
:109C700040912604509127044F3F510509F048F5C3
:109C80001092840410928504109286041092870426
:109C90001092800410928104109282041092830426
:109CA0001092F6041092F7041092F8041092F9043E
:109CB00010928C0410928D0410928E0410928F04D6
:109CC0008091240480628093240484E68093B1010F
:109CD00035C18091250482608093250480912404FD
:109CE00085FF98C08091440599279C0124703070AD
:109CF00082FD04C08091240486FF2AC080913D012A
:109D00008D3331F580911D04882311F180E5809316
:109D1000510484EF91E0A0E0B0E08093520490936E
:109D20005304A0935404B093550480935804909323
:109D30005904A0935A04B0935B0488EE93E0909387
:109D4000B0018093AF01232B19F08DE08093C901FE
:109D50008091430390914403A0914503B091460341
:109D600087399105A105B1058CF480915C0490912F
:109D70005D04A0915E04B0915F04825A9E4FAF4F84
:109D8000BF4F24F08091730A80FD21C088EE93E0DC
:109D90009093B0018093AF018091240486FF0FC09F
:109DA000109251048CE291E0A0E0B0E0809358045E
:109DB00090935904A0935A04B0935B0403C080E3CA
:109DC0008093C901809124048F71809324041092A0
:109DD00084041092850410928604109287041092D5
:109DE00080041092810410928204109283041092D5
:109DF0008C0410928D0410928E0410928F04495E90
:109E0000534008F49BC088EE93E09093270480931E
:109E1000260494C08091240487FF1AC080913D01DC
:109E2000863711F08D33A1F480911D04882381F0D1
:109E30008091C9088093510480EE91EBAFEFBFEFA2
:109E40008093520490935304A0935404B093550408
:109E50002091AF013091B00143E0283E340708F073
:109E600048C02F5F3F4F3093B0012093AF01109255
:109E70008404109285041092860410928704109234
:109E80008004109281041092820410928304109234
:109E90008C0410928D0410928E0410928F04809185
:109EA000430390914403A0914503B09146038C5223
:109EB0009140A040B0408093580490935904A093DF
:109EC0005A04B0935B04285E3340C1F580912404AA
:109ED00087FF34C080913D018B3281F18091240451
:109EE0008F778093240480912404806280932404DB
:109EF00025C080911D04882309F180913D0186379A
:109F000011F08D32D9F480915C0490915D04A091A0
:109F10005E04B0915F04885E9340A040B04074F44A
:109F20008091FC079091FD078D5A93403CF0109270
:109F3000B0011092AF018EE08093C90180915F085B
:109F4000E82FFF27EE0FFF1FEE56F64F808191811D
:109F5000813591050CF454C120916104222309F04C
:109F60004FC180916008E82FFF27EE0FFF1FEE56CC
:109F7000F64F808191818C3491050CF411C1809150
:109F80000C058F5F80930C05893C08F439C1209340
:109F90000C05109227041092260430915D08E32FDF
:109FA000FF27EE0FFF1FEE56F64F80819181873419
:109FB0009105B4F480915E08E82FFF27EE0FFF1F94
:109FC000EE56F64F808191810190F081E02DF7FFF0
:109FD00003C0F095E195FF4FE734F1050CF478C02C
:109FE00041E020915E08A22FBB27AA0FBB1FAE56EF
:109FF000B64F8D919C9111978734910544F0E32FD2
:10A00000FF27EE0FFF1FEE56F64F808191818D9155
:10A010009C918734910574F080915D08E82FFF27AB
:10A02000EE0FFF1FEE56F64F808191818734910528
:10A030000CF042E0E22FFF27EE0FFF1FEE56F64F27
:10A04000808191818634910574F480915D08E82FB8
:10A05000FF27EE0FFF1FEE56F64F80819181873468
:10A0600091050CF043E0E22FFF27EE0FFF1FEE56A5
:10A07000F64F808191818A5B9F4F74F480915D08D7
:10A08000E82FFF27EE0FFF1FEE56F64F80819181DC
:10A09000873491050CF044E0E22FFF27EE0FFF1FFD
:10A0A000EE56F64F808191818A5B9F4F74F48091C8
:10A0B0005D08E82FFF27EE0FFF1FEE56F64F808159
:10A0C0009181863491050CF445E0842F0E94503232
:10A0D00080915E08E82FFF27EE0FFF1FEE56F64F28
:10A0E000808191810190F081E02DF7FF03C0F09510
:10A0F000E195FF4F7E97CCF480915D08E82FFF2714
:10A10000EE0FFF1FEE56F64F808191818A5B9F4FC5
:10A1100064F481E08093EC0510924D0488EE93E0A6
:10A1200090933803809337036BC0809100010E94A5
:10A13000FB3180E00E94510A809183080E94AF9C0D
:10A140008091730A80FF10C08091180190911901CD
:10A15000875B934038F480911801909119018E5ECD
:10A16000924010F40E94771F81E00E94243E982FB5
:10A1700080934D0421E020933503579A8091D105B7
:10A18000882311F087E006C0992319F42093C901B0
:10A1900003C088E18093C90185E08093720527C0E0
:10A1A00080819181855B9F4F4CF580910C058F5F7D
:10A1B00080930C05893C20F12093610420930C05C9
:10A1C000109227041092260482E00E94243E982FC9
:10A1D00080934D048091D105882311F087E005C05C
:10A1E000992311F481E001C088E18093C90168E7F7
:10A1F00070E0809100010E94403D02C020930C0558
:10A2000080915F08E82FFF27EE0FFF1FEE56F64FF5
:10A21000808191818C599F4F0CF026C22091C008FB
:10A22000E22FFF27EF77F070EE0FFF1FE852F64F97
:10A2300080819181069714F084E606C08081918127
:10A240008B5F9F4F1CF48CE980930F058091610414
:10A25000E0916008882309F06AC1FF27EE0FFF1F15
:10A26000EE56F64F808191818C599F4F9CF48091DE
:10A27000CD0883FD0BC0E22FFF27EE0FFF1FEE5628
:10A28000F64F80819181855B9F4FDCF08091C00803
:10A290008823B9F08091CD0883FF46C18091C00822
:10A2A000E82FFF27EE0FFF1FEE56F64F80819181BA
:10A2B000875F9F4F0CF438C180910F05843609F0F9
:10A2C00033C120914D04222329F080912504886018
:10A2D0008093250480911A0190911B01A0911C018B
:10A2E000B0911D018093FE079093FF07A093000893
:10A2F000B093010810924303109244031092450357
:10A300001092460310925C0410925D0410925E0459
:10A3100010925F0410924C0310924D0310924E0362
:10A3200010924F03D0905D08ED2DFF27EE0FFF1F19
:10A33000EE56F64F808191818D599F4FACF48091FC
:10A340005E08E82FFF27EE0FFF1FEE56F64F8081C5
:10A3500091810190F081E02DF7FF03C0F095E19528
:10A36000FF4FE436F10534F48091C008882311F4DE
:10A3700080930D0580910D058F5F80930D058E3FB5
:10A3800008F464C110920D058091D105882309F06D
:10A39000BEC0222309F4BBC080914805882309F080
:10A3A000B6C081E090E0909327048093260481E07A
:10A3B000809361041092F6041092F7041092F8044E
:10A3C0001092F90410928C0410928D0410928E0455
:10A3D00010928F04109288041092890410928A04BB
:10A3E00010928B0480917808E82EFF240027112713
:10A3F0008091770A9091780A9C01442737FD409517
:10A40000542FC801B7010E94C8A0DC01CB01809382
:10A410009C0490939D04A0939E04B0939F0480910C
:10A42000870A9091880A9C01442737FD4095542F54
:10A43000C801B7010E94C8A0DC01CB01809394043D
:10A4400090939504A0939604B09397048091BC04D4
:10A450009091BD04A091BE04B091BF048093980474
:10A4600090939904A0939A04B0939B048091B404B0
:10A470009091B504A091B604B091B7048093900474
:10A4800090939104A0939204B09393041092840447
:10A490001092850410928604109287041092800412
:10A4A00010928104109282041092830484E68093B7
:10A4B0004C0484E38093C901ED2DFF27EE0FFF1FAD
:10A4C000EE56F64F8081918190932B0480932A045D
:10A4D00080915E08E82FFF27EE0FFF1FEE56F64F24
:10A4E0008081918190932904809328041092EE0436
:10A4F0001092EF041092F0041092F1041092F20402
:10A500001092F3041092F4041092F5049FC08CEDA5
:10A5100095E0909338038093370380914D0488230E
:10A5200009F094C081E08DC010920D058FC0FF2707
:10A53000EE0FFF1FEE56F64F808191818536910513
:10A540009CF08091CD0883FD0BC0E22FFF27EE0F1A
:10A55000FF1FEE56F64F80819181855B9F4FDCF0A7
:10A560008091C0088823B9F08091CD0883FF6CC02A
:10A570008091C008E82FFF27EE0FFF1FEE56F64F21
:10A58000808191818E5C9F4F0CF05EC080910F05A1
:10A590008C3909F059C080915D08E82FFF27EE0F34
:10A5A000FF1FEE56F64F808191818D599F4FACF47D
:10A5B00080915E08E82FFF27EE0FFF1FEE56F64F43
:10A5C000808191810190F081E02DF7FF03C0F0952B
:10A5D000E195FF4FE436F1053CF48091C0088823F3
:10A5E00019F480930E0518C010928404109285040B
:10A5F00010928604109287041092800410928104B5
:10A6000010928204109283041092730410927204C8
:10A61000109271041092700480910E058F5F8093E8
:10A620000E058B3F98F01092610410920E05109267
:10A63000270410922604809124048F7180932404AF
:10A6400086E28093C90102C010920E058091200419
:10A650009091210433E0883E9307B8F501969093DA
:10A6600021048093200431C010920F051092210420
:10A67000109220042AC02E5E324038F18091920A56
:10A680009091930A8059914000F580915C049091DB
:10A690005D04A0915E04B0915F048C5D9540A04084
:10A6A000B0409CF480E395E79093210480932004CC
:10A6B00080912604909127048A5E934030F089EEC1
:10A6C00093E0909327048093260480913C0181506D
:10A6D00080933C0180913C018F3F21F080912504C3
:10A6E00084FF2BC40E94A649C0907308D090560ADC
:10A6F000DD2009F48FC080911805909119059C0107
:10A70000220F331F280F391F80915D08A82FBB2708
:10A71000AA0FBB1F8D010E56164F6C2D7727F8011F
:10A7200080819181869FA001879F500D969F500D3B
:10A730001124240F351F37FF02C02D5F3F4F7901D1
:10A74000F594E794F594E794F0921905E0921805D2
:10A7500080911A0590911B05AC01440F551F480FBD
:10A76000591F80915E08A82EBB24AA0CBB1CE2E9ED
:10A770008E2EE9E09E2E8A0C9B1CF4018081918133
:10A78000869F9001879F300D969F300D1124420FB8
:10A79000531F57FF02C04D5F5F4F55954795559525
:10A7A0004795F8018081918190932B0480932A042E
:10A7B000F401808191819093290480932804A85208
:10A7C000B64F80917408282F33278D919C91829FDA
:10A7D000B001839F700D929F700D1124CB018E0DDF
:10A7E0009F1D909319058093180588ED99E0A80E98
:10A7F000B91ED5018D919C91829FF001839FF00D30
:10A80000929FF00D11244E0F5F1F50931B05409334
:10A810001A0548C080913E04E0915D0860915E0891
:10A8200020912A0430912B0440912804509129044E
:10A83000823368F0FF27EE0FFF1FEE56F64F808140
:10A840009181821B930B20913C0433270BC0FF277F
:10A85000EE0FFF1FEE56F64F80819181821B930B06
:10A860002C2D3327829FD001839FB00D929FB00D76
:10A870001124B0931905A0931805E62FFF27EE0FBA
:10A88000FF1FEE56F64F80819181841B950B829FAE
:10A89000F001839FF00D929FF00D1124F0931B05A2
:10A8A000E0931A0580913604882309F451C0DD2015
:10A8B00009F44EC0809118059091190597FD0396F3
:10A8C000DC01B595A795B595A79580911A0590914E
:10A8D0001B0597FD0396FC01F595E795F595E79522
:10A8E0008091C201682F772767FD70956A9F90015C
:10A8F0006B9F300D7A9F300D112480914A05482FAF
:10A90000552747FD50954E9FC0014F9F900D5E9F6C
:10A91000900D1124280F391F37FF02C0295F3F4FC8
:10A9200093E0359527959A95E1F73093730420933A
:10A9300072046E9F90016F9F300D7E9F300D112429
:10A940004A9FC0014B9F900D5A9F900D112450C0FB
:10A950008091BE08E82FFF27EE0FFF1FEC5BFE4F34
:10A96000848587FD8F5F982F95959093C201808194
:10A9700087FD8F5F859580934A05E92FFF27E7FDC7
:10A98000F095A0911805B0911905EA9F9001EB9FF1
:10A99000300DFA9F300D1124682F772767FD7095D1
:10A9A00040911A0550911B05649FC001659F900D51
:10A9B000749F900D1124280F391F37FF02C0295FA3
:10A9C0003F4F83E0359527958A95E1F730937304DF
:10A9D00020937204E49F9001E59F300DF49F300DA9
:10A9E00011246A9FC0016B9F900D7A9F900D1124D6
:10A9F000281B390B37FF02C0295F3F4F03E0359515
:10AA000027950A95E1F730937104209370048091A3
:10AA10006008E82FFF27EE0FFF1FEE56F64F8081EC
:10AA20009181909581959F4F90936F0480936E04D0
:10AA30008530910514F0049705C0FFEF8C3F9F0708
:10AA400034F4049690936F0480936E0404C01092C3
:10AA50006F0410926E0480913605882309F43EC07D
:10AA6000282F3327809172049091730497FD0796E5
:10AA700013E0959587951A95E1F7289FA001299FE6
:10AA8000500D389F500D1124CA0157FD0F96B4E0A8
:10AA900095958795BA95E1F7909373048093720426
:10AAA000809170049091710497FD0796A3E09595AD
:10AAB0008795AA95E1F7289FB001299F700D389FCF
:10AAC000700D1124CB0177FD0F96F4E095958795D5
:10AAD000FA95E1F79093710480937004A09072044A
:10AAE000B09073048091390590913A05A81AB90A7B
:10AAF000B0927304A09272040091700410917104DA
:10AB00008091370590913805081B190B109371043B
:10AB10000093700480915F08E82FFF27EE0FFF1F5E
:10AB2000EE56F64FE080F1808FE790E0E80EF91ED8
:10AB3000F0926D04E0926C04809191019927AA270C
:10AB400097FDA095BA2FBC01CD010E943CA0DC016D
:10AB5000CB0120E030E040E251E4BC01CD010E9495
:10AB6000AA9FDC01CB01BC01CD010E940EA0DC013B
:10AB7000CB018093810A80918F019927AA2797FDA5
:10AB8000A095BA2FBC01CD010E943CA0DC01CB01F5
:10AB900020E030E040E251E4BC01CD010E94AA9FD8
:10ABA000DC01CB01BC01CD010E940EA0DC01CB0178
:10ABB00080932E0A80918E018093450A8091F8053A
:10ABC00080FF59C080918A0A813808F454C080916E
:10ABD000F105992787FD90952C2D3327829FD00171
:10ABE000839FB00D929FB00D1124AA0EBB1EB09290
:10ABF0007304A09272048091F205992787FD9095C5
:10AC0000829FF001839FF00D929FF00D11240E0F93
:10AC10001F1F10937104009370048091F305282F77
:10AC2000332727FD309580916E0490916F04820F39
:10AC3000931F90936F0480936E048091F505282FE5
:10AC4000332727FD309580916E089927289FA00112
:10AC5000299F500D389F500D11245093430140936C
:10AC600042018091F40599278E159F0524F4909355
:10AC70006D0480936C0480916C0490916D0497FF37
:10AC800004C010926D0410926C048091730A82FFCC
:10AC900002C01092560A4091720450917304CA0186
:10ACA00057FD03969C01359527953595279537FFD8
:10ACB00003C0309521953F4F80912E0490912F0431
:10ACC00082179307B4F4CA0157FF03C0909581958A
:10ACD0009F4F97FD039695958795959587959093AA
:10ACE0002F0480932E048536910544F084E690E08D
:10ACF00001C0019790932F0480932E04409170041B
:10AD000050917104CA0157FD03969C013595279512
:10AD10003595279537FF03C0309521953F4F80919A
:10AD20002C0490912D0482179307B4F4CA0157FFA5
:10AD300003C0909581959F4F97FD039695958795B4
:10AD40009595879590932D0480932C0485369105D5
:10AD500044F084E690E001C0019790932D04809325
:10AD60002C048091250484FF08C010922F041092B7
:10AD70002E0410922D0410922C0450915E08E52FA1
:10AD8000FF27EE0FFF1FEE56F64F40919808242F35
:10AD90003327808191812817390744F48091CA08AC
:10ADA00082FF04C081E08093430413C0E52FFF2796
:10ADB000EE0FFF1FEE56F64F842F9927209199082A
:10ADC000821B9109208131812817390714F41092D0
:10ADD000430440915E08E42FFF27EE0FFF1FEE565D
:10ADE000F64F50919808852F992722273327281B43
:10ADF000390B808191818217930744F48091CA08AE
:10AE000083FF04C081E08093420416C08091420415
:10AE1000882391F0E42FFF27EE0FFF1FEE56F64F29
:10AE2000809199089927851B91092081318182178A
:10AE3000930714F41092420450915D08E52FFF2708
:10AE4000EE0FFF1FEE56F64F40919808242F332740
:10AE5000808191812817390744F48091CA0880FFC6
:10AE600004C081E08093400417C08091400488238F
:10AE700099F0E52FFF27EE0FFF1FEE56F64F842FB8
:10AE8000992720919908821B9109208131812817E7
:10AE9000390714F41092400440915D08E42FFF2715
:10AEA000EE0FFF1FEE56F64F50919808852F992709
:10AEB00022273327281B390B808191818217930722
:10AEC00044F48091CA0881FF04C081E0809341046A
:10AED00016C080914104882391F0E42FFF27EE0FE4
:10AEE000FF1FEE56F64F809199089927851B91090F
:10AEF000208131818217930714F4109241048091CC
:10AF00004304882319F480914204811181E08093E5
:10AF1000440480914004882321F4809141048823D3
:10AF200051F081E080934504109244041092430450
:10AF30001092420402C08093450480914404882307
:10AF400021F480914504882369F08091970899271E
:10AF500069817A818617970714F49A83898381E03F
:10AF6000809378048091240499279C012470307088
:10AF700082FF2DC08091390590913A059095819579
:10AF80009F4F909373048093720480913705909142
:10AF90003805909581959F4F90937104809370042C
:10AFA00080919F019091A00190936D0480936C0417
:10AFB0008091730A8B778B668093730A8091540A11
:10AFC0008C7B8093540A88EC80933F041EC0809150
:10AFD000250484FF1AC030936F0420936E043093CD
:10AFE00073042093720430937104209370049AE5E3
:10AFF0009093810A88E78093560A90932E0A809353
:10B00000450A10924404109245048091480A909198
:10B01000490AA0914A0AB0914B0A2091BC04309190
:10B02000BD044091BE045091BF04820F931FA41F22
:10B03000B51F8093480A9093490AA0934A0AB09397
:10B040004B0A8091500A9091510AA091520AB091F6
:10B05000530A2091B4043091B5044091B604509144
:10B06000B704820F931FA41FB51F8093500A9093BB
:10B07000510AA093520AB093530A80913D0A9091CD
:10B080003E0AA0913F0AB091400A2091B804309145
:10B09000B9044091BA045091BB042B833C834D8387
:10B0A0005E83820F931FA41FB51F80933D0A909368
:10B0B0003E0AA0933F0AB093400A80912F0A9091D4
:10B0C000300AA091310AB091320A4091B0045091F7
:10B0D000B1046091B2047091B3044F8358876987BB
:10B0E0007A87840F951FA61FB71F80932F0A90930E
:10B0F000300AA093310AB093320A1091560A1123F4
:10B1000009F066C080913E04823308F061C08091EE
:10B11000690882FD5DC01092BC041092BD041092BB
:10B12000BE041092BF041092B4041092B5041092A1
:10B13000B6041092B70410929C0410929D041092D1
:10B140009E0410929F041092940410929504109201
:10B1500096041092970410928C0410928D04109211
:10B160008E0410928F041092F6041092F70410923D
:10B17000F8041092F9041092A0041092A104109205
:10B18000A2041092A3048091AD019091AE0190931E
:10B190007B0480937A04AA2797FDA095BA2F20916B
:10B1A0003E0130913F014091400150914101BC016D
:10B1B000CD010E94C8A0DC01CB018093830A90934B
:10B1C000840AA093850AB093860A81E080934C0498
:10B1D000509145045B87552381F480914404882372
:10B1E00061F4112309F065C080913E04823308F0B8
:10B1F00060C08091690882FD5CC01092AC0410921E
:10B20000AD041092AE041092AF041092A8041092F4
:10B21000A9041092AA041092AB041092480A10924A
:10B22000490A10924A0A10924B0A1092500A109240
:10B23000510A1092520A1092530A10923D0A10922B
:10B240003E0A10923F0A1092400A10922F0A109262
:10B25000300A1092310A1092320A80919C04909127
:10B260009D04A0919E04B0919F04809398049093B4
:10B270009904A0939A04B0939B04809194049091B4
:10B280009504A0919604B0919704809390049093B4
:10B290009104A0939204B0939304109248031092E7
:10B2A0004703109249041092480410924B041092E4
:10B2B0004A048091690882FD04C080913E04823373
:10B2C00018F01092560A04C0809190018093560A9B
:10B2D0006B85662309F0E0C180914404882309F05E
:10B2E000DBC18091FC079091FD07815092402CF4C6
:10B2F00080916104882309F4CFC19090030BA09042
:10B3000078082090770A3090780A4090870A509009
:10B31000880A6091BC047091BD048091BE04909134
:10B32000BF042091B4043091B5044091B60450910B
:10B33000B7042A8B3B8B4C8B5D8B19140CF0B9C076
:10B34000BB24CC24DD24A60195010E943CA17901F7
:10B350008A018091CC0A9091CD0A281A390AC1013C
:10B36000AA2797FDA095BA2FE81AF90A0A0B1B0B1A
:10B370006A897B898C899D89A60195010E943CA1DF
:10B3800059016A018091CE0A9091CF0A481A590A50
:10B39000C201AA2797FDA095BA2FA81AB90ACA0A0E
:10B3A000DB0A292C332427FC3094432C532CC8016E
:10B3B000B701A20191010E94C8A097FF04C061508B
:10B3C0007E4F8F4F9F4F3B014C0109E0959487942E
:10B3D000779467940A95D1F7C601B501A20191014E
:10B3E0000E94C8A097FF04C061507E4F8F4F9F4FAF
:10B3F0005B016C0119E0D594C794B794A7941A9592
:10B40000D1F780912E0490912F04813491053CF462
:10B4100080912C0490912D0481349105D4F0D401B5
:10B42000C30197FE03C00196A11DB11D3C014D0152
:10B430009594879477946794D601C501D7FE03C08D
:10B440000196A11DB11D5C016D01D594C794B794FF
:10B45000A7948091050B282F332727FD3095432F84
:10B46000532F261537054805590514F439014A01AB
:10B47000992787FD9095909581959F4FAA2797FDD5
:10B48000A095BA2F681679068A069B0614F43C012B
:10B490004D012A153B054C055D0514F459016A015F
:10B4A000A816B906CA06DB060CF0CEC05C016D0119
:10B4B000CBC0EA2CFF2400271127A80197010E9486
:10B4C0003CA139014A01C101AA2797FDA095BA2FD5
:10B4D000681A790A8A0A9B0A6A897B898C899D89FC
:10B4E000A80197010E943CA159016A01C201AA2743
:10B4F00097FDA095BA2FA81AB90ACA0ADB0AD40187
:10B50000C30197FE03C00F96A11DB11D3C014D0163
:10B51000F4E09594879477946794FA95D1F7D601DF
:10B52000C501D7FE03C00F96A11DB11D5C016D01C1
:10B53000E4E0D594C794B794A794EA95D1F78091A5
:10B540002E0490912F04813491053CF480912C04B9
:10B5500090912D0481349105A4F0C401B30123E03E
:10B5600030E040E050E00E943CA139014A01C601B0
:10B57000B50123E030E040E050E00E943CA15901D9
:10B580006A0180916008E82FFF27EE0FFF1FEE563B
:10B59000F64F808191810190F081E02DF7FF03C08B
:10B5A000F095E195FF4F7A97A4F0C401B30123E031
:10B5B00030E040E050E00E943CA139014A01C60160
:10B5C000B50123E030E040E050E00E943CA1590189
:10B5D0006A0189E18093AB0131E263167104810451
:10B5E00091042CF070E2672E712C812C912C40EE8E
:10B5F00064164FEF74064FEF84064FEF940644F441
:10B6000060EE662E6FEF762E6FEF862E6FEF962E22
:10B6100051E2A516B104C104D1042CF050E2A52ECC
:10B62000B12CC12CD12C60EEA6166FEFB6066FEFD1
:10B63000C6066FEFD60644F440EEA42E4FEFB42EAC
:10B640004FEFC42E4FEFD42E80919C0490919D0417
:10B65000A0919E04B0919F0486199709A809B90981
:10B6600080939C0490939D04A0939E04B0939F04A8
:10B670008091940490919504A0919604B0919704C0
:10B680008A199B09AC09BD09809394049093950491
:10B69000A0939604B0939704809147039091480338
:10B6A0008F3F910509F008F4C9C57B85772309F020
:10B6B00053C580914404882309F04EC580917804D5
:10B6C000882309F049C58091A0088C87882309F454
:10B6D00043C58091560A882309F43EC58091480AE3
:10B6E0009091490AA0914A0AB0914B0AB7FF04C051
:10B6F00081509F4FAF4FBF4FE92EFA2E0B2F1127CE
:10B7000007FD1A95E092480AF092490A00934A0A06
:10B7100010934B0A8091500A9091510AA091520ABD
:10B72000B091530AB7FF04C081509F4FAF4FBF4F36
:10B73000892F9A2FAB2FBB27A7FDBA958D879E87A0
:10B74000AF87B88B8093500A9093510AA093520A06
:10B75000B093530A80917808A82EBB24CC24DD2412
:10B760002091AC043091AD044091AE045091AF04EF
:10B77000C601B5010E94C8A097FF04C061507F4F69
:10B780008F4F9F4F672E782E892E992487FC9A948D
:10B790006092AC047092AD048092AE049092AF04BB
:10B7A0002091A8043091A9044091AA045091AB04BF
:10B7B000C601B5010E94C8A097FF04C061507F4F29
:10B7C0008F4F9F4F272E382E492E552447FC5A94D1
:10B7D0002092A8043092A9044092AA045092AB048B
:10B7E0008091A4049091A504A091A604B091A7040F
:10B7F000B7FF04C081509F4FAF4FBF4F892F9A2F83
:10B80000AB2FBB27A7FDBA958093A4049093A50402
:10B81000A093A604B093A704D801C701861997097D
:10B82000A809B9098093020590930305A093040524
:10B83000B093050520919F08E22EFF2400271127D1
:10B84000BC01CD01A80197010E943CA159016A01E8
:10B850002093100530931105409312055093130562
:10B860008D859E85AF85B88982199309A409B5098C
:10B870008093060590930705A0930805B0930905EA
:10B88000BC01CD01A80197010E943CA120931405A1
:10B89000309315054093160550931705D601C50141
:10B8A000D7FE04C081509F4FAF4FBF4F892F9A2FB3
:10B8B000AB2FBB27A7FDBA9590934904809348040A
:10B8C00057FF04C021503F4F4F4F5F4FBB2757FDDD
:10B8D000BA95A52F942F832F90934B0480934A04FD
:10B8E00080912E0490912F0481349105DCF4809195
:10B8F0002C0490912D0481349105A4F4809160086A
:10B90000E82FFF27EE0FFF1FEE56F64F8081918143
:10B910000190F081E02DF7FF03C0F095E195FF4F16
:10B920007A97E4F08091030B8F3FC1F48091480433
:10B930009091490497FD01969595879590934904B8
:10B940008093480480914A0490914B0497FD01969E
:10B950009595879590934B0480934A0480913D0A76
:10B9600090913E0AA0913F0AB091400AB7FF04C0EF
:10B9700081509F4FAF4FBF4F892F9A2FAB2FBB27BF
:10B98000A7FDBA9580933D0A90933E0AA0933F0A83
:10B99000B093400A80912F0A9091300AA091310A09
:10B9A000B091320AB7FF04C081509F4FAF4FBF4FD5
:10B9B000892F9A2FAB2FBB27A7FDBA9580932F0A0B
:10B9C0009093300AA093310AB093320A8091BC045C
:10B9D0009091BD04A091BE04B091BF042B813C8125
:10B9E0004D815E81281B390B4A0B5B0B2093FA04B7
:10B9F0003093FB044093FC045093FD048091B40405
:10BA00009091B504A091B604B091B704EF80F8848A
:10BA100009851A85E81AF90A0A0B1B0BE092FE0445
:10BA2000F092FF0400930005109301052093020596
:10BA3000309303054093040550930505E0920605F5
:10BA4000F09207050093080510930905809198046A
:10BA500090919904A0919A04B0919B04821B930B3E
:10BA6000A40BB50B8093980490939904A0939A0427
:10BA7000B0939B048091900490919104A0919204C2
:10BA8000B09193048E199F09A00BB10B8093900481
:10BA900090939104A0939204B09393049C8599236E
:10BAA000E1F02091760430917704213831054CF093
:10BAB0008091CE049091CF0401969093CF0480930F
:10BAC000CE0420583F4F4CF48091CE049091CF0487
:10BAD00001979093CF048093CE0410927704109234
:10BAE000760481E090E090931D0580931C05E09022
:10BAF0000205F09003050091040510910505D80199
:10BB0000C70117FF07C088279927DC018E199F09F5
:10BB1000A00BB10B81509240A040B04034F084E0C3
:10BB200090E090931D0580931C05809122059091D3
:10BB30002305A0912405B09125052091480A309154
:10BB4000490A40914A0A50914B0A821B930BA40B5D
:10BB5000B50B815E914BAF4FBF4F8F539C49A040B7
:10BB6000B04028F08091040B89310CF4FFC021E033
:10BB7000E21620E1F20620E0020720E012070CF4B2
:10BB800073C080911E05882309F46AC0D801C701DB
:10BB900017FF07C088279927DC018E199F09A00B82
:10BBA000B10B9C01AD01B7FF04C021503E4F4F4F78
:10BBB0005F4FF9E05595479537952795FA95D1F759
:10BBC00080911C0590911D05820F931F90931D0578
:10BBD00080931C05D801C70117FF03C00796A11D5C
:10BBE000B11DE3E0B595A79597958795EA95D1F7AF
:10BBF0008093100590931105A0931205B09313053F
:10BC000089589341A040B04064F088E893E1A0E0F7
:10BC1000B0E08093100590931105A0931205B093A6
:10BC20001305209110053091110540911205509196
:10BC3000130557FF04C021503F4F4F4F5F4F232F35
:10BC4000342F452F552747FD5A95809148049091F0
:10BC50004904820F931F909349048093480406C0BF
:10BC600081E080931E0502C010921E0540E0E4169C
:10BC700040EFF4064FEF04074FEF14070CF073C0CA
:10BC800080911F05882309F46AC0D801C70117FFF6
:10BC900007C088279927DC018E199F09A00BB10BDB
:10BCA0009C01AD01B7FF04C021503E4F4F4F5F4F85
:10BCB00069E055954795379527956A95D1F7809115
:10BCC0001C0590911D05820F931F90931D05809375
:10BCD0001C05D801C70117FF03C00796A11DB11DA0
:10BCE00023E0B595A795979587952A95D1F78093E9
:10BCF000100590931105A0931205B0931305885772
:10BD00009C4EAF4FBF4F64F488E79CEEAFEFBFEFA0
:10BD10008093100590931105A0931205B09313051D
:10BD20002091100530911105409112055091130595
:10BD300057FF04C021503F4F4F4F5F4F232F342FE9
:10BD4000452F552747FD5A95809148049091490405
:10BD5000820F931F909349048093480411C081E09F
:10BD600080931F050DC010921F050AC010921D057B
:10BD700010921C0584E690E09093AA018093A9019B
:10BD80006C85262F332780911C0590911D0528175F
:10BD9000390724F430931D0520931C051091040BE2
:10BDA000112379F0212F332727FD309580911C0531
:10BDB00090911D052817390724F430931D05209311
:10BDC0001C05409102055091030560910405709196
:10BDD0000505413851056105710574F08091D20463
:10BDE0009091D30420911C0530911D05820F931F63
:10BDF0009093D3048093D20440585F4F6F4F7F4F8E
:10BE000074F48091D2049091D30420911C05309158
:10BE10001D05821B930B9093D3048093D20481E081
:10BE200090E090931D0580931C05C0900605D0906E
:10BE30000705E0900805F0900905D701C601F7FE57
:10BE400007C088279927DC018C199D09AE09BF0915
:10BE500081509240A040B04034F084E090E0909354
:10BE60001D0580931C058091260590912705A091C2
:10BE70002805B09129052091500A3091510A40912E
:10BE8000520A5091530A821B930BA40BB50B815E8F
:10BE9000914BAF4FBF4F8F539C49A040B04018F01B
:10BEA00019310CF4FFC021E0C21620E1D20620E0D7
:10BEB000E20620E0F2060CF473C08091200588238E
:10BEC00009F46AC0D701C601F7FE07C08827992781
:10BED000DC018C199D09AE09BF099C01AD01B7FFBA
:10BEE00004C021503E4F4F4F5F4F09E05595479595
:10BEF000379527950A95D1F780911C0590911D05DE
:10BF0000820F931F90931D0580931C05D701C601D6
:10BF1000F7FE03C00796A11DB11D13E0B595A795C7
:10BF2000979587951A95D1F78093140590931505E9
:10BF3000A0931605B093170589589341A040B040CF
:10BF400064F088E893E1A0E0B0E08093140590935A
:10BF50001505A0931605B09317052091140530918F
:10BF60001505409116055091170557FF04C0215043
:10BF70003F4F4F4F5F4F232F342F452F552747FDFE
:10BF80005A9580914A0490914B04820F931F90938D
:10BF90004B0480934A0406C081E08093200502C0D0
:10BFA0001092200540E0C41640EFD4064FEFE4069F
:10BFB0004FEFF4060CF073C080912105882309F43B
:10BFC0006AC0D701C601F7FE07C088279927DC01A0
:10BFD0008C199D09AE09BF099C01AD01B7FF04C0D2
:10BFE00021503E4F4F4F5F4FE9E0559547953795AC
:10BFF0002795EA95D1F780911C0590911D05820F38
:10C00000931F90931D0580931C05D701C601F7FE71
:10C0100003C00796A11DB11D73E0B595A79597952F
:10C0200087957A95D1F78093140590931505A09381
:10C030001605B093170588579C4EAF4FBF4F64F459
:10C0400088E79CEEAFEFBFEF809314059093150542
:10C05000A0931605B093170520911405309115058E
:10C06000409116055091170557FF04C021503F4FCE
:10C070004F4F5F4F232F342F452F552747FD5A959C
:10C0800080914A0490914B04820F931F90934B042C
:10C0900080934A0411C081E0809321050DC0109265
:10C0A00021050AC010921D0510921C0584E690E03F
:10C0B0009093AA018093A9016C85262F3327809144
:10C0C0001C0590911D052817390724F430931D0590
:10C0D00020931C058091040B882379F0282F3327A7
:10C0E00027FD309580911C0590911D052817390773
:10C0F00024F430931D0520931C05409106055091B2
:10C1000007056091080570910905413851056105E1
:10C11000710574F08091D0049091D10420911C0598
:10C1200030911D05820F931F9093D1048093D0040A
:10C1300040585F4F6F4F7F4FCCF48091D004909167
:10C14000D10420911C0530911D05821B930B909307
:10C15000D1048093D0040AC010924B0410924A0478
:10C160001092490410924804109278048091560A63
:10C17000882341F410924B0410924A04109249040F
:10C18000109248048091480A9091490AA0914A0A65
:10C19000B0914B0A8093220590932305A093240528
:10C1A000B09325058091500A9091510AA091520AAE
:10C1B000B091530A8093260590932705A0932805F4
:10C1C000B09329051092AC041092AD041092AE0405
:10C1D0001092AF041092A8041092A9041092AA041D
:10C1E0001092AB041092A4041092A5041092A6041D
:10C1F0001092A7041092480A1092490A10924A0A13
:10C2000010924B0A1092500A1092510A1092520A40
:10C210001092530A10923D0A10923E0A10923F0A61
:10C220001092400A10922F0A1092300A1092310A8E
:10C230001092320A1092480310924703E0906E0465
:10C24000F0906F04C701F7FE04C0882799278E1964
:10C250009F0904973CF08091730A84FD03C082E338
:10C2600080934C0410917508A12EBB24CC24DD24AE
:10C27000B701882777FD8095982F9701F7FE04C0B6
:10C28000222733272E193F09442737FD4095542F85
:10C290000E94C8A09B01AC01C601B5010E94C8A0C4
:10C2A00097FF04C061507E4F8F4F9F4F59E0959587
:10C2B0008795779567955A95D1F79B01812F992797
:10C2C0008E9DD0018F9DB00D9E9DB00D1124CD018E
:10C2D000B7FD03969595879595958795280F391FF6
:10C2E00080912004909121048150924010F020E030
:10C2F00030E080914E0490914F04280F391F44275D
:10C3000037FD4095542F2093F6043093F704409363
:10C31000F8045093F90480918C0490918D04A091BD
:10C320008E04B0918F04821B930BA40BB50B8093EA
:10C330008C0490938D04A0938E04B0938F04815548
:10C34000934CA040B04064F080E593ECA0E0B0E0F6
:10C3500080938C0490938D04A0938E04B0938F04EB
:10C3600080918C0490918D04A0918E04B0918F04E3
:10C37000805B9C43AF4FBF4F64F480EB9CE3AFEF17
:10C38000BFEF80938C0490938D04A0938E04B093A0
:10C390008F044090AD015090AE0157FCFFC08091DA
:10C3A000730A83FFFBC080913E04833308F0F6C01C
:10C3B0008091AC0181508093AC01882309F0F2C0D8
:10C3C0008DE08093AC018091BC049091BD04A0915C
:10C3D000BE04B091BF04B7FF04C081509E4FAF4F61
:10C3E000BF4F09E0B595A795979587950A95D1F721
:10C3F0007C0197FF04C0F094E194F108F3948091DC
:10C40000B4049091B504A091B604B091B704B7FFFD
:10C4100004C081509E4FAF4FBF4F19E0B595A7950F
:10C42000979587951A95D1F79C0197FF03C0309592
:10C4300021953F4FE216F3060CF47901B701F7FEA0
:10C4400002C0695F7F4F8B01B3E015950795BA95E0
:10C45000E1F70E5F1F4F6090830A7090840A80900E
:10C46000850A9090860A20913E0130913F014091CB
:10C47000400150914101C401B3010E943CA1590106
:10C480006A0130932D0A20932C0A421A530AC201E2
:10C49000845E9D4F68E671E00E9407A19C01245BC9
:10C4A00030408091A9019091AA01009731F0019745
:10C4B0009093AA018093A9011BC049E1E416F104FD
:10C4C000BCF48091760490917704820F931F90932F
:10C4D00077048093760480914C04882349F081503E
:10C4E00080934C04882321F4B0927B04A0927A04B8
:10C4F0008091A9019091AA01892BF9F48091AB0157
:10C500009927289FB001299F700D389F700D112425
:10C51000CB01B8010E9407A1CB01AA2797FDA095E6
:10C52000BA2F680E791E8A1E9B1E6092830A709233
:10C53000840A8092850A9092860A80914C0488230E
:10C5400069F580917A0490917B0420912C0A3091B6
:10C550002D0A821B930B845E9D4F68E671E00E945A
:10C5600007A19C01245B3040809194018695992716
:10C57000289FD001299FB00D389FB00D11249D0137
:10C58000B7FF02C0215F3F4FA4E035952795AA95DC
:10C59000E1F730934F0420934E0404C010924F04EF
:10C5A00010924E0480917804882381F010928004C8
:10C5B00010928104109282041092830410928404D9
:10C5C000109285041092860410928704009145040D
:10C5D0000023F1F48091560A282F3327442755274A
:10C5E0008091BC049091BD04A091BE04B091BF04A1
:10C5F000BC01CD010E94C8A0DC01CB01BC01CD0172
:10C6000028EF3AE240E050E00E943CA1390102C02C
:10C6100066247724109144041123F1F48091560A82
:10C62000282F3327442755278091B4049091B504CF
:10C63000A091B604B091B704BC01CD010E94C8A07E
:10C64000DC01CB01BC01CD0128EF3AE240E050E033
:10C650000E943CA1290102C0442455248091290A4A
:10C6600090912A0A893C91051CF088EC90E005C065
:10C6700088539F4F34F488E39FEF90932A0A809366
:10C68000290A8091350A9091360A893C91051CF05F
:10C6900088EC90E005C088539F4F34F488E39FEF07
:10C6A0009093360A8093350A8091560A2091810A28
:10C6B0006091370A7091380A882309F040C0CB0195
:10C6C000AA2797FDA095BA2FA22EBB24CC24DD2447
:10C6D000BC01CD01A60195010E94C8A097FF04C02E
:10C6E000615C7F4F8F4F9F4FF6E0959587957795CB
:10C6F0006795FA95D1F77093380A6093370A80915D
:10C70000270A9091280AAA2797FDA095BA2FBC0165
:10C71000CD01A60195010E94C8A097FF04C0615CED
:10C720007F4F8F4F9F4FE6E095958795779567955B
:10C73000EA95D1F77093280A6093270A6FC0CB015E
:10C74000AA2797FDA095BA2FA22EBB24CC24DD24C6
:10C75000BC01CD01A60195010E94C8A09B01AC01BE
:10C760008091290A90912A0AAA2797FDA095BA2FAD
:10C7700067E0880F991FAA1FBB1F6A95D1F7280F82
:10C78000391F4A1F5B1F57FF04C0215C3F4F4F4FAB
:10C790005F4FA6E05595479537952795AA95D1F710
:10C7A000C301820F931F9093380A8093370A8091B8
:10C7B000270A9091280AAA2797FDA095BA2FBC01B5
:10C7C000CD01A60195010E94C8A09B01AC018091FA
:10C7D000350A9091360AAA2797FDA095BA2FF7E05F
:10C7E000880F991FAA1FBB1FFA95D1F7280F391F71
:10C7F0004A1F5B1F57FF04C0215C3F4F4F4F5F4FE5
:10C80000E6E05595479537952795EA95D1F7C2010A
:10C81000820F931F9093280A8093270A80917C0AA5
:10C8200090917D0A880F991FAA2797FDA095BA2F8E
:10C8300020912E0A332744275527BC01CD010E94A1
:10C84000C8A05B016C0197FF08C02FE330E040E017
:10C8500050E0A20EB31EC41ED51E76E0D594C79438
:10C86000B794A7947A95D1F78091450A282F33275A
:10C87000442755278091A0049091A104A091A2047F
:10C88000B091A304BC01CD010E94C8A0DC01CB0182
:10C89000BC01CD0120EF35E540E050E00E943CA115
:10C8A000B501620F731F70937D0A60937C0A8091BB
:10C8B000370A9091380A8150904134F080E090E13D
:10C8C0009093380A8093370A8091370A9091380AFA
:10C8D0008050904F34F480E090EF9093380A80932A
:10C8E000370A8091270A9091280A8150904134F0AC
:10C8F00080E090E19093280A8093270A8091270A8C
:10C900009091280A8050904F34F480E090EF9093FB
:10C91000280A8093270A6150704134F080E090E14A
:10C9200090937D0A80937C0A80917C0A90917D0A85
:10C930008050904F34F480E090EF90937D0A809384
:10C940007C0A80910101482F552780912201909106
:10C9500023014817590794F42091220130912301B3
:10C9600069817A81649FC001659F900D749F900DCD
:10C970001124B9010E94F3A07A83698389819A8185
:10C98000880F991F880F991F9A8389838091730A52
:10C9900080FD02C00C940F6F112311F00C940F6FE7
:10C9A000002311F00C940F6F8091D10599278F7798
:10C9B0009070009711F00C940F6F4C018091D4048B
:10C9C0009091D504892BD9F5809118019091190186
:10C9D0008959934058F087B5803F20F480914B03EC
:10C9E000815011C081E08093350555C080911801B8
:10C9F0009091190184369105E8F487B58031B0F043
:10CA000080914B038F5F80934B039FE089029001DD
:10CA1000112480910808821B87BD8CE291E09093DD
:10CA20003803809337038EE591E031C081E0809335
:10CA3000340531C000933405009335052CC0909225
:10CA40004A038092490380911D04882321F081E0EC
:10CA50000E943B9B17C080915C0490915D04A09163
:10CA60005E04B0915F0454E0880F991FAA1FBB1F9A
:10CA70005A95D1F780934C0390934D03A0934E03A6
:10CA8000B0934F038091D4049091D5040197909373
:10CA9000D5048093D4048091730A20913F0481FFD0
:10CAA00040C0223320F080913E048D3848F18091BF
:10CAB000B20181508093B2018F3F09F059C080913B
:10CAC000C901882339F480917904882319F088E218
:10CAD0008093C9011092790480915C0490915D0467
:10CAE000A0915E04B0915F04809358049093590420
:10CAF000A0935A04B0935B0481E08093B20138C0E4
:10CB00002734B0F18091C901882339F480917904E8
:10CB1000882319F487E28093C90188EC8093B201DD
:10CB200024C08091420190914301820F911D209178
:10CB30006E083327829FF001839FF00D929FF00DC6
:10CB40001124CF01AA2797FDA095BA2F80935804EE
:10CB500090935904A0935A04B0935B0480913E04CF
:10CB60008D3818F01092790403C081E08093790425
:10CB70008091BC049091BD04A091BE04B091BF040B
:10CB8000E0903E01F0903F01009140011091410181
:10CB9000BC01CD01A80197010E943CA159016A0185
:10CBA0008091B4049091B504A091B604B091B704FB
:10CBB000BC01CD01A80197010E943CA1B901C501AA
:10CBC0000E944C929093420A8093410ACC9734F091
:10CBD0008CE390E09093420A8093410A8091410A4D
:10CBE0009091420A0E940C7C9093420A8093410AE1
:10CBF00080E280933D011092570410925604809178
:10CC00007904882309F46FC78091250499279C0132
:10CC10002071307084FD67C7809124048260809306
:10CC200024047091540A872F992741E0C42ED12CF7
:10CC3000C822D92280FD04C08091730A81FD10C0F2
:10CC4000E980FA8030932B0520932A05309357040E
:10CC50002093560480912504806C80932504DFC2C4
:10CC60008091250481FFAEC200919F011091A00127
:10CC7000C8010F96A0906C04B0906D048A159B05B6
:10CC80000CF06EC080913405882309F069C0809152
:10CC90002C0590912D05459784F080914303909148
:10CCA0004403A0914503B0914603809358049093A8
:10CCB0005904A0935A04B0935B048091250487FF24
:10CCC00015C0809125048F778093250480914303BC
:10CCD00090914403A0914503B0914603809358047A
:10CCE00090935904A0935A04B0935B048091250457
:10CCF000806480932504E090330AEE20F1F0809167
:10CD0000580490915904A0915A04B0915B04BC015D
:10CD1000CD0124E630E040E050E00E943CA18E2DA1
:10CD20009927AA27BB2782179307A407B5072CF4D6
:10CD3000D0925704C092560410C0C501801B910BBD
:10CD40000F9797FF03C0909581959F4F909357043D
:10CD5000809356048BE280933D011092500434C1BD
:10CD6000C8010F97A816B906C4F5209135052223EE
:10CD7000A1F58091250486FF15C0809125048F7B45
:10CD8000809325048091430390914403A09145032F
:10CD9000B09146038093580490935904A0935A0489
:10CDA000B0935B0480912504806880932504C501BD
:10CDB000801B910B0F9697FF03C0909581959F4F15
:10CDC000909581959F4F90935704809356048DE2E0
:10CDD00080933D0120935004F7C08DE380933D0183
:10CDE00060915104662371F12091520430915304F3
:10CDF00040915404509155048091580490915904E5
:10CE0000A0915A04B0915B0482179307A407B50759
:10CE1000CCF480912504806480932504862F992783
:10CE200090935704809356048AE0809350048EE5D3
:10CE300080933D018091250487FFC6C08091250421
:10CE40008F7733C0662309F443C020915204309198
:10CE5000530440915404509155048091580490918A
:10CE60005904A0915A04B0915B04281739074A0766
:10CE70005B0774F580912504806880932504862FD4
:10CE80009927909581959F4F9093570480935604CE
:10CE900086EF8093500486E780933D0180912504BE
:10CEA00086FF92C0809125048F7B8093250480911A
:10CEB000430390914403A0914503B09146038093AE
:10CEC000580490935904A0935A04B0935B047CC017
:10CED00080912504807C09F477C0809150048823D8
:10CEE00009F04CC08091430390914403A091450305
:10CEF000B0914603885C9040A040B0402091580417
:10CF00003091590440915A0450915B048217930761
:10CF1000A407B5076CF08091430390914403A0915E
:10CF20004503B0914603885C9040A040B0401DC0CE
:10CF30008091430390914403A0914503B09146032F
:10CF400088539F4FAF4FBF4F281739074A075B07DA
:10CF5000BCF08091430390914403A0914503B091AC
:10CF6000460388539F4FAF4FBF4F80935804909311
:10CF70005904A0935A04B0935B0402C01092500469
:10CF8000809125048F738093250410922B051092B5
:10CF90002A0571FF06C084EF91E0909338038093D7
:10CFA000370380916004882379F480915C04909128
:10CFB0005D04A0915E04B0915F04C397A105B10523
:10CFC0001CF081E08093600460912A0570912B052C
:10CFD0008091560490915704680F791F70932B0528
:10CFE00060932A05CB0177FF04C088279927861B09
:10CFF000970B855F91400CF4CEC0409150044423C0
:10D0000089F18091520490915304209158043091F9
:10D010005904821B930B0996439748F4809152045C
:10D0200090915304A0915404B091550412C0242F40
:10D03000332727FD3095432F532F8091580490912B
:10D040005904A0915A04B0915B04820F931FA41F4E
:10D05000B51F8093580490935904A0935A04B09339
:10D060005B0424C0209158043091590440915A0423
:10D0700050915B0480916E081616170644F463E025
:10D080000E94E7A0280F311D411D511D07C063E01C
:10D090000E94E7A0281B3109410951092093580437
:10D0A0003093590440935A0450935B0410922B051B
:10D0B00010922A05E0905C04F0905D0400915E04FB
:10D0C00010915F04D801C70180509440A040B04047
:10D0D000209158043091590440915A0450915B04B6
:10D0E00082179307A407B5075CF4D801C7018050E5
:10D0F0009C4FAF4FBF4F281739074A075B0744F0D3
:10D100008093580490935904A0935A04B0935B04FD
:10D110008091540A81FF06C084E690E09093380322
:10D1200080933703809172088823A9F58091510478
:10D13000882389F5409146045091470457FF02C067
:10D140004D5F5F4F559547955595479580912201C5
:10D1500090912301209101013327489FB001499FFD
:10D16000700D589F700D1124CB01B9010E9407A1C9
:10D170007093A00160939F01663471051CF486E4EE
:10D1800090E005C06739710534F086E990E090932E
:10D19000A00180939F018091D4049091D504892BA4
:10D1A000D1F18091430390914403A0914503B09144
:10D1B00046038093580490935904A0935A04B09363
:10D1C0005B0429C080915C0490915D04A0915E0491
:10D1D000B0915F0480599140A040B04080935804C2
:10D1E00090935904A0935A04B0935B048091720801
:10D1F000882311F0992702C088E790E09093A0015E
:10D2000080939F0189819A8190934704809346047B
:10D210008EE280933D01E0904604F09047048091B7
:10D22000430390914403A0914503B091460320919C
:10D2300058043091590440915A0450915B042817C6
:10D2400039074A075B0724F08091540A80FD97C490
:10D2500080911D046091D4047091D504882309F055
:10D260007EC2672B49F0E0904604F090470410928C
:10D270002D0510922C05E1C0809143039091440349
:10D28000A0914503B0914603821B930BA40BB50BF1
:10D290008093FA049093FB04A093FC04B093FD04E4
:10D2A0008230E0E89E07EFEFAE07EFEFBE072CF409
:10D2B00081E090E8AFEFBFEF09C08F5F9F47A040CC
:10D2C000B04064F08FEF9FE7A0E0B0E08093FA04F5
:10D2D0009093FB04A093FC04B093FD048091FA04A6
:10D2E0009091FB0490932D0580932C0580919601DD
:10D2F000282F3327442755278091FA049091FB0467
:10D30000A091FC04B091FD04BC01CD010E94C8A015
:10D3100097FF04C0615E7F4F8F4F9F4F25E095952B
:10D320008795779567952A95D1F76093FA0470935E
:10D33000FB048093FC049093FD0465302EEF72078C
:10D340002FEF82072FEF92072CF484E09EEFAFEFD0
:10D35000BFEF09C0605074408040904064F080E0AE
:10D3600094E0A0E0B0E08093FA049093FB04A093D3
:10D37000FC04B093FD048090FA049090FB0420918B
:10D38000490330914A0337FF02C0295F3F4F03E052
:10D39000359527950A95E1F74FEF223834071CF4AD
:10D3A00021E83FEF05C02038310514F020E830E0D7
:10D3B000C901AA2797FDA095BA2F2091970133277D
:10D3C00044275527BC01CD010E94C8A097FF04C087
:10D3D0006D5F7F4F8F4F9F4F12E0959587957795A3
:10D3E00067951A95D1F79B015FEF613075071CF4C3
:10D3F00020E03FEF06C06F3F710519F014F020E008
:10D4000031E080912504807C49F0C90137FD039605
:10D410009C0135952795359527950DC08091540A27
:10D4200080FF09C0C90137FD07969C01A3E035952F
:10D430002795AA95E1F7820E931E2091950122234C
:10D4400009F454C060917C0470917D0480917E0445
:10D4500090917F0497FF04C061587F4F8F4F9F4F7B
:10D46000F7E09595879577956795FA95D1F73327E6
:10D47000442755270E94C8A097FF04C0615E7F4FD4
:10D480008F4F9F4FE5E09595879577956795EA953E
:10D49000D1F76093FA047093FB048093FC0490939B
:10D4A000FD046138AFEF7A07AFEF8A07AFEF9A0755
:10D4B0002CF480E89FEFAFEFBFEF0AC06F3F71051C
:10D4C0008105910569F064F080E091E0A0E0B0E0B2
:10D4D0008093FA049093FB04A093FC04B093FD04A2
:10D4E0008091FA049091FB04880E991E809193011B
:10D4F000282F33278091070B992787FD9095289F28
:10D50000F001299FF00D389FF00D11249F01F7FFC6
:10D5100002C021583F4F220F232F221F330BFFEF52
:10D5200021383F071CF420E83FEF06C02F3F3105AC
:10D5300019F014F020E031E0280D391DC901AA27A7
:10D5400097FDA095BA2F00914604109147049801C9
:10D55000442737FD4095542FBC01CD010E94C8A03F
:10D5600097FF04C061507E4F8F4F9F4F59E09595B4
:10D570008795779567955A95D1F7E61AF70A8091BE
:10D58000560490915704892B09F064C010161106B7
:10D590000CF060C020912C0530912D05C90137FF9A
:10D5A00003C0309521953F4F2D33310540F48091D4
:10D5B0007404909175048E159F0574F526C02C5344
:10D5C000304045E0369527954A95E1F72031310501
:10D5D00010F02FE030E0409174045091750418165B
:10D5E0001906E4F480E190E0821B930B489F9001C0
:10D5F000499F300D589F300D1124B4E03695279582
:10D60000BA95E1F72E153F0520F580919D01909187
:10D610009E01E816F906F4F07C011CC0205F3F4F24
:10D6200080919D0190919E01829FB001839F700D1A
:10D63000929F700D11249B01A4E036952795AA9521
:10D64000E1F74E155F0514F07A0104C0E216F30607
:10D6500008F07901C701AA2797FDA095BA2FFDE030
:10D66000880F991FAA1FBB1FFA95D1F72091410A75
:10D670003091420A442737FD4095542FBC01CD011B
:10D680000E943CA12093FE043093FF0440930005C8
:10D6900050930105E090FE04F090FF0480912E0568
:10D6A00090912F059C01220F331F280F391F2E0D3B
:10D6B0003F1D37FF02C02D5F3F4FA901559547958C
:10D6C0005595479550932F0540932E0580916A08F4
:10D6D000282F3327220F331F220F331F241735071C
:10D6E0006CF480917B0A282F3327220F331F220FDF
:10D6F000331F205530404217530724F030932F0535
:10D7000020932E058091540A80FF14C080912E052D
:10D7100090912F05A981BA818A179B0724F0B093B5
:10D720002F05A0932E05E0912E05F0912F05FA8389
:10D73000E98325C229813A81201B310B37FF02C0C2
:10D740002D5F3F4F359527953595279540912E05AF
:10D7500050912F05420F531F5A83498310C2672BE4
:10D7600049F0E0904604F090470410922D05109285
:10D770002C0538C18091430390914403A091450347
:10D78000B0914603821B930BA40BB50B8093FA0454
:10D790009093FB04A093FC04B093FD04823050E806
:10D7A00095075FEFA5075FEFB5072CF481E090E8E0
:10D7B000AFEFBFEF09C08F5F9F47A040B04064F05C
:10D7C0008FEF9FE7A0E0B0E08093FA049093FB0412
:10D7D000A093FC04B093FD048091FA049091FB04A3
:10D7E00090932D0580932C0580919601282F332747
:10D7F000442755278091FA049091FB04A091FC04E2
:10D80000B091FD04BC01CD010E94C8A097FF04C0E7
:10D81000615E7F4F8F4F9F4F05E095958795779578
:10D8200067950A95D1F76093FA047093FB0480938F
:10D83000FC049093FD046530A8EF7A07AFEF8A07E8
:10D84000AFEF9A072CF484E098EFAFEFBFEF09C079
:10D85000605078408040904064F080E098E0A0E024
:10D86000B0E08093FA049093FB04A093FC04B0937F
:10D87000FD048090FA049090FB0480919501282F7C
:10D8800033278091500390915103829FF001839F31
:10D89000F00D929FF00D11249F01F7FF02C021505F
:10D8A0003F4F232F330F330B8091490390914A034D
:10D8B000820F931FAA2797FDA095BA2F8093FA0491
:10D8C0009093FB04A093FC04B093FD04809150045A
:10D8D0002091560430915704882331F0B3E0220F91
:10D8E000331FBA95E1F71BC080916E089927289FD6
:10D8F000A001299F500D389F500D11249A01A3E0DB
:10D90000220F331FAA95E1F7240F351F37FF02C0FE
:10D91000215E3F4FF5E035952795FA95E1F7309375
:10D920001F0420931E0480911E0490911F049C01EB
:10D93000442737FD4095542F8091FA049091FB04C1
:10D94000A091FC04B091FD04821B930BA40BB50BBA
:10D950008093FA049093FB04A093FC04B093FD041D
:10D9600020919701332744275527BC01CD010E9400
:10D97000C8A097FF04C0615E7F4F8F4F9F4FE5E0C7
:10D980009595879577956795EA95D1F76093FA0411
:10D990007093FB048093FC049093FD04653058EF72
:10D9A00075075FEF85075FEF95072CF484E098EF2C
:10D9B000AFEFBFEF09C0605078408040904064F006
:10D9C00080E098E0A0E0B0E08093FA049093FB043C
:10D9D000A093FC04B093FD048091FA049091FB04A1
:10D9E000880E991EE818F9088091740490917504C6
:10D9F0008E159F053CF480919D0190919E01E81643
:10DA0000F9060CF07C01C701AA2797FDA095BA2F53
:10DA10005DE0880F991FAA1FBB1F5A95D1F720916F
:10DA2000410A3091420A442737FD4095542FBC01EA
:10DA3000CD010E943CA12093FE043093FF0440934B
:10DA4000000550930105E090FE04F090FF048091E2
:10DA50002E0590912F059C01220F331F280F391F8F
:10DA60002E0D3F1D37FF02C02D5F3F4FA901559579
:10DA700047955595479550932F0540932E058091D6
:10DA80006A08282F3327220F331F220F331F241732
:10DA900035076CF480917B0A282F3327220F331F20
:10DAA000220F331F205530404217530724F0309384
:10DAB0002F0520932E058091540A20912E05309138
:10DAC0002F0580FF0DC0E981FA812E173F0724F052
:10DAD000F0932F05E0932E0520912E0530912F0510
:10DAE0003A8329834CC080917208882301F56091A4
:10DAF00046047091470477FF02C06D5F7F4F7595B4
:10DB00006795759567954091220150912301809109
:10DB10000101282F3327649FC001659F900D749FDA
:10DB2000900D1124B9010E9407A1CB0101C09927D2
:10DB30009093A00180939F0180919F019091A001FB
:10DB4000873491051CF486E490E005C08639910580
:10DB500034F086E990E09093A00180939F01498181
:10DB60005A8150932F0540932E0580912504806C97
:10DB700080932504809124048D7F809324048091D8
:10DB8000250499279C012270307081FF39C1809152
:10DB9000300590913105A0913205B0913305009781
:10DBA000A105B10521F0809160048130B9F4809124
:10DBB000460490914704AA2797FDA095BA2F1EE02E
:10DBC000880F991FAA1FBB1F1A95D1F780933005A4
:10DBD00090933105A0933205B09333058091600492
:10DBE000813019F482E08093600469817A817B013D
:10DBF0000027F7FC0095102F8091410A9091420A6E
:10DC00009C01442737FD4095542FC801B7010E945D
:10DC1000C8A0DC01CB018093FE049093FF04A09385
:10DC20000005B0930105B7FF04C08150904EAF4F7F
:10DC3000BF4F7C018D01FDE015950795F794E794A2
:10DC4000FA95D1F7E092FE04F092FF0400930005EC
:10DC50001093010560912604709127048FE0603ACB
:10DC6000780750F58091300590913105A0913205EB
:10DC7000B09133059C01AD01EAE056954795379583
:10DC80002795EA95D1F7821B930BA40BB50BA8013E
:10DC90009701F4E0220F331F441F551FFA95D1F767
:10DCA000820F931FA41FB51F8093300590933105F9
:10DCB000A0933205B093330560547F4118F58091ED
:10DCC000300590913105A0913205B09133059C014A
:10DCD000AD01ECE05695479537952795EA95D1F734
:10DCE000821B930BA40BB50BA801970172E0220FC6
:10DCF000331F441F551F7A95D1F7820F931FA41F1E
:10DD0000B51F41C08091490390914A038091490316
:10DD100090914A0397FF03C0909581959F4F843659
:10DD20009105CCF58091430390914403A091450364
:10DD3000B09146039C018091580490915904281B8E
:10DD4000390B37FF03C0309521953F4F2F3F3105E9
:10DD500009F00CF58091300590913105A0913205C4
:10DD6000B09133059C01AD016EE05695479537950E
:10DD700027956A95D1F7821B930BA40BB50B8E0DDB
:10DD80009F1DA01FB11F8093300590933105A09374
:10DD90003205B09333058091300590913105A09103
:10DDA0003205B09133050EE0B695A7959795879506
:10DDB0000A95D1F7909347048093460440917008E8
:10DDC000442399F055279C01BA010E9407A1C9017B
:10DDD000861B970B9093750480937404260F371F4E
:10DDE00030939E0120939D011FC0109275041092E4
:10DDF00074048FEF93E090939E0180939D0114C073
:10DE00001092600410923005109231051092320584
:10DE100010923305309347042093460405C0809147
:10DE20002504806C809325048091440581FF37C0D0
:10DE300089819A8197FD0396959587959595879504
:10DE400020912204309123042817390760F480912F
:10DE5000460490914704892B31F0220F331F220F83
:10DE6000331F3A8329838091430390914403A09107
:10DE70004503B09146038093580490935904A093AE
:10DE80005A04B0935B0488E99AE390933803809333
:10DE9000370380E09EE090930B0180930A0120916C
:10DEA0003C0A822F9927880F991F880F991F8896FF
:10DEB000A981BA818A179B0714F09A838983B0914C
:10DEC0007B0AB98B8B2F9927880F991F880F991F71
:10DED00080559040E981FA818E179F0714F49A8348
:10DEE000898380918103882341F480910E0B8F3FB9
:10DEF00021F4809148058823E1F0809126049091D7
:10DF000027040297C097A8F449815A811416150670
:10DF100084F481E090E09093270480932604622F9C
:10DF20007727660F771F660F771F685D7F4F7A83AD
:10DF3000698389819A819093C6078093C5078091F0
:10DF4000F6049091F704A091F804B091F90462E00E
:10DF5000880F991FAA1FBB1F6A95D1F700917C0AF1
:10DF600010917D0A081B190BA981BA81A13AB1054C
:10DF70008CF0CD01B7FD0196959587958017910797
:10DF80000CF48C01909581959F4F081719076CF43C
:10DF90008C010BC00135110514F000E510E0BFEF56
:10DFA000003B1B0714F400EB1FEFE9892E2F3327EA
:10DFB000220F331F220F331FC90149815A81841B4D
:10DFC000950B801791070CF48C0169817A81621B93
:10DFD000730B061717070CF48B012091370A309149
:10DFE000380AE0917204F09173042E1B3F0B3093BA
:10DFF000470A2093460A4091270A5091280A209008
:10E00000700430907104421953095093260A4093CA
:10E01000250A80917F08893008F5682F7727629F4D
:10E02000C001639F900D729F900D112497FD07967C
:10E030004C0193E0959487949A95E1F7649FC00111
:10E04000659F900D749F900D112497FD07967C019C
:10E0500083E0F594E7948A95E1F71FC08695682FD1
:10E060007727629FC001639F900D729F900D1124CE
:10E0700097FD03964C019594879495948794649F9B
:10E08000C001659F900D749F900D112497FD03961C
:10E090007C01F594E794F594E7948091560A8823DF
:10E0A00009F4C4C06E1A7F0A9301442737FD4095D6
:10E0B000542F8091840490918504A0918604B0919E
:10E0C0008704820F931FA41FB51F8093840490932D
:10E0D0008504A0938604B093870481509D47A04097
:10E0E000B04064F080E09DE7A0E0B0E0809384045D
:10E0F00090938504A0938604B09387048091840450
:10E1000090918504A0918604B09187048050934833
:10E11000AF4FBF4F64F480E093E8AFEFBFEF809361
:10E12000840490938504A0938604B093870480911F
:10E130009A0190919B015C01CC24B7FCC094DC2C2B
:10E140008091840490918504A0918604B091870405
:10E15000BC01CD01A60195010E943CA1820E931E37
:10E160001092EE041092EF041092F0041092F10459
:10E17000421853089201442737FD4095542F80914F
:10E18000800490918104A0918204B0918304820F55
:10E19000931FA41FB51F8093800490938104A093C4
:10E1A0008204B093830481509D47A040B04064F046
:10E1B00080E09DE7A0E0B0E080938004909381042C
:10E1C000A0938204B0938304809180049091810491
:10E1D000A0918204B091830480509348AF4FBF4F09
:10E1E00064F480E093E8AFEFBFEF809380049093F6
:10E1F0008104A0938204B093830480918004909161
:10E200008104A0918204B0918304BC01CD01A601D8
:10E2100095010E943CA1E20EF31E1092F2041092AE
:10E22000F3041092F4041092F504C7C08091460ADA
:10E230009091470A9C01442737FD4095542F8091C7
:10E24000EE049091EF04A091F004B091F104820FDC
:10E25000931FA41FB51F8093EE049093EF04A09327
:10E26000F004B093F10481509D47A040B04064F0A9
:10E2700080E09DE7A0E0B0E08093EE049093EF048F
:10E28000A093F004B093F1048091EE049091EF0418
:10E29000A091F004B091F10480509348AF4FBF4F6C
:10E2A00064F480E093E8AFEFBFEF8093EE049093C7
:10E2B000EF04A093F004B093F10480919801909141
:10E2C00099015C01CC24B7FCC094DC2C8091EE0455
:10E2D0009091EF04A091F004B091F104BC01CD0144
:10E2E000A60195010E943CA1820E931E1092840407
:10E2F0001092850410928604109287048091250A5A
:10E300009091260A9C01442737FD4095542F809117
:10E31000F2049091F304A091F404B091F504820FFB
:10E32000931FA41FB51F8093F2049093F304A0934E
:10E33000F404B093F50481509D47A040B04064F0D0
:10E3400080E09DE7A0E0B0E08093F2049093F304B6
:10E35000A093F404B093F5048091F2049091F30437
:10E36000A091F404B091F50480509348AF4FBF4F93
:10E3700064F480E093E8AFEFBFEF8093F2049093F2
:10E38000F304A093F404B093F5048091F204909107
:10E39000F304A091F404B091F504BC01CD01A601F1
:10E3A00095010E943CA1E20EF31E1092800410928F
:10E3B0008104109282041092830480918201682F5C
:10E3C000772788279927980117FF04C0222733272A
:10E3D000201B310B37FF02C02F5F3F4F359527952C
:10E3E000A981BA812A0F3B1F442737FD4095542F3E
:10E3F0000E94C8A097FF04C0615C7F4F8F4F9F4F62
:10E40000E6E09595879577956795EA95D1F79B0115
:10E41000681579050CF44B0144275527421B530B13
:10E42000841695060CF44A012E153F050CF47B0169
:10E43000E416F5060CF47A0180913C0A282E332468
:10E440005090C10861E3A62E69E0B62E58EEC52EA5
:10E4500058E0D52E4BE0442E38E5632E3AE0732E7B
:10E46000F601208112160CF029C1203429F42981EB
:10E470003A813F8B2E8B1FC049815A81CA01AA273E
:10E4800097FDA095BA2F332727FD3095432F532FA3
:10E49000BC01CD010E94C8A097FF04C0615C7F4F02
:10E4A0008F4F9F4F26E095958795779567952A958D
:10E4B000D1F77F8B6E8BF6012181203439F42E89C0
:10E4C0003F89280D391D3F8B2E8B2AC0203C39F403
:10E4D0004E895F89481959095F8B4E8B21C0C40151
:10E4E000AA2797FDA095BA2F332727FD3095432FF4
:10E4F000532FBC01CD010E94C8A097FF04C0615CEE
:10E500007F4F8F4F9F4FB6E095958795779567958D
:10E51000BA95D1F7AE89BF89A60FB71FBF8BAE8B57
:10E52000F6012281203439F42E893F892E0D3F1DBA
:10E530003F8B2E8B2AC0203C39F44E895F894E19BF
:10E540005F095F8B4E8B21C0C701AA2797FDA0955D
:10E55000BA2F332727FD3095432F532FBC01CD0110
:10E560000E94C8A097FF04C0615C7F4F8F4F9F4FF0
:10E57000A6E09595879577956795AA95D1F7AE8989
:10E58000BF89A60FB71FBF8BAE8BF6012381203446
:10E5900039F42E893F89200F311F3F8B2E8B2AC0E3
:10E5A000203C39F44E895F89401B510B5F8B4E8BA9
:10E5B00021C0C801AA2797FDA095BA2F332727FDB0
:10E5C0003095432F532FBC01CD010E94C8A097FF67
:10E5D00004C0615C7F4F8F4F9F4FF6E09595879504
:10E5E00077956795FA95D1F7AE89BF89A60FB71FC2
:10E5F000BF8BAE8BF301808191812E893F89821779
:10E60000930764F4B901680F791F77FF02C06F5F49
:10E610007F4F759567957F8B6E8B1DC0552049F494
:10E620004E895F89440F551F481B590B5F8B4E8BDA
:10E6300012C051E0551578F4252D33276E897F8956
:10E64000861B970BB9010E9407A1AE89BF89A60F4F
:10E65000B71FBF8BAE8BC101880F991F880F991F01
:10E66000EE89FF898E179F0764F4F9898F2F992708
:10E67000880F991F880F991F2E893F8928173907FE
:10E6800014F09F8B8E8B8E899F8997FD03969595AD
:10E69000879595958795F5018183880F991F880F38
:10E6A000991F2E893F89281B390BC901880F828346
:10E6B000EE89FF89D301ED93FC9303C0F50111822C
:10E6C00012824A9422E030E0620E731E44E050E071
:10E6D000C40ED51E68E070E0A60EB71E47FEC0CE81
:10E6E000E2E1C95E0C9473A184B1806A84B93D9A59
:10E6F00082E58CBD1DBC459A81E080938D0A8AEA33
:10E7000080939E0A83E880939F0A8AE08093A00A00
:10E710001092A20A1092A10A1092A40A1092A30ABF
:10E720001092060B1092C20A089530918D0A33237D
:10E7300009F070C00DB407FE6DC083E0809336030E
:10E74000459A2EB580914B0599278130910589F026
:10E75000823091051CF4892B21F03EC00297B9F05C
:10E760003BC03093C10A20934C052138A9F581E0C4
:10E7700008C0253549F480914C05820F80934C05E3
:10E7800082E080934B0528C030934B0525C08091D3
:10E79000C10AE82FFF27ED51F54F20838F5F80934B
:10E7A000C10A90914C058032A0F0291769F480E2EB
:10E7B000A3EEBAE0E3ECFAE00D9001928A95E1F75E
:10E7C00081E08093C20A02C03093C20A10924B05C6
:10E7D00003C0920F90934C0520919D0A2232A0F421
:10E7E00045980000000000000000E091960AF091BA
:10E7F000970AE20FF11D80818EBD8091BF0A908142
:10E80000890F8093BF0A03C081E080938D0A2F5F38
:10E8100020939D0A0895EF92FF920F931F9380918A
:10E8200078089927880F991F880F991F7C01002766
:10E83000F7FC0095102F8091BC049091BD04A0912D
:10E84000BE04B091BF04BC01CD01A80197010E9494
:10E850003CA13093A20A2093A10A8091B404909124
:10E86000B504A091B604B091B704BC01CD01A801D4
:10E8700097010E943CA13093A40A2093A30A2091FF
:10E88000830A3091840A4091850A5091860ADA0100
:10E89000C90173E0880F991FAA1FBB1F7A95D1F792
:10E8A000820F931FA41FB51F820F931FA41FB51FB4
:10E8B00020913E0130913F01409140015091410132
:10E8C000BC01CD010E943CA13093AA0A2093A90A61
:10E8D0008091CE049091CF0420915603309157033C
:10E8E000821B930B9093B00A8093AF0AE091C4040B
:10E8F000F091C50480914D0A90914E0ABF010E948B
:10E9000007A1CB019B01220F331F220F331F280FBA
:10E91000391F280F391F37FF02C02D5F3F4F359534
:10E920002795359527953093A60A2093A50A8091BF
:10E930007F0A9091800ABF010E9407A19B01220FCC
:10E94000331F220F331F260F371F260F371F37FFA6
:10E9500002C02D5F3F4F359527953595279530930C
:10E96000A80A2093A70A1092C5041092C40410921A
:10E970004E0A10924D0A1092800A10927F0A8091DE
:10E98000A00A9927AA27BB27FC013A97E830F1058E
:10E9900008F028C2E058FF4F0C948EA180913E04ED
:10E9A0008093B30A80913D048093B40A80913C0423
:10E9B0008093B50A80913B048093B60A80913A0413
:10E9C0008093B70A809139048093B80A8091380403
:10E9D0008093B90A809137048093BA0A8091250404
:10E9E0008093BB0A80912504837F809325048091C6
:10E9F00000018093BC0A8091C2088093BD0A809177
:10EA000024048093BE0A4299EDC180912404877F3B
:10EA100080932404E7C18091080B9091090B909397
:10EA2000B40A8093B30A80910C0B90910D0B9093D4
:10EA3000B60A8093B50A80912201909123018093B8
:10EA4000B70A8091340A8093B80A80913D0180937F
:10EA5000B90A90914D059093BA0AE92FFF2713E068
:10EA6000EE0FFF1F1A95E1F7EF5CF64F868180935A
:10EA7000BB0A83818093BC0A87818093BD0A85810C
:10EA80008093BE0A9F5F90934D05E92FFF27EE0FFD
:10EA9000FF1FEE0FFF1FE552F74F8585882309F012
:10EAA000A1C1992309F49EC1892F992701966CE091
:10EAB00070E00E9407A19C01982FE82FFF27EE0F1E
:10EAC000FF1FEE0FFF1FE552F74F8585882311F4D6
:10EAD000222351F720934D0585C180910101809338
:10EAE000B30A8091AE088093B40A8091AF088093F6
:10EAF000B50A8091B0088093B60A8091B1088093DE
:10EB0000B70A8091B5088093B80A8091B6088093BF
:10EB1000B90A8091B7088093BA0A8091BA088093A5
:10EB2000BB0A8091B8088093BC0A8091B908809391
:10EB3000BD0A8091BB0854C18091AC088093B30A90
:10EB400080918308863081F080910003823451F0F7
:10EB50000E945481E82FFF27E95EFD4E8491809347
:10EB6000000302C00E945481809173058093B40A0F
:10EB70008091C9088093B50A35C1F89480915F08E7
:10EB8000E82FFF27EE0FFF1FEE56F64F0190F081A2
:10EB9000E02DE038F1051CF0EFE7F0E006C02FEFC4
:10EBA000E138F20714F4E1E8FFEFE093B30A809153
:10EBB0006008E82FFF27EE0FFF1FEE56F64F01907B
:10EBC000F081E02DE038F1051CF0EFE7F0E006C041
:10EBD0007FEFE138F70714F4E1E8FFEFE093B40AC0
:10EBE00080915E08E82FFF27EE0FFF1FEE56F64FCD
:10EBF0000190F081E02DE038F1051CF0EFE7F0E046
:10EC000006C08FEFE138F80714F4E1E8FFEFE09376
:10EC1000B50A80915D08E82FFF27EE0FFF1FEE5623
:10EC2000F64F0190F081E02DE038F1051CF0EFE7A0
:10EC3000F0E006C02FEFE138F20714F4E1E8FFEF4F
:10EC40007894E093B60A809163048093B70A809128
:10EC500064048093B80A809165048093B90A809116
:10EC600066048093BA0A809167048093BB0A8091FE
:10EC700068048093BC0A809169048093BD0A8091E6
:10EC80006A04AEC08091EC05863018F01092EC0555
:10EC900085E08093B30A8091BC088093B40A809188
:10ECA0005C0490915D04A0915E04B0915F04BC018E
:10ECB000CD0125E030E040E050E00E943CA13093DF
:10ECC000B60A2093B50A8091580490915904A091F6
:10ECD0005A04B0915B04BC01CD0125E030E040E076
:10ECE00050E00E943CA13093B80A2093B70A80916B
:10ECF000B2088093B90A8091B3088093BA0A8091D0
:10ED0000B4088093BB0A809162048093BC0A10927D
:10ED1000BD0A8091C5079091C60797FD039695950A
:10ED20008795959587955CC01092B30A8BE5809383
:10ED3000B40A8BE08093B50A87E38093B60A80918A
:10ED400002018093B70A8091D1058093B80A90910F
:10ED5000D2059093B90A8F778093D10590719093E3
:10ED6000D2051092BA0A8091730A8093BB0A8091EF
:10ED7000540A8093BC0A8091BE088093BD0A80919A
:10ED8000CD082EC0809191088093B30A8091CB0862
:10ED90008093B40A80918A018093B50A80918A0891
:10EDA0008093B60A80918B088093B70A80918C0873
:10EDB0008093B80A809189018093B90A80918E0866
:10EDC0008093BA0A80918F088093BB0A8091900843
:10EDD0008093BC0A80910E0B8093BD0A8091EF074F
:10EDE0008093BE0A8091C20A882309F47DC1609194
:10EDF000C30A8091C301681719F08AEF8093C1019B
:10EE00006093C30181E08093AC014091C40A5091AA
:10EE1000C50ACA0181509E4F8F5F9340B0F4209184
:10EE2000C60A3091C70AC90181509E4F8F5F934037
:10EE300060F48091690885FF08C050933A054093BB
:10EE4000390530933805209337058091CA0A90918F
:10EE5000CB0A21E08936920724F49093AE01809387
:10EE6000AD012091D40A3091D50A80913703909159
:10EE700038038217930740F480910803882321F414
:10EE80003093380320933703862F992789369105CD
:10EE900009F4A5C08A36910544F48736910571F0CE
:10EEA0008836910509F462C027C18A36910509F4B4
:10EEB00014C18B36910509F4E2C01EC18091D60AB7
:10EEC0008093030B8091D70A8093050B8091D80A19
:10EED0008093040B8091D90A8093AB018091DA0A68
:10EEE0008093070B8091DB0A8093C2018091DC0A3A
:10EEF00080934A058091DD0A80933605809136041F
:10EF00008823F9F02091DE0A3091DF0A37FD19C01D
:10EF100030937B0420937A0490919308992389F08D
:10EF20008FE0989FC0011124281B390BC901885913
:10EF30009E4F68E671E00E9407A190937B04809346
:10EF40007A0420914105309142058091E00A909128
:10EF5000E10A280F391F37FF02C02F5F3F4F359559
:10EF600027953093420520934105C6C08091D60A6B
:10EF70008093980A8091D70A8093990A8091D80A41
:10EF800080939A0A8091D90A80939B0A8091DA0A29
:10EF900080939C0A8091B5079091DB0A892B80931E
:10EFA000B5079091B60793708091DC0A8C70982B0E
:10EFB0009093B6078091DD0A809348058091DE0A20
:10EFC0008093B3018091DF0A8093060B8091E00A61
:10EFD000809344058091E10A809343058DC0809120
:10EFE000D60A80938E0A8091D70A80938F0A8091E7
:10EFF000D80A8093900A8091D90A8093910A8091CF
:10F00000DA0A9091DB0A9093930A8093920A809196
:10F01000DC0A9091DD0A9093950A8093940A80917E
:10F02000DE0A992787FD90959093CD098093CC09AE
:10F030008091DF0A809351048091E00A9091E10A67
:10F040009C01442737FD4095542FDA01C90163E044
:10F05000880F991FAA1FBB1F6A95D1F7820F931FB4
:10F06000A41FB51F820F931FA41FB51F80935204C6
:10F0700090935304A0935404B09355043DC08091E1
:10F08000D60A809347058091D70A809346058091E0
:10F09000D80A809345059091D90A992349F0809127
:10F0A000C901882319F08151833010F49093C9016C
:10F0B0008091DA0A809378058091DB0A8093770546
:10F0C0008091DC0A9091DD0A909375058093740518
:10F0D0008091DE0A809376050FC080918308863088
:10F0E00059F40E94AD8108C010923A05109239057A
:10F0F00010923805109237051F910F91FF90EF90F5
:10F10000089580918D0A882319F145988EE99AE037
:10F110009093970A8093960A90914905E92FFF27CB
:10F12000EC54FE4F9F5F9093490580818093A00A25
:10F130009D3010F01092490510928D0A0E940B74B8
:10F1400081E080939D0A80919E0A8093BF0A8EBDC4
:10F15000089587B18C6087B94298439810924F0503
:10F1600080E88093C50110924E058093C4010895F4
:10F170008091CC099091CD0981589F4F39F08091B1
:10F18000CC099091CD0981588093590580915405FF
:10F190008150809354058F3F09F043C189E08093EB
:10F1A000540580912504992780739070892B21F450
:10F1B0008091D20580FF1DC08091AA08882351F05C
:10F1C00080915705882319F484E080934F0581E0EE
:10F1D000809357058091AB088823B9F0809158053A
:10F1E000882319F484E080934E0581E080935805CC
:10F1F0000CC010925705109258058091A608809374
:10F2000055058091A808809356058091570588235D
:10F2100009F073C08091CA08282F332724FF07C044
:10F2200080916104882319F425FD80C081C09091EC
:10F23000A708983F48F080914F0A8D3D28F08091B3
:10F24000550588236CF00AC0983F68F080914F0AFA
:10F25000853049F48091550587FF02C0429801C06E
:10F26000429A81E032C080914F05815080934F05D2
:10F270008F3F09F05EC08091CD0885FF29C0909135
:10F280005905892F869580934F05992351F48091D4
:10F29000550587FF02C0429801C0429A1092C501ED
:10F2A00048C08091C50190915505882341F4809311
:10F2B000590580E88093C5019923D4F137C098237C
:10F2C00011F0429A01C0429886958093C50131C0E1
:10F2D00080914F0A869580934F058091C5018130BA
:10F2E00021F41092590580E801C086958093C501EC
:10F2F0008091C5019091550517C080914F058150AF
:10F3000080934F058F3FA9F489E080934F0580914A
:10F31000C501813011F480E801C086958093C50154
:10F320008091C5019091AA08892311F0429A01C0E9
:10F33000429880915805882309F043C09091CA08EB
:10F3400097FF07C080916104882319F496FD52C08D
:10F3500053C09091A908983F48F080917A0A8D3D5A
:10F3600028F08091560588236CF00AC0983F78F009
:10F3700080917A0A853059F48091560587FF02C042
:10F38000439801C0439A81E08093C40136C08091C4
:10F390004E05815080934E058F3F79F580917A0A12
:10F3A000869580934E058091C401813011F480E8E8
:10F3B00001C086958093C4018091C4019091560547
:10F3C00017C080914E05815080934E058F3FA9F460
:10F3D00089E080934E058091C401813011F480E86A
:10F3E00001C086958093C4018091C4019091AB08BF
:10F3F000892311F0439A01C04398429B05C0809134
:10F400002404886080932404439B06C080912404D4
:10F410008061809324040895809124048F7E8093DA
:10F42000240408954FB724E130E0F8948091C90096
:10F430008F778093C9008091C9008F7B8093C9002A
:10F440008091C9008F7D8093C900832F9927809375
:10F45000CD002093CC008091C80082608093C800CA
:10F4600080E18093C9008091CA008F778093CA00A1
:10F470008091CA008F7B8093CA008091CA008F7DE3
:10F480008093CA008091CA008F7E8093CA008091C9
:10F49000CA00877F8093CA008091C9008B7F8093C8
:10F4A000C9008091CA0084608093CA008091CA001C
:10F4B00082608093CA008091C80087FF03C080915A
:10F4C000CE00F9CF8091C90080688093C9004FBFFA
:10F4D0000895EF92FF920F931F93CF93DF93482FDE
:10F4E00000E010E08091C601813061F41092C60105
:10F4F00084E480935A0510925C0510925B0510928B
:10F500005D0539C180915A05882319F421E030E066
:10F5100001C0980190915B05992371F4232B11F0A0
:10F5200081E010C084E480935A0590935C05909329
:10F530005B0590935D0508C1913069F4232B09F0B8
:10F54000F9C082E080935B0580915C058F5F8093BA
:10F550005C0583E0F7C09230D1F4232B09F0EAC0B8
:10F5600083E080935A0540935D0590915C0592304D
:10F5700039F410925E0547FF03C081E080935E0579
:10F5800083E080935B059F5F90935C05DDC09330C3
:10F5900009F0D0C0232B09F0CDC090935A0582E02A
:10F5A00080935B0580915C058F5F80935C05209163
:10F5B0005D05822F9927782F6627842F9927682B3E
:10F5C000792B80918308813049F47370CB0180508E
:10F5D000924063E070E00E9407A117C0823061F49E
:10F5E0007770CB018050944066E070E00E9407A1E4
:10F5F0002695269526950BC0737068567140CB01F1
:10F6000077FD0196BC017595679526952695022F85
:10F6100011270F7010700F5F1F4F0D30110508F08C
:10F6200082C07801E00EF11EF701EE56F64F8081A0
:10F6300091819B01281B390BC90137FF03C09095AD
:10F6400081959F4F069704F5E091C508EE2351F090
:10F65000FF27EE0FFF1FEE56F64F80819181843613
:10F66000910594F480916204883C30F480916204A6
:10F67000865F8093620408C088EC80936204809166
:10F680006F008F7D80936F00F701EE56F64F8081FB
:10F6900091819C01220F331F280F391F260F371F1E
:10F6A00037FF02C02D5F3F4FE901D595C795D5952E
:10F6B000C795CB0101968C179D0714F4219706C0BE
:10F6C00061507040C617D7070CF4219680916204F0
:10F6D000843BD0F0F701EE56F64F80819181FE0118
:10F6E000E81BF90BCF0163E070E00E9407A1CB019A
:10F6F000880F991F860F971F28ED39E0E20EF31E41
:10F70000F7019183808307C028ED39E0E20EF31EF4
:10F71000F70111821082000F111F0E56164FF801CB
:10F72000D183C08311C00231110570F081E0809354
:10F73000C6010AC081E08093C60110925C05109258
:10F740005E0584E480935A0580915C05803198F0D1
:10F7500080915E05882331F48091C601882311F4DD
:10F7600080933C0110925C0510925E0510925B053F
:10F7700084E480935A05E6E0CDB7DEB70C947FA110
:10F78000CF93FC0197FF05C0CFEFF095E195FF4FB8
:10F7900001C0C1E028E631E0CF01B9010E9407A114
:10F7A000FC018B35910554F08B5590408A359105BD
:10F7B00038F484EB90E08E1B9F0BFC0141E00DC000
:10F7C000CF01855B90408A35910518F4E45BF040E9
:10F7D00003C02E1B3F0BF9014FEFEE0FFF1FEC593B
:10F7E000F64F259134918C2F992787FD9095289F6E
:10F7F000B001299F700D389F700D1124842F992717
:10F8000087FD9095689FA001699F500D789F500DCE
:10F810001124CA01CF9108952AE530E0281B390B45
:10F82000C9010E94C07B0895CF93DF9380E00E94BE
:10F83000289480912201909123016AE070E00E9457
:10F8400007A19F938F9380912201909123016AE0F9
:10F8500070E00E9407A17F936F9384E49AE09F93E6
:10F860008F93CBE1D4E9DF93CF93E091B805F0918A
:10F87000B90509952DB73EB7285F3F4F2DBF809141
:10F88000C101882361F186E00E9428948091B30130
:10F8900099279F938F938091920A9091930A6AE09F
:10F8A00070E00E94F3A07F936F938FED90E09F93A1
:10F8B0008F9380912C0A90912D0A9F938F938DE4C2
:10F8C0009AE09F938F93DF93CF93E091B805F091E7
:10F8D000B90509958DB79EB70C968DBF12C086E00D
:10F8E0000E9428948BE59AE09F938F93DF93CF93A8
:10F8F000E091B805F091B90509950F900F900F9020
:10F900000F9080914805882309F452C080915F05CB
:10F91000909160050E946A1A882391F08091C70136
:10F92000882319F01092C70103C081E08093C701BA
:10F930008CED95E00E94611A9093600580935F05BD
:10F940008091C7018823E1F080E00E9428941F92F3
:10F950001F929091480581E1989FC001112487551D
:10F96000944F9F938F93DF93CF93E091B805F091DD
:10F97000B90509952DB73EB72A5F3F4F2DBF3BC054
:10F9800086E00E9428948091480599279F938F9341
:10F9900082E69AE09F938F93DF93CF93E091B8052F
:10F9A000F091B90509958DB79EB706968DBF23C016
:10F9B000809172058823F9F00E942E9480E10E94C4
:10F9C00028948EEC98E09F938F9380910001992763
:10F9D0009F938F938EE69AE09F938F93DF93CF93BD
:10F9E000E091B805F091B90509952DB73EB7285FAC
:10F9F0003F4F2DBF5CC080E10E942894809102039C
:10FA0000909103036CE370E00E94F3A09F938F93A7
:10FA100080910203909103036CE370E00E94F3A0D5
:10FA20007F936F9380910C0B90910D0B9F938F930D
:10FA300089E79AE09F938F93CBE1D4E9DF93CF934B
:10FA4000E091B805F091B90509958091730A2DB739
:10FA50003EB7265F3F4F2DBF80FF29C08AE10E943D
:10FA6000289480913D0199279F938F9380915C0406
:10FA700090915D04A0915E04B0915F04BC01CD0142
:10FA800024E630E040E050E00E943CA13F932F93F9
:10FA900086E89AE09F938F93DF93CF93E091B80528
:10FAA000F091B90509958DB79EB708968DBFDF9186
:10FAB000CF910895CF93DF9380E00E9428948091A6
:10FAC0005009992787FD90959F938F9380914809BE
:10FAD000992787FD90959F938F938091400999274F
:10FAE00087FD90959F938F9380913809992787FD83
:10FAF00090959F938F938DE89AE09F938F93CBE19E
:10FB0000D4E9DF93CF93E091B805F091B905099559
:10FB100080E10E9428942DB73EB7245F3F4F2DBF50
:10FB200080917009992787FD90959F938F9380917D
:10FB30006809992787FD90959F938F93809160091D
:10FB4000992787FD90959F938F93809158099927C6
:10FB500087FD90959F938F938DE99AE09F938F9364
:10FB6000DF93CF93E091B805F091B90509958091A5
:10FB70005B082DB73EB7245F3F4F2DBF853098F40B
:10FB800080E10E9428948DEA9AE09F938F93DF93FF
:10FB9000CF93E091B805F091B90509950F900F90BA
:10FBA0000F900F9018C08730B0F488E10E9428941D
:10FBB0008FED90E09F938F938EEB9AE09F938F93BE
:10FBC000DF93CF93E091B805F091B90509958DB712
:10FBD0009EB706968DBFDF91CF9108950F931F9327
:10FBE00080E00E9428942AE030E08091080B9091F8
:10FBF000090BB9010E94F3A09F938F938091080B8A
:10FC00009091090BB9010E94F3A07F936F938091AB
:10FC1000220190912301B9010E9407A19F938F9324
:10FC20008091220190912301B9010E9407A17F9345
:10FC30006F9387EC9AE09F938F930BE114E91F93E6
:10FC40000F93E091B805F091B905099580E10E9404
:10FC500028948DB79EB70C968DBF80910C0B909118
:10FC60000D0B9F938F9380910A0B90910B0B9F9399
:10FC70008F9389ED9AE09F938F931F930F93E09159
:10FC8000B805F091B90509958DB79EB708968DBF57
:10FC90001F910F910895EF92FF920F931F9380E0B1
:10FCA0000E9428948FEDE82EF12CFF92EF92809124
:10FCB000AD019091AE019F938F9380914705992755
:10FCC0009F938F9385EE9AE09F938F930BE114E9B6
:10FCD0001F930F93E091B805F091B905099580E164
:10FCE0000E9428948DB79EB70A968DBF80914505D6
:10FCF00099279F938F93FF92EF92809146059927C2
:10FD00009F938F9388EF9AE09F938F931F930F9306
:10FD1000E091B805F091B90509958DB79EB70A969F
:10FD20008DBF1F910F91FF90EF9008950F931F9338
:10FD3000CF93DF938091C101CBE1D4E9882309F40B
:10FD40007DC080E00E94289480918F0A99279F931C
:10FD50008F938091910A99279F938F938BE09BE0DB
:10FD60009F938F938E01DF93CF93E091B805F0912D
:10FD7000B90509958DB79EB708968DBF8091900AF9
:10FD8000833031F48CE00E9428948AE19BE005C026
:10FD90008CE00E9428948FE19BE09F938F93DF93E8
:10FDA000CF93E091B805F091B90509950F900F90A8
:10FDB0000F900F9080918E0A81FF12C08CE00E94FC
:10FDC000289484E29BE09F938F931F930F93E0917D
:10FDD000B805F091B90509950F900F900F900F900D
:10FDE00080E10E9428948091B30199279F938F937B
:10FDF0008FED90E09F938F938091940A9091950A54
:10FE00009F938F938091920A9091930A6AE070E099
:10FE10000E94F3A07F936F9389E29BE09F938F935F
:10FE20008BE194E99F938F93E091B805F091B90528
:10FE300009958DB79EB70C968DBF12C082E00E94C7
:10FE400028948CE39BE09F938F93DF93CF93E09173
:10FE5000B805F091B90509950F900F900F900F908C
:10FE6000DF91CF911F910F910895CF93C82F80E01C
:10FE70000E9428948091AC099091AD0981589F4FC0
:10FE80009F938F9389E49BE09F938F938BE194E9F9
:10FE90009F938F93E091B805F091B90509958DB7BF
:10FEA0009EB706968DBFCF3231F48091AC09909108
:10FEB000AD09499607C0CF3449F48091AC099091BF
:10FEC000AD0949979093AD098093AC098091AC0935
:10FED0009091AD0982589F4F1CF481E89FEF09C0B3
:10FEE0008091AC099091AD098038910534F080E89B
:10FEF00090E09093AD098093AC09CF910895CF9392
:10FF0000C82F80E10E9428948091AE099091AF099A
:10FF100081589F4F9F938F9389E59BE09F938F9389
:10FF20008BE194E99F938F93E091B805F091B90527
:10FF300009958DB79EB706968DBFCF3231F480916B
:10FF4000AE099091AF09029607C0CF3449F4809171
:10FF5000AE099091AF0902979093AF098093AE09D3
:10FF60008091AE099091AF0982589F4F1CF481E8AF
:10FF70009FEF09C08091AE099091AF09803891053B
:10FF800034F080E890E09093AF098093AE09CF9170
:10FF90000895CF93C82F209161052093620599277A
:10FFA0008F329105E1F0803391051CF44F9779F081
:10FFB00027C08F349105D9F08F38910509F586E077
:10FFC000289FF0011124E65EF54F849117C086E06A
:10FFD000289FF0011124E55EF54F84910FC086E063
:10FFE000289FF0011124E45EF54F849107C086E05C
:10FFF000289FF0011124E35EF54F84918093610501
:020000021000EC
:1000000090916105809162059813C0E08091C801CC
:10001000282F33278F5F8093C80120FF0FC00E94D5
:100020002E949091610586E0989FF0011124E25E84
:10003000F54F259134918C2FF901099580E090E0DE
:10004000CF9108951092090B1092080B10920D0B8E
:1000500010920C0B10920B0B10920A0B10920E0BBD
:100060008AE090E00E94611A909364058093630592
:100070000895CF93DF9380916305909164050E946A
:100080006A1A882309F4AFC08091630590916405D2
:100090000A969093640580936305E0E0F0E09F0189
:1000A00090E05FEFA1E3B9E04BE0ED018B8187FFCA
:1000B0000BC09F5F8D81E80FF11D8981280F311DD5
:1000C0008E81851708F4582F4150189647FFEDCFC1
:1000D00050930E0B232B41F52091690530916A0551
:1000E00040916B0550916C05BB27A52F942F832F52
:1000F0009093680580936705AA27BB27281B390BB7
:100100004A0B5B0BCF01AA27BB27280F391F4A1FB9
:100110005B1F2093690530936A0540936B055093EC
:100120006C05E5E0F0E013C02091670530916805AB
:100130002E173F0718F4E21BF30B02C0E0E0F0E0DB
:10014000892F9927880F991FE80FF91F3596F0938B
:10015000090BE093080BEF3FF10578F48091220141
:10016000909123018E9F90018F9F300D9E9F300DA7
:100170001124C90164E670E013C0CF0196958795FC
:10018000969587952091220130912301289FA00107
:10019000299F500D389F500D1124CA0169E170E06C
:1001A0000E94F3A070930B0B60930A0B20916505DE
:1001B000309166052E0F3F1F30936605209365052D
:1001C0005EE02131350778F080910C0B90910D0B9A
:1001D000019690930D0B80930C0B20513E40309371
:1001E000660520936505DF91CF91089530917905DB
:1001F000E32FFF2783E0EE0FFF1F8A95E1F7EF5C07
:10020000F64F2781422F552747FD509580917A055B
:100210009927841795072CF420937A0530937C0551
:100220000AC0222341F080917B059927481759077E
:1002300014F420937B05832F8F5F809379058D3095
:10024000D0F01092790580917B058F3F19F0809353
:100250006E0502C010926E0580917A0580936F053D
:1002600080917C0580936D058FEF80937B051092C4
:100270007A0510927C05089595E1899F802D1124BF
:100280000E94D1998CEF9DE09F938F9383EA99E927
:100290009F938F93E091B805F091B90509950F9060
:1002A0000F900F900F900895CF93C0E02091C90157
:1002B000209373058091250485FF02C0C0E123C00F
:1002C000909148059923B1F080916104882349F405
:1002D000E92FFF27EE0FFF1FE659F44F8491882383
:1002E00049F4E92FFF27EE0FFF1FE759F44FC491A0
:1002F000CC2349F48091CD0886FD03C01092C9013A
:1003000004C0C22F02C0C093730580917D058C1775
:1003100071F480917E0590917F050E946A1A88236E
:1003200019F480E090E017C088E893E102C080ED06
:1003300097E00E94611A90937F0580937E05CC23FD
:1003400031F08091C901C81711F41092C901C0930E
:100350007D058C2F9927CF91089540E050E030E043
:100360008091E10A99278A38910589F08B389105A7
:1003700024F48938910541F013C08D38910569F056
:100380008E38910539F00CC047E65BE008C04FE3BA
:100390005CE005C04FE05BE002C04BE35BE03CE2A9
:1003A0009091D60A20E08091D70A281770F493170D
:1003B00060F4DA01A90FB11DE22FFF27ED53F54FCD
:1003C00085898C939F5F2F5FEECF089520E335E7FB
:1003D00080913D018B3211F08D32F9F480916E08DD
:1003E000282F33278091560490915704829FA001B3
:1003F000839F500D929F500D1124CA0163E070E05D
:100400000E9407A1CB019B01205D3A48C196C1978C
:1004100008F03FC02EEF34E73CC0803229F58091D0
:10042000250481FF36C02091700530917105205D53
:100430003A4855E72133350748F085E7243938072E
:1004400018F420E335E702C02456304045E7203356
:100450003407F8F454E72D3C350718F020E335E76E
:1004600018C02C593F4F15C08E3549F49091510456
:100470008AE0989F90011124205D3A480AC086378F
:1004800041F4909151048AE0989FC0011124281BE7
:10049000390BC9010895EF92FF920F931F9399278B
:1004A0008A38910509F478C18B38910524F489388C
:1004B000910551F023C38D38910509F462C28E383D
:1004C000910509F4BDC11AC30E945481182F80936D
:1004D000410C80915C0490915D04A0915E04B09108
:1004E0005F04BC01CD0124E630E040E050E00E9412
:1004F0003CA1DA01C9018C509E4F90936D0B809303
:100500006C0B112319F40E94E68102C080E395E789
:100510009093730B8093720B8091720B9091730B7D
:100520009093750B8093740B9093770B8093760B5D
:1005300020916C0B30916D0B8091700B9091710B31
:100540002817390724F43093710B2093700B809196
:100550006E0B90916F0B8217930724F430936F0BFF
:1005600020936E0B1092690B87E69BE090939005A9
:1005700080938F0580913D0180938D0B80912404A1
:1005800080FF02C083E401C080E280938E0B209143
:100590004805222309F1822F6AE00E94E7A0805DCE
:1005A0008093780B822F0E94E7A0892F805D809333
:1005B000790B8AE380937A0B81E1289FF001112463
:1005C000ABE7BBE0E755F44F9FE084918D939150EA
:1005D000319697FFFACF8FC28091250485FF0CC01A
:1005E000A8E7BBE0E0EDFDE094E184918D939150AC
:1005F000319697FFFACF7FC280917205882311F15F
:10060000A8E7BBE0E9ECFDE096E084918D93915082
:10061000319697FFFACF80910001805D80937C0B2B
:10062000AFE7BBE0EEECF8E09BE081918D93915059
:1006300097FFFBCF80E280938A0B80938B0B809394
:100640008C0B59C230917705332309F499C087E5A3
:100650008093780B80E58093790B40E240937A0B8E
:1006600020917805822F6AE00E94E7A0805D809348
:100670007B0B822F0E94E7A0892F805D80937C0BEB
:100680008FE280937D0B832F0E94E7A0805D809393
:100690007E0B832F0E94E7A0892F805D80937F0BC4
:1006A0004093800B209174053091750583E0293EBD
:1006B000380780F0C90168EE73E00E94F3A0CB0117
:1006C000805D8093810BC90168EE73E00E94F3A006
:1006D0009C0102C04093810B2536310580F0C90191
:1006E00064E670E00E94F3A0CB01805D8093820BF2
:1006F000C90164E670E00E94F3A09C0103C080E29F
:100700008093820BC9016AE070E00E94F3A0CB01E4
:10071000805D8093830BC9016AE070E00E94F3A0C2
:10072000805D8093840B8DE68093850B80E28093BF
:10073000860B20917605253660F0822F64E60E94B4
:10074000E7A0805D8093870B822F0E94E7A0292F6E
:1007500002C08093870B822F6AE00E94E7A0805D31
:100760008093880B822F0E94E7A0892F805D809361
:10077000890B83E780938A0B80E280938B0BBBC14C
:10078000A8E7BBE0E6EEFDE094E184918D93915003
:10079000319697FFFACFAFC180915C0490915D04D0
:1007A000A0915E04B0915F04BC01CD0124E630E06D
:1007B00040E050E00E943CA1DA01C9018C509E4FFC
:1007C0009093550C8093540C8091410C882319F41C
:1007D0000E94E68102C080E395E79093570C8093D6
:1007E000560C88E78093580C80918F0A8093590C9F
:1007F00080918E0A81FF02C084E407C08091900A34
:10080000833011F480E201C081E280935A0C8FE3BF
:100810009CE09093900580938F058091B301809325
:10082000660C80915A0C8093680C8091940A909188
:10083000950A97FD01969595879580935B0C5BC112
:100840000E94F68080915C0490915D04A0915E040A
:10085000B0915F04BC01CD0124E630E040E050E0FF
:100860000E943CA1DA01C9018C509E4F90932A0B43
:100870008093290B80912201909123019093240B66
:100880008093230B80912201909123019093260B5A
:100890008093250B80912C0A90912D0A97FD01964B
:1008A000959587958093150B80931C0B2091940A46
:1008B0003091950A37FF02C02F5F3F4F359527953E
:1008C00020931A0B8091920A9091930A64E170E050
:1008D0000E94F3A060931B0B2093210B6093220BCB
:1008E0008091410C882319F40E94E68102C080E3C4
:1008F00095E79093320B8093310B88E78093330B0D
:10090000809122019091230190932E0B80932D0BC7
:1009100080916E058C5E8093270B80916F058C5EB5
:100920008093280B80910C0B90910D0B6AE070E086
:100930000E94F3A07093300B60932F0B1092110B59
:100940008091080B9091090B90932C0B80932B0BAB
:100950008FE09BE09093900580938F052091020398
:1009600030910303C9016CE370E00E94F3A060932F
:10097000360BC9016CE370E00E94F3A08093370B43
:10098000BAC00E94F6808091920A9091930A64E620
:1009900070E00E94F3A07093510B6093500B809114
:1009A0002C0A90912D0A97FD019695958795809335
:1009B000410B8091940A9091950A97FD0196959527
:1009C00087958093460B80910101482F55279A0106
:1009D0002B5F3F4F80912201909123012817390707
:1009E00084F48091220190912301841B950B9C013A
:1009F000220F331F280F391F822F825180934D0BF6
:100A000002C010924D0BE0905C04F0905D040091E8
:100A10005E0410915F04C801B70124E630E040E0B5
:100A200050E00E943CA130934F0B20934E0B37FFB8
:100A300004C010924F0B10924E0BC801B70124E670
:100A400030E040E050E00E943CA1DA01C9018C5046
:100A50009E4F9093530B8093520B80912201909163
:100A600023019093480B8093470B80912201909132
:100A7000230190934A0B8093490B8091410C88236A
:100A800019F40E94E68102C080E395E79093550B2C
:100A90008093540B88E78093560B809122019091AC
:100AA000230190935A0B8093590B80916E058C5EB5
:100AB00080934B0B80916F058C5E80934C0B8091E3
:100AC0000C0B90910D0B6AE070E00E94F3A0709304
:100AD0005C0B60935B0B10923D0B8091080B909127
:100AE000090B9093580B8093570B8BE39BE09093EB
:100AF000900580938F052CE230E002C020E030E0CA
:100B0000C9011F910F91FF90EF900895EF92FF920E
:100B10000F931F93CF93DF93809170059091710590
:100B20009C0153E0220F331F5A95E1F7281B390B24
:100B30008091490390914A03280F391F37FF02C063
:100B4000295F3F4F43E0359527954A95E1F730936C
:100B500071052093700590918105992309F026C3B2
:100B600080918005282F3327442755278F5F809356
:100B70008005F9012131310508F015C3E857FF4F11
:100B80000C948EA18091250485FF2AC080E00E94EC
:100B9000D19980912201909123016AE070E00E9436
:100BA00007A19F938F9380912201909123016AE086
:100BB00070E00E9407A17F936F9382E19EE09F9374
:100BC0008F9384EC99E99F938F93E091B805F0910E
:100BD000B90509952DB73EB7285F3F4F2DBF28C0F7
:100BE00080E00E94D19980912201909123016AE0D6
:100BF00070E00E9407A19F938F93809122019091B2
:100C000023016AE070E00E9407A17F936F938FE158
:100C10009EE09F938F9383EA99E99F938F93E0914E
:100C2000B805F091B90509958DB79EB708968DBFA7
:100C30008091730A80FF3FC0809179048823E9F096
:100C40008AE00E94D19980913D0199279F938F93CB
:100C500080915C0490915D04A0915E04B0915F046A
:100C6000BC01CD0124E630E040E050E00E943CA110
:100C70003F932F938CE29EE09BC68AE00E94D1991D
:100C800080915C0490915D04A0915E04B0915F043A
:100C9000BC01CD0124E630E040E050E00E943CA1E0
:100CA0003F932F9388E39EE09F938F9383EA99E984
:100CB0009F938F93A4C78AE00E94D19983E49EE01A
:100CC0009F938F9383EA99E90C942A8F809125044E
:100CD00085FF2AC085E10E94D199809102039091FD
:100CE00003036CE370E00E94F3A09F938F938091C5
:100CF0000203909103036CE370E00E94F3A07F93E2
:100D00006F938DE49EE09F938F9384EC99E99F937A
:100D10008F93E091B805F091B90509952DB73EB7CD
:100D2000285F3F4F2DBF28C085E10E94D199809157
:100D30000203909103036CE370E00E94F3A09F9381
:100D40008F9380910203909103036CE370E00E9403
:100D5000F3A07F936F938AE59EE09F938F9383EA3E
:100D600099E99F938F93E091B805F091B9050995A2
:100D70008DB79EB708968DBF8FE10E94D19980E60E
:100D800090E09F938F9380912C0A90912D0A9F93CE
:100D90008F9387E69EE09F938F93C3EAD9E9DF9311
:100DA000CF93E091B805F091B9050995809124049D
:100DB0002DB73EB7285F3F4F2DBF80FF06C089E2A9
:100DC0000E94D19982E79EE06FC389E20E94D19987
:100DD00084E79EE0B5C68091250485FF1BC08AE2AA
:100DE0000E94D19980910C0B90910D0B9F938F9342
:100DF00086E79EE09F938F9384EC99E99F938F936E
:100E0000E091B805F091B90509958DB79EB70696A2
:100E10008DBF1BC08AE20E94D19980910C0B9091EA
:100E20000D0B9F938F938EE79EE09F938F9383EAA2
:100E300099E99F938F93E091B805F091B9050995D1
:100E40002DB73EB72A5F3F4F2DBF86E30E94D19951
:100E50008091080B9091090B6AE070E00E94F3A06A
:100E60009F938F938091080B9091090B6AE070E03B
:100E70000E94F3A07F936F9386E89EE09F938F93E9
:100E800083EA99E99F938F93E091B805F091B905B2
:100E900009958DB79EB70896BAC689E00E94D19988
:100EA00082E99EE09F938F9303EA19E91F930F93C2
:100EB000E091B805F091B90509958EE10E94D199AC
:100EC0000F900F900F900F9084E99EE09F938F9367
:100ED0001F930F93E091B805F091B905099583E34D
:100EE0000E94D1990F900F900F900F9086E99EE08D
:100EF0009F938F931F930F93E091B805F091B905DD
:100F000009958FE30E94D1990F900F900F900F9049
:100F100088E99EE09F938F931F930F93E091B8050C
:100F2000F091B90509958EE70E94D1990F900F9025
:100F30000F900F908EEA9EE09F938F931F930F93D5
:100F40008BC78091C101882309F462C08DE50E949E
:100F5000D19984EC9EE09F938F93C3EAD9E9DF9304
:100F6000CF93E091B805F091B905099584E50E9409
:100F7000D1990F900F900F900F9080918F0A992721
:100F80009F938F9386EC9EE09F938F93DF93CF93F5
:100F9000E091B805F091B90509958EE50E94D199C7
:100FA0002DB73EB72A5F3F4F2DBF8091920A909197
:100FB000930A6AE070E00E94F3A07F936F938FEC36
:100FC0009EE09F938F93DF93CF93E091B805F091CC
:100FD000B90509958DB79EB706968DBF8091900A89
:100FE000833081F480918E0A81FF06C08BE50E94D8
:100FF000D19989ED9EE0A4C58BE50E94D1998CED35
:101000009EE09EC58BE50E94D1998FED9EE01EC7A4
:1010100084E0CFC38091C101882309F47AC0809114
:10102000830593EAE92E99E9F92E882309F44BC048
:1010300089E60E94D1998091470599279F938F93C4
:1010400082EE9EE09F938F93FF92EF92E091B8051E
:10105000F091B905099585E70E94D1992DB73EB762
:101060002A5F3F4F2DBF8091B30199279F938F93A4
:1010700000E610E01F930F938091940A9091950AD7
:101080009F938F938DEE9EE09F938F93FF92EF92AD
:10109000E091B805F091B905099582E70E94D199D0
:1010A0008DB79EB70A968DBF8091450599279F936E
:1010B0008F931F930F938091460599279F938F934A
:1010C00089EF9EE064C689E60E94D1998091B301C0
:1010D00099279F938F9380E690E09F938F938091C1
:1010E000940A9091950A9F938F938091910A9927E2
:1010F0009F938F9389E09FE09F938F93FF92EF924E
:10110000E091B805F091B90509958DB79EB70C9699
:101110007EC585E04EC3909148059923D1F080911A
:101120008C05882381F0903270F487E00E943C8126
:1011300083E90E94D1998091480599279F938F93C5
:1011400082E29FE0A0C383E90E94D1998DE29FE0F3
:10115000AFC38091250403EAE02E09E9F02E85FF54
:1011600006C084E90E94D19983E39FE0D6C383E956
:101170000E94D19986E49FE0D0C38091A40C863070
:1011800059F480918305882319F0109283058BC64A
:1011900081E08093830587C6883009F084C60E9469
:1011A000D69981E0D7C39093800585C6913009F028
:1011B000DCC380918005282F3327442755278F5F74
:1011C00080938005F9012131310508F06FC6E7569B
:1011D000FF4F0C948EA18091250485FF43C080E0D1
:1011E0000E94D19980910C0B90910D0B9F938F933E
:1011F00080912201909123016AE070E00E9407A192
:101200009F938F9380912201909123016AE070E077
:101210000E9407A17F936F93809102039091030333
:101220006CE370E00E94F3A09F938F938091020380
:10123000909103036CE370E00E94F3A07F936F939F
:101240008CE59FE09F938F9384EC99E99F938F9314
:10125000E091B805F091B90509952DB73EB7225F29
:101260003F4FA2C580E00E94D19980910C0B9091D4
:101270000D0B9F938F9380912201909123016AE03F
:1012800070E00E9407A19F938F938091220190911B
:1012900023016AE070E00E9407A17F936F93809121
:1012A0000203909103036CE370E00E94F3A09F930C
:1012B0008F9380910203909103036CE370E00E948E
:1012C000F3A07F936F9387E79FE0BEC285E10E9402
:1012D000D19980E690E09F938F938091AD0190919A
:1012E000AE019F938F9382E99FE09F938F93C3EA10
:1012F000D9E9DF93CF93E091B805F091B90509954D
:101300008091730A2DB73EB7285F3F4F2DBF80FFF6
:1013100051C080917904882339F18FE10E94D199DD
:1013200080915C0490915D04A0915E04B0915F0493
:10133000BC01CD0124E630E040E050E00E943CA139
:101340003F932F938CE99FE09F938F9383EB99E9D1
:101350009F938F93E091B805F091B90509958DB7EA
:101360009EB706968DBF38C08FE10E94D1998091BB
:101370005C0490915D04A0915E04B0915F04BC0197
:10138000CD0124E630E040E050E00E943CA13F93D4
:101390002F9385EA9FE09F938F93DF93CF93E09104
:1013A000B805F091B90509952DB73EB72A5F3F4FB3
:1013B0002DBF12C08FE10E94D1998EEA9FE09F93CA
:1013C0008F93DF93CF93E091B805F091B90509951C
:1013D0000F900F900F900F9089E20E94D199809109
:1013E0003D0199279F938F9388EB9FE004C48091E0
:1013F000C1018823F9F08BE20E94D1998091B30159
:1014000099279F938F938091920A9091930A6AE013
:1014100070E00E94F3A07F936F9380E690E09F932B
:101420008F938091940A9091950A9F938F938BEB61
:101430009FE058C182E0BDC18FE30E94D1998091A5
:101440000A0B90910B0B9F938F938091080B9091B7
:10145000090B6AE070E00E94F3A09F938F93809144
:10146000080B9091090B6AE070E00E94F3A07F9353
:101470006F9382ED9FE09F938F93C3EAD9E9DF9347
:10148000CF93E091B805F091B905099580912404B6
:101490002DB73EB7265F3F4F2DBF80FF0AC082E5C4
:1014A0000E94D19986EE9FE09F938F9383EB99E9F9
:1014B000D1C482E50E94D19989EE9FE041C3809119
:1014C000C10113EAE12E19E9F12E882309F449C07C
:1014D00084E50E94D19980918F0A99279F938F93D9
:1014E0008091910A99279F938F938CEE9FE09F9311
:1014F0008F93E701FF92EF92E091B805F091B90563
:1015000009958DB79EB708968DBF8091900A83305C
:1015100051F484E60E94D1998FEF9FE09F938F93BF
:10152000FF92EF920BC084E60E94D19985E090E192
:101530009F938F9384EC99E99F938F93E091B805E3
:10154000F091B90509950F900F900F900F90809131
:101550008E0A81FFB0C484E60E94D1998BE090E1AD
:10156000EFC284E50E94D19981E190E1D6C18091DA
:101570008205C3EAEC2EC9E9FC2E882309F450C089
:1015800089E60E94D19980914E096AE00E94E7A005
:10159000892F99279F938F9380914E090E94E7A0EE
:1015A00099279F938F93809146090E94E7A0892FE6
:1015B00099279F938F93809146090E94E7A09927CE
:1015C0009F938F9380913E090E94E7A0892F9927CE
:1015D0009F938F9380913E090E94E7A099279F9344
:1015E0008F93809136090E94E7A0892F99279F93B6
:1015F0008F93809136090E94E7A099279F938F933C
:1016000087E290E19F938F93FF92EF92E091B8056C
:10161000F091B90509952DB73EB72C5E3F4FC4C375
:1016200089E60E94D19980E690E09F938F93809104
:101630005009992787FD90959F938F938091480932
:10164000992787FD90959F938F93809140099927C3
:1016500087FD90959F938F9380913809992787FDF7
:1016600090959F938F9384E490E19F938F93FF9243
:10167000EF92E091B805F091B90509958DB79EB745
:101680000E96C5C28091820590915B08882309F46B
:101690008DC0943009F48CC09630A1F58EE70E947D
:1016A000D19980915E096AE00E94E7A0892F99276D
:1016B0009F938F9380915E090E94E7A099279F9343
:1016C0008F93809156090E94E7A0892F99279F93B5
:1016D0008F93809156090E94E7A099279F938F933B
:1016E00087E590E19F938F9383EA99E99F938F9386
:1016F000E091B805F091B90509952DB73EB7245F83
:101700003F4F52C3973008F4D6C38EE70E94D19959
:1017100080916E096AE00E94E7A0892F99279F9324
:101720008F9380916E090E94E7A099279F938F93D2
:10173000809166090E94E7A0892F99279F938F9334
:10174000809166090E94E7A099279F938F938091CB
:101750005E090E94E7A0892F99279F938F9380911C
:101760005E090E94E7A099279F938F938091560965
:101770000E94E7A0892F99279F938F938091560904
:101780000E94E7A099279F938F9386E690E19F930D
:101790008F9383EA99E99F938F93E091B805F09135
:1017A000B90509958DB79EB7449631C2943021F49E
:1017B00086E00E943C817FC39630F1F48EE70E9460
:1017C000D19980E690E09F938F938091600999274B
:1017D00087FD90959F938F9380915809992787FD56
:1017E00090959F938F9383E890E19F938F9383EAE3
:1017F00099E99F938F93CFC2973008F45CC38EE72B
:101800000E94D19980E690E09F938F938091700918
:10181000992787FD90959F938F93809168099927C9
:1018200087FD90959F938F9380916009992787FDFD
:1018300090959F938F9380915809992787FD909554
:101840009F938F9386E990E19F938F9383EA99E921
:101850009F938F930ECF90914805992309F44AC026
:1018600080918C058823F9F09032E8F487E00E949B
:101870003C8183E90E94D1998091480599279F93E3
:101880008F9389EA90E19F938F9383EB99E99F93DC
:101890008F93E091B805F091B90509952DB73EB742
:1018A0002A5F3F4F81C283E90E94D19984EB90E186
:1018B0009F938F9303EA19E91F930F93E091B80563
:1018C000F091B90509951F921F929091480581E109
:1018D000989FC00111248755944F9F938F931F9316
:1018E0000F93E091B805F091B90509958DB79EB7B2
:1018F0000A968DC180912504B3EAEB2EB9E9FB2E3F
:1019000085FF06C084E90E94D1998AEB90E105C069
:1019100083E90E94D1998DEC90E19F938F93FF9280
:10192000EF929AC28091A40C863079F4809182055E
:10193000882319F01092820503C081E0809382050C
:1019400085E00E943C8186E0A3C2883031F40E9489
:10195000D69982E080938105A4C2813009F0A3C2A8
:101960000E94D699109281059CC2923009F0A1C2C2
:1019700080918005282F3327442755278F5F809338
:101980008005F9012131310508F090C2E655FF4F7D
:101990000C948EA180E00E94D1998EEC98E09F93E8
:1019A0008F938091000199279F938F9383EE90E10D
:1019B0009F938F9383EB99E99F938F93E091B80561
:1019C000F091B90509952DB73EB7285F3F4FECC19F
:1019D00085E10E94D1998CED98E09F938F9380913F
:1019E00001016AE00E94E7A0892F99279F938F93B6
:1019F000809101010E94E7A099279F938F9382EF26
:101A000090E19F938F9383EA99E99F938F93E0915D
:101A1000B805F091B905099569CF8AE20E94D1997C
:101A200083E091E19F938F93C3EAD9E9DF93CF934A
:101A3000E091B805F091B90509958091730A0F906E
:101A40000F900F900F9080FF41C080916908909196
:101A50003F0481FD0BC0892F99279F938F9388E0C6
:101A600091E19F938F93DF93CF9313CFE091B805CC
:101A7000F091B905933318F082E191E102C089E158
:101A800091E19F938F93DF93CF9309950F900F90E0
:101A90000F900F908091540AE091B805F091B9052C
:101AA00090913F0480FF0BC0892F99279F938F93BC
:101AB00080E291E19F938F93DF93CF93A4C0892F0E
:101AC00099279F938F9386E291E1C4C08CE291E1C4
:101AD00037C08FE30E94D19985E391E19F938F9363
:101AE000C3EAD9E9DF93CF93E091B805F091B90546
:101AF00009950F900F900F900F908091BF08882349
:101B000019F489E391E11CC080913604E091B80595
:101B1000F091B905882319F082E491E102C089E4CB
:101B200091E19F938F93DF93CF9309950F900F903F
:101B30000F900F908091CC0886FFBDC180E591E1A8
:101B40009F938F93DF93CF9387C184E50E94D199B0
:101B500087E591E19F938F93C3EAD9E9DF93CF9310
:101B6000E091B805F091B90509958091730A0F903D
:101B70000F900F900F9085FD03C08CE591E108C098
:101B80008091AD080E948A49823358F485E691E13C
:101B90009F938F93DF93CF93E091B805F091B905B0
:101BA00016C0843B18F08CE691E1F2CF8091CC080E
:101BB000E091B805F091B90585FF03C083E791E195
:101BC00002C08AE791E19F938F93DF93CF930995AA
:101BD0000F900F900F900F908091C308882309F405
:101BE0006AC18EE50E94D1998091C30899279F937D
:101BF0008F9381E891E19F938F93DF93CF93E0914F
:101C0000B805F091B90509958DB79EB706968DBFB9
